:1000000000800020BD010000099D0000C19C00008F
:10001000C19C0000C19C0000C19C0000C19C00006C
:10002000C19C0000C19C0000C19C0000099D000013
:10003000099D0000C19C0000899300008D94000080
:10004000099D0000099D0000099D0000099D000018
:10005000099D0000099D0000099D0000099D000008
:10006000099D0000099D0000099D0000099D0000F8
:10007000099D0000099D0000099D0000099D0000E8
:10008000099D0000099D0000099D0000099D0000D8
:10009000099D0000099D0000099D0000099D0000C8
:1000A000C5780000D1780000099D0000099D00007E
:1000B000099D0000099D0000099D0000099D0000A8
:1000C000099D0000099D0000099D0000099D000098
:1000D000099D0000099D0000099D0000099D000088
:1000E000099D0000099D0000099D0000099D000078
:1000F000099D000075BD0000099D0000A1BE000023
:10010000099D0000E1A60000099D0000099D000076
:10011000099D0000099D0000099D0000099D000047
:10012000099D0000099D0000099D0000099D000037
:10013000099D0000099D0000099D0000099D000027
:10014000099D0000099D0000099D0000099D000017
:10015000799500008D950000A1950000B5950000EF
:10016000099D0000FDA90000099D0000099D0000F7
:10017000099D0000099D0000099D0000099D0000E7
:10018000099D0000099D0000099D0000099D0000D7
:10019000099D0000099D0000099D0000099D0000C7
:1001A000099D0000099D0000099D0000099D0000B7
:1001B000099D0000099D0000099D0000564B4CF26E
:1001C000205210B51A804DF628121A8000BF00BFC9
:1001D00009F09EFD514B4FF010621A60504A9A6030
:1001E000504ADA60504A136813F4807304D14F49BF
:1001F0000B604FF4A85313604D4B1A78110703D5C9
:100200001A7842F008021A704A4B4B492A221A7097
:100210004A4A4B4B8B4204D252F8040F43F8040B6A
:10022000F8E7484B484900228B4202D243F8042B9E
:10023000FAE74649464A002352F8230041F82300D2
:1002400001336F2BF8D1434B434A802103F8011B44
:100250009342FBD1414B3D4A1A60414B8A221A70AE
:10026000A3F5805324225A70A0221A709A7992071B
:10027000FCD59A79D406FCD43A4A937903F00C035E
:10028000082B384BF9D103221A7140225A719A79FE
:100290009006FCD5334A9179324B4906FBD5324A58
:1002A000324911600221516020221A709A7902F0BD
:1002B0000C020C2AFAD12E4B2E4A1A602E4B2F4AD2
:1002C0001A6000225A60072243F8042C2C4AC3F813
:1002D0000C2D62B60AF0CCF8144B1B68DA0705D572
:1002E000284809F099FE284B284A1A60284B1B78A9
:1002F0005B0609D5244C254B22689A4204D121483B
:1003000009F08AFE002323600DF082F809F006FD53
:1003100009F034FCFEE700BF0E20054030800440A9
:10032000823F04000100002B10D0034014D0034092
:1003300002D0074000E007404C9AFF1FA4000100D4
:100340004088FF1F4C9AFF1F34A1FF1F0082FF1F30
:100350000000000000E400E05FE400E008ED00E0E1
:100360000050064000400640448004400000030165
:1003700004800440C010050014E000E0FF76010096
:100380000000202094A6B05D1CE00340A5C3945A51
:1003900000F00740FFFFFFFFFFFFFFFFFFFFFFFF32
:1003A000FFFFFFFFFFFFFFFFFFFFFFFFFFFFFFFF5D
:1003B000FFFFFFFFFFFFFFFFFFFFFFFFFFFFFFFF4D
:1003C000FFFFFFFFFFFFFFFFFFFFFFFFFFFFFFFF3D
:1003D000FFFFFFFFFFFFFFFFFFFFFFFFFFFFFFFF2D
:1003E000FFFFFFFFFFFFFFFFFFFFFFFFFFFFFFFF1D
:1003F000FFFFFFFFFFFFFFFFFFFFFFFFFFFFFFFF0D
:10040000FFFFFFFFFFFFFFFFFFFFFFFFDEF9FFFF23
:1004100010B5054C237833B9044B13B10448AFF33E
:1004200000800123237010BD4C9AFF1F00000000C4
:10043000A8000100084B10B51BB108490848AFF3EC
:1004400000800848036803B910BD074B002BFBD0A0
:10045000BDE81040184700BF00000000509AFF1F81
:10046000A80001004C9AFF1F0000000038B50446A8
:10047000104621700A491D460CF0ACFD01464FF0B4
:100480007E500CF05BFE07490CF0A4FDE560606057
:100490002561656109F07CFFE061204638BD00BF41
:1004A000DB0FC9400024744938B50446104621705A
:1004B00009491D460CF08EFD01464FF07E500CF0B0
:1004C0003DFE06490CF086FDE560606025616561D2
:1004D00009F05EFFE06138BDDB0FC94000247449BC
:1004E00038B503780446032B20D8DFE803F01A1848
:1004F0001002C16840690CF063FC0D490546606854
:100500000CF01CFE014628460CF018FE38BD0849C8
:1005100040680CF013FEE1680CF05CFD38BDC0686B
:1005200038BDC16840690CF04BFC38BD002038BDB7
:100530000024744970B504460E4609F029FF0546AB
:10054000E069281A0CF0F2FCE3682361E56166615A
:10055000A061014660680CF0F1FD0146A060104802
:100560000CF0ECFD0CF0C2F80BF062FD0CF0D4FBCB
:10057000054601464FF07E500CF022FC61690CF0FC
:1005800029FD2169064628460CF024FD0146304627
:100590000CF018FCE0602046BDE87040FFF7A0BFFB
:1005A000000080BF08B50E2009F0C2F9114B1B886E
:1005B000012B19D0104B1B88984213DB40F6FF71BA
:1005C0008842D4BFC3EB0001C3EB0101C1EB013191
:1005D000C3F57F630F33282091FBF3F1BDE808409A
:1005E00009F02CBD0021F3E70146BDE808401420C6
:1005F00009F024BD5A9BFF1FEE9AFF1F10B5044659
:1006000008F098FF204610BD70B44C88A04220D955
:1006100001230133DBB21CB2660031F8144084427E
:100620001D46F6D3A04211D005F10045013D965B71
:1006300031F8151032F81530401AF21A00FB02F0AA
:10064000641A90FBF4F4E01870BC7047905B70BCC7
:10065000704702260125E5E700280CDA064A4342E6
:1006600082FB0320DA17C2EB600000EB4000A3EB33
:100670008000C0F10C007047ABAAAA2A2DE9F04710
:100680000C2009F021F90C2009F0D6FD9549142021
:1006900009F0E2FD9449954806F01AFE0221032074
:1006A00009F070FE0221042009F06CFE02210520F1
:1006B00009F068FE0221062009F064FE01210A20EB
:1006C00009F060FE0121092009F05CFE01210D20E6
:1006D00009F058FE0121282009F054FE01211420C0
:1006E00009F050FE02210B2009F04CFE01210C20E4
:1006F00009F048FE0C20002109F030FE042009F02A
:1007000033FE70B3052009F02FFE044680B30024A9
:100710002046774D287004F04DFB2B78EBB920462E
:1007200005F00EFE734B74491B88744C0988744A9B
:100730002170A3F5AF7140F23A7303FB01F382FB22
:100740000312DB176F4D7048A3EB621332335A214B
:100750002B6007F067F990B9FEE7BDE8F04706F0B7
:10076000C7BC062009F000FE0028CBD10124D0E749
:10077000032009F0F9FDB0FA80F04009C9E7634AA7
:1007800063481268DFF8D8A100230121FFF78CFE2F
:100790000B2009F0E9FD011E0CBF012300238AF89C
:1007A000003002D1112009F0EDFDDFF87481594EBF
:1007B000594F5A4D0023C8F8003033603B604FF06A
:1007C000040914E009F0B4F833681844306009F003
:1007D000010080F0010003F029FA2B88002B14BFE0
:1007E0004B20FA2009F0F6FDB9F1010919D00F20CC
:1007F00009F0E2FF3B6803440E203B6009F098F8E3
:10080000D8F800309AF800200344C8F800301520CA
:10081000002AD7D1112009F0CFFF33681844306087
:10082000D5E73B68D8F800203D493068DFF834E16F
:100830002D88002BB8BF0333002AB8BF03329210B3
:100840000A603849384A0988128800284FEAA30309
:10085000B8BF03303B608010344F30605E1A1944DB
:100860003E60CEF80010324F324E3349C2EB000EDC
:100870000244C7F800E032600B605DB94FF4FA70D3
:1008800003F0E4F903F0CEF904F052FD40F2DC503D
:1008900009F0A0FD294B012504201D6009F064FD2D
:1008A00010B9274B20701D70264B1B881C2B0FD0B6
:1008B000254A264B1078187005F04CFC03F0AEF971
:1008C00045F6BF5222492348BDE8F04708F0E8BD8D
:1008D000214B18880028EBD0204BC0B2197805F0C6
:1008E00081FBE5E7001B3746801A0600548FFF1F87
:1008F000AC9BFF1F5C9BFF1FA29AFF1FCD9BFF1F9E
:10090000B5814E1BA489FF1F889BFF1F2089FF1FF5
:10091000F49AFF1FBC9AFF1FAC9AFF1FEE9BFF1FAC
:10092000549BFF1FA089FF1FA889FF1FA89BFF1FC3
:10093000289BFF1F909BFF1F409BFF1F949AFF1F48
:100940001A9BFF1FF09AFF1F3A9BFF1F7E9BFF1F02
:10095000A50500002C9BFF1FA09AFF1FCC9AFF1F2C
:10096000EA9BFF1FC89BFF1FF0B40E8886420DD282
:1009700003F10043013B31F81350854202D9F0BC2A
:10098000FFF742BE32F81300F0BC70471088F0BC8D
:10099000704700BF094B1B880C2B09D8084A80B24E
:1009A00052F8232028B143F6FE73984203D9108CE5
:1009B0007047108870470349FFF726BE5E9BFF1FF4
:1009C00048E6000004E50000374A38491088384AF4
:1009D000F8B5384B12881B68834248DB9342A8BFA6
:1009E000134698420B60C8BF002342DD101AB0F5D1
:1009F000804FAABF9B03C3EB8333013093FBF0F01E
:100A0000FFF7C8FF2C4B2D4F1C883B68C0F3C61561
:100A100005FB04F47F2CA8BF7F249D42064608D026
:100A2000274B1B88002B38D1264B1B88002B30D13D
:100A30003D60254D2B689E4205D0214B1B885A1FD7
:100A4000032A1DD92E60214D2B689C420ED0204BCD
:100A5000188848B11A4B1F4A1B88D35C834203D0C5
:100A6000C0B2E1B205F0BEFA2C60F8BDF8BD034695
:100A700008609A42D4BFC0EB0203C0EB0303B5E7A2
:100A8000144AD05C2030C0B206F07F0105F0AAFA0B
:100A9000D8E7284605F01AFBCAE70E4A2946D05C7B
:100AA00005F0A0FAC0E700BFEE9AFF1FE49AFF1F0F
:100AB000FA9BFF1F889AFF1F9E9AFF1F749AFF1FC1
:100AC000849AFF1F709BFF1FC09AFF1F6C9AFF1F25
:100AD0007C9BFF1F2889FF1F2DE9F04F172089B04D
:100AE00009F06AFEA34B1860162009F065FEA24BC0
:100AF000A24A1B8810600C2B00F05B83DFF8C492C5
:100B00009F4AB9F800109F4B52F8214000221A70FA
:100B10009D4B9E4D1B889E4A2E88013B32F91370D7
:100B2000002E5CD09B4B9C4A1B889C491278013B51
:100B300031F91380002A40F0DE80112009F03CFEDC
:100B4000974B0093D3F800A00646B24540F3DE80F1
:100B5000944BDFF874B21B88934A9449128802922E
:100B6000012BDBF8003001912046C8EB030800F0B0
:100B70007D820CF0DBF9029A019951F822100CF0F9
:100B800029FA014600200CF01BF90CF0E9FBCAEB36
:100B90000802B045B8BFB0469042CAEB080880F2E0
:100BA000798200FB0888013298FBF2F0804BDFF875
:100BB0001C820193D8F80030034403EBD3735B101D
:100BC000C8F800302B88012B11D17A4B04937A4A54
:100BD0001D687A4B029203934FF0000A47E0704B76
:100BE0000093DFF8E4B1724BDFF8E0810193724BC0
:100BF00002931D460F2009F0DFFD2B6898428246C4
:100C000041DA684A1288012A00F00182664A059397
:100C10001288684B654D0392204604930CF086F9C8
:100C2000039A644B55F822101D680CF0D3F9014665
:100C300000200CF0C5F80CF093FBEF1B059B57450B
:100C4000A7EB0302B8BF5746FF1A9042BABF013262
:100C500000FB0777474397FBF2F7D8F80020574B84
:100C60000393BB1803EBD3735B10C8F80030544BED
:100C70001B88013B032B00F29582DFE813F06B0128
:100C80004801A9008E014D4B03931B68984240F325
:100C9000A781444A1288012A00F0A782424A07939A
:100CA000444B1188414A1D680493204606910592E1
:100CB0000CF03CF9059A069952F821100CF08AF9CB
:100CC0000CF04EFB079B2F445745A7EB0302A8BF30
:100CD0005746FF1AD8F800309042BABF00FB07779A
:100CE0000132474397FBF2F73B4403EBD3735B10AE
:100CF000C8F80030BBE7152008F01AFE284B009317
:100D0000D3F800A00646B2453FF722AF284B019327
:100D1000D3F800A0B24580F26E81224BDFF8A8B074
:100D20001B88214A012BDBF8003000F07882128802
:100D30001E4903922046029198440CF0F7F802995C
:100D4000039A51F822100CF045F90CF009FBB0455C
:100D5000CAEB0802A8BFB046CAEB08089042B6BF6B
:100D600000FB088800FB08F8013298FBF2F0DFF87E
:100D70005C801FE77C9AFF1FF09AFF1F449BFF1FB8
:100D80003C89FF1FB69AFF1F7889FF1F829AFF1FB9
:100D9000C8E600007A89FF1FEA9BFF1FE0E600001B
:100DA000289BFF1FF69BFF1F369BFF1FA0E600003E
:100DB000909BFF1FAC9AFF1FA89BFF1FC89BFF1FA4
:100DC000AA89FF1F829BFF1FBC9AFF1F989AFF1FD3
:100DD00028460CF0ABF8B2490CF0FCF8054650463A
:100DE0000CF0A4F8AF490CF0F5F8014628460BF0DA
:100DF000E9FF0CF0B5FA049B05461D60DBF8000026
:100E00000CF094F8A6490CF0E5F8074630460CF0D3
:100E10008DF8A4490CF0DEF8014638460BF0D2FFFD
:100E20000CF09EFACBF800009F4AA04B1688198858
:100E30009F4AA04B12681B889F4FC6EB050E354496
:100E4000029EC6F800E0461A084403990D60009916
:100E50000E6001993E8808609A4280F289810025DF
:100E6000C3EB060E954974450F6880F27681611CCC
:100E70009F4205FB01F50EF1010E95FBFEF5C0F258
:100E8000E181BE42A8BF3E46F61A01FB06F494FB80
:100E9000FEF49A4200F33681BB42C0F23381884CA3
:100EA00020680CF043F887490CF094F886490BF061
:100EB00089FF0CF055FAA0F5FF531C3B082B98BF97
:100EC0004FF40050D8F80030184400282060C0F2D9
:100ED0004281B0F5804F80F252817C4B1B781BB170
:100EE000B0F5005F40F05381794D2B78002B40F036
:100EF0005481784D20682B68714C984204D080B2A0
:100F000005F04EF923682B6009B0BDE8F08F284644
:100F10000CF00CF870490CF05DF8054650460CF0EA
:100F200005F86E490CF056F8014628460BF04AFFCA
:100F30000CF016FA049B05461D60DBF800000BF070
:100F4000F5FF65490CF046F8074630460BF0EEFF1A
:100F500062495FE728460BF0E9FF61490CF03AF877
:100F6000054650460BF0E2FF5E490CF033F80146AF
:100F700028460BF027FF0CF0F3F9049B05461D6093
:100F8000DBF800000BF0D2FF55490CF023F80746C0
:100F900030460BF0CBFF53493CE728460BF0C6FF29
:100FA00048490CF017F8054650460BF0BFFF4E4974
:100FB0000CF010F8014628460BF004FF0CF0D0F9B5
:100FC000049B05461D60DBF800000BF0AFFF3D49B8
:100FD0000CF000F8074630460BF0A8FF424919E72D
:100FE000D8F80030414A049203EBD3735B101568C4
:100FF000C8F800303BE6DFF80481DFF804B1D8F828
:10100000003003EBD3735B10C8F80030DAE5384AE0
:101010000693364B1188374A1D6804932046059184
:1010200003920BF083FF039A059952F821100BF0FD
:10103000D1FF0CF095F9EF1B069B5745A7EB030278
:10104000B8BF5746FF1AD8F800309042BABF0132F5
:1010500000FB0777474397FBF2F73B4403EBD3735F
:10106000254A03925B10C8F8003000E60BF05EFFE3
:10107000029A019951F822100BF0ACFF0CF070F9B4
:10108000CAEB0802B045B8BFB0468242CAEB0808B6
:101090003FF787AD00FB08F898FBF2F086E500BF4C
:1010A000CDCC4C3FCDCC4C3EA089FF1FA889FF1F63
:1010B0007C9AFF1FE89BFF1F589BFF1F449BFF1F4D
:1010C0007489FF1F9A99193FCDCC4C457A9CFF1F1C
:1010D0009D9AFF1F2489FF1F6666663FCDCCCC3DDD
:1010E0003333733FCDCC4C3DCDCCCC3EAC9AFF1FBF
:1010F000369BFF1FA0E60000C89BFF1F989AFF1FAA
:10110000BC9AFF1FB9F80030002B3FF4C8AE2B1B70
:10111000002BB8BF5B42092B47DD05F500500130BD
:10112000001B0BF003FF4D494D4C0BF053FF0546E0
:1011300020680BF0FBFE4B490BF04CFF01462846A4
:101140000BF040FE0CF00CF9D8F8003018440028E1
:101150002060BFF6BEAE002213E09F4205FB04F5FF
:10116000B8BF002195FBFEF56EDA91FBFEF490E628
:10117000B242D4BFC3EB0205C3EB060570E643F6EB
:10118000FF72394B22601B78002B3FF4ADAE02F0AA
:1011900049FD364B01221A70ABE602F03FFD0023F9
:1011A0002B70A6E6DBF800003EE64FF400502C4C16
:1011B00088E6012009F000FB2D4B1B6898427FF761
:1011C0009DACDFF8C4902B4AB9F800102A4B52F8B6
:1011D000210001221A700BF0A9FE4FF07C510BF098
:1011E000F9FE0CF0BDF8044692E42449244A069323
:1011F0002046244B0D88059204930BF097FE059A28
:10120000049B52F825101D680BF0E4FE01460020F7
:101210000BF0D6FD0CF0A4F82F44069B54E5118882
:10122000174A03912046029298440BF07FFE029ADF
:10123000039952F821100BF0CDFE014600200BF06F
:10124000BFFD82E51E461FE6B742D4BFC3EB0701D0
:10125000C3EB060104FB01F187E700BFCDCCCC3E18
:101260007489FF1F9A99193F7A9CFF1F9D9AFF1F4F
:10127000A489FF1F3C89FF1FB69AFF1F369BFF1FE3
:10128000A0E60000AC9AFF1F829BFF1F08B5244B0D
:101290001B88FBB1234B1B78FBB1234B1B78E3B1BD
:1012A000224B1B78CBB1224B1B78B3B1214B224888
:1012B0001A78C2B9214A2249008812880968024472
:1012C000B1EB620F09DD01221A706420BDE808400D
:1012D00002F0BCBC174A117801B908BD1370BDE813
:1012E000084004F027BF154A16490088128809688B
:1012F0000244B1EB620FF0DD00221A7004F01AFF15
:10130000642002F0A3FC642002F0A0FC642002F040
:101310009DFC4FF41670BDE8084009F05BB800BFB3
:10132000A89AFF1FE89AFF1FA59AFF1FA69AFF1F02
:10133000A79AFF1F909AFF1F589BFF1FE89BFF1F54
:101340007C9AFF1F449BFF1F2DE9F84FAB4C206890
:101350000BF0ECFDAA490BF03DFE0546102009F00C
:101360002BFA0BF0E3FDA7490BF034FE29460BF0F6
:1013700029FD0BF0F5FFA44B20601B88192B00F012
:101380008C801A2B00F0A4800126B1469F4D2B883B
:10139000002B2DD020689E4F3A88824233DD9D4A33
:1013A0001178002977D00024012B147000F09D8063
:1013B000022B40F03F81002E00F09D80964D2B685F
:1013C000002B00F098800420214604F00BFE934B84
:1013D0002C60188800285ED0B9F1000F5BD0C0B235
:1013E000002104F0FFFD8E4B00221A60BDE8F88F4B
:1013F0008A4A1288002ACDD1864B1978002972D0EA
:101400001A70BDE8F88F834991F80080B8F1000F99
:1014100033D14FF0010E042B81F800E02DD1002EC6
:1014200040F02C812B88022B01D0032B66D07B4B04
:10143000188800282FD0B9F1000F2CD023683C88E1
:10144000784AA342128880F2D1800023141B7E2C9C
:10145000734DD5BFC3EB8313C3EBC3135B000134E0
:1014600093FBF4F42B680134A34203D0C0B2E1B281
:1014700004F0B8FD2C60BDE8F88F2B88012B67D0F5
:10148000022BD2D1002ED2D0DFF88CB1DFF894A19C
:10149000DBF8003087E0BDE8F88F634D634F2B78B1
:1014A0004BB15E4A128832B13978994200F0D98046
:1014B000D0B27F2105E03A789A4246D0574B18784F
:1014C000002104F08FFD00262B783B70B1465DE7CC
:1014D000554B1B78002B0BBF012600264FF000094F
:1014E0004FF0010952E7BDE8F88F26B14A4D2A684E
:1014F000002A40F0BB80494B18886BE74C4B1B8897
:10150000092B94D0002E92D023683D88454AAB42E7
:10151000128880F2D9800023551B7E2DDFF8F8B0A9
:10152000D5BFC3EB8313C3EBC3135B00013593FB40
:10153000F5F5DBF800300135AB4203D0E9B24A20C3
:1015400004F050FDCBF8005071E70026B1461DE7CE
:10155000002E3FF46CAFDFF8CCA0BAF80030984210
:10156000D4BFC2EB0008C2EB03089A1A7E2A40F3EC
:10157000A280C8EBC81002F1010890FBF8F808F14E
:101580000108DFF894B0DBF80030434504D05FFA7F
:1015900088F1012004F026FD2B88CBF80080022B77
:1015A0007FF443AF43462268B7F80080BAF80010D2
:1015B000424579DA0022C8EB0108B8F17E0FD3BFAB
:1015C000C2EB8212C2EBC21208F10108520092FB78
:1015D000F8F808F10108984504D05FFA88F1042072
:1015E00004F000FD2B88CBF800801EE79342D4BFA7
:1015F000C4EB0303C4EB020328E700BF489BFF1FB3
:101600009A99193FCDCCCC3EF09AFF1FAE9BFF1F9D
:10161000B49BFF1FA49AFF1FB89AFF1F709AFF1F69
:10162000E09AFF1F269BFF1FE09BFF1F169BFF1FDB
:10163000849AFF1F032B2CD12C4B1B88092B3FF4C2
:101640005AAF002E3FF457AF294D2B68002B3FF4C3
:1016500052AF4A20214604F0C5FC264B2C60188866
:10166000B8E6254D00262B88B14694E6184621465B
:1016700004F0B8FC1F4B2C601888ABE67F2140209B
:1016800004F0B0FC2B88012B25D0022B7FF4CDAECB
:10169000FAE6042B7FF42FAF002E3FF42CAF214647
:1016A000402004F09FFC26E78A42D4BFC8EB020228
:1016B000C8EB01027FE7C8EB88184FEA480898FB9F
:1016C000F2F808F101085CE79342D4BFC5EB0303CD
:1016D000C5EB020320E720683A88DFF820A090429B
:1016E000BAF80030FFF641AF39E700BF849AFF1F18
:1016F000B89AFF1F709AFF1FAE9BFF1F269BFF1F0C
:1017000038B51C4B1B881D2B26D01B4B1B88012B6F
:1017100025D01A4A1A4B14881B681A4AA342128809
:1017200018DB9342D4BFC4EB0303C4EB0203141BC6
:101730007F2CC6BFDB010134C3EBC31393FBF4F46E
:10174000114D2B689C4203D0E1B2052004F04AFC05
:101750002C6038BD0023EAE70C4B1C88F0E70C4BEB
:101760000C4A0D491B6812680C689B1A1C1B84F3F9
:101770000704E5E7F09AFF1F829AFF1F949BFF1F63
:10178000C49BFF1FEA9AFF1F849BFF1FCC9AFF1F79
:10179000409BFF1F3489FF1FBC9BFF1F10B50C4CE3
:1017A000236843B90B4B1B88022B0CD00A4A002339
:1017B0001370236010BD0021052004F013FC054BBD
:1017C0001B88022BF2D10021412004F00BFCEDE735
:1017D000849BFF1F249BFF1FB89BFF1F10B5304B3E
:1017E0001B78ABB1152008F0A3F82E4A2E4B1288B7
:1017F00018601D2A15D02D4A12881AB3012A3AD032
:101800002B4B1B78002B35D0BDE81040FFF7C6BF2F
:10181000112008F0D1FF234A234B128818601D2A9B
:10182000E9D1244B1B78002BEAD0214C23782BB92B
:10183000214B1B88022B14D001232370BDE81040DC
:10184000FFF75EBF1C4A1288002AD9D01B491B68CB
:1018500009889942D4DC164C2378002BEED1022A59
:10186000EAD17F21412004F0BDFBE5E7104B1B7856
:10187000002BC9D110BD0F2008F09EFF0E4B104A5F
:101880001B881060002BF1D00E4A0F4912680968BE
:10189000521A9042EADC064C2278002ACAD0CDE7E0
:1018A000EA9BFF1FF09AFF1FC49BFF1F829AFF1F36
:1018B000B89BFF1FE09BFF1F249BFF1F949BFF1FF4
:1018C000BC9BFF1F409BFF1F3489FF1F2DE9F04F7A
:1018D00087B003AD8A4F2C4606AE611BC9B289485A
:1018E00006F064F83B88834294BF0020012004F88E
:1018F000010BA642F1D1844D84499DF80C308448F7
:101900002B709DF80E50834E0D709DF810109DF8B1
:101910001420814F814C01709DF812003070002618
:101920003A70267072B9002840F0D5807C4A19B10F
:101930001178002940F0E180002D00F0D4800223CE
:10194000237005E0002940F08C800523744A237041
:10195000744DDFF814B29DF80DE09DF80F00DFF82C
:101960000CA2DFF80C92DFF80C826F4F6F4E1370F1
:101970009DF811109DF816209DF8133085F800E0B1
:101980008BF800009DF815E09DF817C089F800203D
:10199000012088F8003087F800E08AF8001086F807
:1019A00000C008F009FF624A624BD2F800E07045BF
:1019B000CCBF012200221A7057DD5F4B198818290D
:1019C00053D80C395D4B2D781A789BF800C09AF8E3
:1019D00000A099F8003098F80080DFF89C913F78DB
:1019E00036782478A2EB4502AAEB8A0BCCEB0202F4
:1019F0005A44C3EB837BC3EB8B03134403EB4803D1
:101A0000B9F80020DFF874913B4406FB02334FF035
:101A10000C0B1BFB0433C9F80030BAF1000F06D0E1
:101A20002EB1042A0CBF02330433C9F80030444AF3
:101A3000444C12882488033A02EB420203EB8202F0
:101A400022440C3A114495B1B8F1000F0FD0BCF10B
:101A5000000F44D1BAF1000F4BD13B4A012414705E
:101A60000EE0062323702E4A72E70021AAE7364AC9
:101A700000241470BCF1000F00D027BB4FF0000C05
:101A8000324A704582F800C0C4BF314A1360314AFF
:101A90001368994213D0304B304C1868019001986C
:101AA00020601B6802932E4C029B248811601B1A35
:101AB000A34284BF2B4B196007B0BDE8F08F2748C5
:101AC000254B0068EDE7002DD8D1BAF1000FD5D134
:101AD0004FF0010CD4E704232370114A38E71A4A67
:101AE00000241470CAE7002B3FF432AF01232370A7
:101AF0002EE7154A82F800C0C2E70323237027E7C8
:101B00005C9BFF1F889BFF1FA59AFF1FA69AFF1FC4
:101B1000A79AFF1FA49BFF1FAA9AFF1F789AFF1F77
:101B2000349BFF1FEB9BFF1FEC9AFF1FF49BFF1FD3
:101B3000A489FF1FE09BFF1FF09AFF1F7089FF1F02
:101B4000189BFF1FC29BFF1F389BFF1F399BFF1F66
:101B5000F09BFF1F8C9AFF1FE09CFF1FB09AFF1F96
:101B6000F89BFF1FC49AFF1FEC9BFF1FED9BFF1FFD
:101B7000E89AFF1F6E9BFF1F529BFF1FE49BFF1FF6
:101B80002DE9F04F3A4B1B788BB0002B6BD10E2018
:101B900007F0CEFE0BF0CAF901463648364C374DF9
:101BA000FEF7C8FC3348FEF79BFC0BF0D9FB80F333
:101BB0000C002060FFF78AFE2E68012E7AD0022EDC
:101BC00000F0A882032E00F0B7832D4C23682D4A25
:101BD0002D4E0993099B177830682C4C0721012260
:101BE000181A11FB07229042236000F28E82284EC1
:101BF00032689A1A0D2A00F28182264E32689A1AA9
:101C0000132A00F27682244E32689A1A252A18D9AD
:101C1000224B1B88002B40F06581214B1B78002B49
:101C200040F060811F4B1B881B3B9BB2022B04D8EA
:101C30001D4B1B78002B40F0588102F025F82368DB
:101C400033601A4D2A689B1A502B00F21182184BF0
:101C50001B88012B00F0298204F058FA04F086F862
:101C60000BB0BDE8F08F05F0CBF80BB0BDE8F08FFE
:101C7000AC9BFF1FF49AFF1F889AFF1F949AFF1FC7
:101C8000E09CFF1FCC9BFF1F9C9BFF1FD09AFF1F58
:101C9000789BFF1F4C9BFF1FDC9BFF1FA89AFF1F19
:101CA000909AFF1FF09AFF1FE09BFF1F209BFF1FD2
:101CB0005A9BFF1FDFF82883A34AB8F80000137867
:101CC000834204D0C3B21846137004F05BF9DFF806
:101CD0000C939E4AB9F800301178994204D09C4F79
:101CE0003978002940F033879A4A236812889A4C41
:101CF0009A42C0F2FF80994A1278002A40F0FA8096
:101D0000DFF8E0A2BAF8003023B9954B1B88002B0E
:101D100000F01D85934A944B11881B88934A0B440D
:101D200012685B109342924A126880F2C0840021CC
:101D30009342B4BF01230B4604910093ACBF4FF014
:101D4000010B8B4605910E2007F0F2FD894B8A4A64
:101D50001B68176803930133A7F25232002B8446A5
:101D6000029240F30587802BA8BF8023834A8449D1
:101D700012780191002A00F0C7800978914200F0A2
:101D8000C380B9F80010DFF854E2994201F0EF8007
:101D90006F49AEF800307B4B4FF0010E81F800E048
:101DA0001978DFF844E2019B8EF800101A70009B4E
:101DB000002B00F01B81BAF80030002B00F01681D8
:101DC000714B1B685A1C002A40F3D686802A00F308
:101DD000D2866E4E6E496F48368809880068314455
:101DE000B0EB610FC1F2B881A3F148020F2A02D80B
:101DF000473BA8F800300E2007F09AFD6FF45473AB
:101E00001F44874202DC644B00221A70002008F055
:101E1000D3FC624A624B1168624E1B888842D4BF71
:101E2000002201223270002B00F038845E4B1E78B5
:101E3000964240D088423EDD5C490E78002E00F08C
:101E40007B875B4991F800C0BCF1000F40F07287BE
:101E5000584F0097584F59480297564F007887F8C7
:101E600000C0554F4FF0010E87F800C081F800E028
:101E7000002841F0328152490978002901F0208080
:101E8000504903910E460978002941F016804E48CA
:101E9000494F0078397001210297317058B1454897
:101EA00043490090002008700099029F0870039930
:101EB00001263E7008701A70444B1B88A3F11B0268
:101EC000012A40F21F861D2B7FF480AE3E4F3B78E7
:101ED000002B41F0C9803E4E3378002B40F06784E0
:101EE000337073E6FFF7D2F99CE62B68012B7FF481
:101EF000A4AEA4E62168374A0691069836491060D8
:101F000002220B602A60FBE61E49DFF8DCE009785C
:101F100000293FF448AF9EF8000081423FF443AFF0
:101F200003984B2840F3EA871833802BB9F8000058
:101F3000A8BF802398423FF436AF28480380044866
:101F4000012303702FE700BF7E9BFF1FCD9BFF1F68
:101F50001A9BFF1FEE9AFF1FE09CFF1F909AFF1F26
:101F6000149BFF1F589BFF1FE89BFF1F7C9AFF1FBE
:101F7000449BFF1FF09BFF1F549BFF1F389BFF1FBD
:101F8000CE9BFF1F399BFF1FE49BFF1FB49BFF1FCE
:101F9000269BFF1F489BFF1FE19BFF1FA489FF1F7C
:101FA000809BFF1FC99AFF1FDC9AFF1FE89AFF1F43
:101FB000C89AFF1F3C9BFF1F9C9AFF1F6E9BFF1F31
:101FC000EB9BFF1FCA9AFF1FE09BFF1FF09AFF1FAA
:101FD000169BFF1F689AFF1FD09BFF1FA29AFF1F2F
:101FE0003A9BFF1FB09BFF1FCF9BFF1F029B9C458F
:101FF000BFF601AFAC4B1B88002B3FF4FCAEBBF12E
:10200000000F7FF4DDAEA94B1B881BB1059B002B95
:102010007FF4D6AE049B002B3FF4EDAEA44B1A78B0
:10202000002A7FF4E8AEDFF8048398F8006001220C
:102030001A70002E40F058839E4B1B78002B01F045
:10204000CC809D4B1B78002B01F0DD809B4B1B78D7
:10205000002B7FF4D0AE9A4B1B78002B3FF4CBAE15
:10206000B9F8003097490A3BA9F800300A70C2E677
:1020700002F0E8FE944B1B7873B9944B1B785BB964
:10208000934B1B7843B9934B1B782BB9924B1B781E
:1020900013B901F0C3FD01E001F0CCFD23682B6012
:1020A0008E4B1B88012B7FF4D7AD8D4A8D4B116869
:1020B0008D481A78A1F118032A2101FB03F1016070
:1020C000002A00F0A782894A1368994200F34383EB
:1020D00080F24D8386480068D0F17F0048BF03300E
:1020E000801001301B1A994200F341831360194696
:1020F00092E2FFF773FB2368336084E5FEF7ECFCA4
:10210000FFF722F92368336077E5FEF75DFC23686B
:1021100033606CE5774A26681288B24204DB6E4B66
:102120001B78002B00F03E83734C744823680793A0
:10213000734B079900681B88091A994263D8002BD2
:1021400061D0704B198800293FF440AD6E4B6F4849
:102150001B680088B342B8BF33469A4240F3F58704
:102160006B4B1A60DFF8C88188F800105C4FFEF7EF
:102170002BFC38687F2840F3D985664B7F3883FB7A
:102180000032C317C3EB620303EB4303A0EB8300EE
:102190007330614B01931B883860002B40F0D5866B
:1021A0004B4B00931B78002B00F00E845B4E337872
:1021B000002B00F00984DFF87C91DFF858A14FF084
:1021C000000B0CE003F17300C0B298F8001003F0AC
:1021D00031FF33780BF1010B5B4540F3F5833B682E
:1021E00059F8040F1844A0F17F038AFB0321DA1782
:1021F000C2EB610202EB42027F28A3EB8203E1DC27
:10220000FEF72AFAE0E7404B40491B6808883D4941
:10221000B342B8BF33469A4200F3AB823C4E0988C2
:102220008342A8BF0346336000299BD19A42C8BFAE
:102230000B4640F3A582801AB0F5804FAABF9B03DE
:10224000C3EB8333013093FBF0F0FEF7A3FBC0F345
:10225000C6100AF06BFE324B064618880AF066FE7E
:102260003049074630460AF0B5FE014638460AF0C6
:10227000B1FE31460AF0A6FD4FF07E5106460BF046
:1022800047F8002840F04787274930460BF05EF8B2
:10229000002840F01C8730460BF088F8C0B2DFF809
:1022A000908088F8000061E7149BFF1FB29BFF1F1E
:1022B000E19BFF1FEB9BFF1FEC9BFF1FED9BFF1F95
:1022C000E89AFF1F1A9BFF1F9C9AFF1FC89AFF1FC7
:1022D0003C9BFF1FCA9AFF1F909AFF1F5A9BFF1F2C
:1022E000C49AFF1FB89BFF1F989BFF1FD89AFF1F20
:1022F000849BFF1FEE9AFF1FE09CFF1F689AFF1F41
:10230000749BFF1F509BFF1FD09BFF1FFA9BFF1F5B
:10231000E49AFF1FABAAAA2A1C9BFF1F3889FF1F44
:10232000809AFF1FCDCCCC3D0000FE42789AFF1F63
:10233000D49AFF1F7889FF1FC14B26681988B142C4
:1023400053DDC04B1B78002B4FD1DFF8489399F831
:1023500000007F2840F35886A3F155337F3803F1FE
:10236000004383FB0032C317C3EB620303EB430359
:10237000A0EB83007330B44B01931B88C0B289F883
:102380000000002B40F0B986B04B00931B78002B67
:1023900000F0FF84AE4E3378002B00F0FA84AD4F8E
:1023A000DFF8B8824FF0000A0AE003F17300C0B210
:1023B00003F068FE33780AF1010A534540F3E984DB
:1023C00057F8043F99F800001844A0F17F0388FBF8
:1023D0000321DA17C2EB610202EB42027F28A3EB72
:1023E0008203E2DCFEF738F9E1E79B4F38687F288B
:1023F00040F3CD81994B7F3883FB0032C317C3EB89
:10240000620303EB4303A0EB83007330DFF8849295
:1024100099F800A0824500F04282914B1B88002B66
:1024200043D1904A904812680088914205DC82426C
:10243000D4BFC1EB0203C1EB0003411AB1F5804FD9
:10244000A6BF9B030131C3EB833393FBF1F0FEF78F
:10245000A1FAC0F3C6100AF069FD844B064618883D
:102460000AF064FD8249804630460AF0B3FD014619
:1024700040460AF0AFFD31460AF0A4FC4FF07E5111
:1024800006460AF045FF002840F034867949304678
:102490000AF05CFF002840F0178630460AF086FFFD
:1024A000C0B2DFF8F48188F80000BAF17F0F40F382
:1024B00038846A48AAF17F0A80FB0A304FEAEA733F
:1024C000C3EB600000EB4000AAEB800073305F4B71
:1024D00000931B78C0B289F80000002B40F06B839A
:1024E000654B03931B78002B40F06085634B029390
:1024F0001B78002B40F02286534B0193029B1B78E4
:10250000B3B35F4B99F800201B881344A3F1180064
:102510007F2840F363855148973B80FB0320DA17FF
:10252000C2EB600000EB4000A3EB800303F17300FB
:10253000C0B203F0A7FD534B534A197899F8003005
:1025400032F811201344A3F118007F2840F342858C
:102550004248973B80FB0320DA17C2EB600000EB98
:102560004000A3EB800303F17300C0B203F08AFDC7
:10257000009B1B78002B00F0B384019B324E19881E
:10258000002900F0098538687F2840F31183334B18
:102590007F3883FB0032C317C3EB620303EB4303B3
:1025A000A0EB830073303860002940F0BE84009BAC
:1025B0001B78002B00F07E81254E3378002B00F035
:1025C0007981DFF890A0DFF8D0804FF0000B0CE0AD
:1025D00003F17300C0B298F8001003F02BFD3378BC
:1025E0000BF1010B5B4540F365813B685AF8040F22
:1025F0001A4A1844A0F17F0382FB0321DA17C2EBC9
:10260000610202EB42027F28A3EB8203E0DCFEF7CB
:1026100023F8DFE71D4B19601D4B1B68A92202FB45
:1026200003F3002BBCBF03F57F533F339B13543B95
:10263000194481F30C01282007F000FDFFF70CBBC3
:10264000EE9AFF1F909AFF1F1C9BFF1F3C9BFF1FD2
:102650003889FF1F7889FF1FC49AFF1FABAAAA2AD7
:10266000509BFF1FE49AFF1FFA9BFF1F809AFF1FDA
:10267000CDCCCC3D0000FE42CA9AFF1F9C9AFF1FA2
:10268000B69BFF1FC09BFF1FD49BFF1FD89AFF1F45
:102690007489FF1F729BFF1FD49AFF1FAD4EAE4877
:1026A000AE49AF4A337003700B70137004E4934269
:1026B0004FF0000B6EDA0123CDF800B0CDF814B066
:1026C0000493FFF740BBA74B1B78002B7FF493AB21
:1026D000039BA54A243B83F34703D9B25B201360D5
:1026E00003F080FC98F80060032E30D1DFF8CC8234
:1026F00098F80030002B40F0E0859C4F3B78002B91
:1027000040F0CE85974E3378002B40F0BC85984B37
:102710001B78002B40F0AA85964A1380964B1B78B5
:10272000002B40F09685954B7F221A8098F8003058
:102730006BB93B785BB933784BB9914A7F2107205D
:10274000138003F04FFC7F210B2003F04BFC8D4BDB
:102750001F68FFF750BB8C480068D0F17F0048BF6E
:10276000033003EBA00301339942BFF6BFAC116005
:1027700052E7864B09881A6000297FF4F3AC1346B0
:102780009842D4BFC2EB0003C2EB030353E5FDF74D
:1027900063FF3BE60123CDF810B0CDF800B0059300
:1027A000FFF7D1BA01232B60794CFFF70FBA794BB1
:1027B0006A20198803F09AFD3B783370FFF706BA58
:1027C000029B1B78002B40D0734A3B68128813444D
:1027D000A3F118007F2840F308847048973B80FBE2
:1027E0000320DA17C2EB600000EB4000A3EB80038C
:1027F00003F17300DFF8C881C0B298F8001003F04D
:1028000019FC67490B78022B9ABF5A1CD2B20022DE
:102810000A7064493B6831F812201344A3F1180090
:102820007F2840F3DF835D48973B80FB0320DA1766
:10283000C2EB600000EB4000A3EB800303F17300E8
:1028400098F80010C0B203F0F5FB019B1B88002B29
:1028500000F06583009B1B783BB9039B1B7823B971
:10286000029B1B78002B00F087843B4B1B78002BCE
:1028700000F06B814C490B78082B00F266814B48C5
:102880003A6800684A4E0133DBB25F1E101A46F800
:1028900027000B70474B2668198889F80020B14241
:1028A0003B4CBFF693A92268434B0892089A1A60E2
:1028B000FFF78CB9039B1B78002B81D03B68A3F1F9
:1028C0000C007F2840F36F8334488B3B80FB032050
:1028D000DA17C2EB600000EB4000A3EB800303F1CA
:1028E0007300DFF8DC80C0B298F8001003F0A2FBA0
:1028F000009B1B78002B3FF463AF2B4E3378002BEB
:102900003FF45EAFDFF8BCA04FF0000B0CE003F12A
:102910007300C0B298F8001003F08CFB33780BF111
:10292000010B5B457FF74CAF3B685AF8040F1B4A1D
:102930001844A0F18B0382FB0321DA17C2EB61027A
:102940000C3802EB42027F28A3EB8203DFDCFDF7A9
:1029500083FEDEE79C9AFF1FC89AFF1F3C9BFF1F68
:10296000CA9AFF1FE89AFF1F8C9BFF1FED9BFF1F5A
:10297000EC9BFF1F709BFF1F6E9BFF1F509BFF1F59
:10298000849AFF1F549BFF1F849BFF1FE49AFF1F25
:10299000E09CFF1FCC9AFF1FB69BFF1FABAAAA2A81
:1029A000C09BFF1FD49BFF1F3889FF1FA09BFF1FE9
:1029B0007C89FF1FEE9AFF1F889CFF1FEB9BFF1F68
:1029C000D49AFF1F7889FF1FAF4B1B78002B40F074
:1029D000C3823B68AD4A1278002A45D0A3F10C00AF
:1029E0007F2840F30E83AA4A8B3B82FB0321DA1730
:1029F000C2EB610202EB4202A3EB820303F173001C
:102A0000C0B298F8001003F015FB009B1B7853B37D
:102A1000A04E33783BB3DFF8C492DFF874A24FF0D6
:102A2000000B0BE003F17300C0B298F8001003F044
:102A300001FB33780BF1010B5B4514DD3B6859F862
:102A4000040F1844A0F18B038AFB0321DA17C2EBB1
:102A500061020C3802EB42027F28A3EB8203E1DC27
:102A6000FDF7FAFDE0E73B688B4A1278002A3ED07A
:102A70008A4A10880344A3F118007F2840F3BE82DD
:102A8000834A973B82FB0321DA17C2EB610202EB18
:102A90004202A3EB820303F17300C0B298F8001066
:102AA00003F0C8FA7E490B78022B9ABF5A1CD2B2A7
:102AB00000220A707B493B6831F812201344A3F1CD
:102AC00018007F2840F39782714A973B82FB0321CD
:102AD000DA17C2EB610202EB4202A3EB820303F1BD
:102AE0007300C0B298F8001003F0A4FA3B68019A92
:102AF0001288002A00F022826B4903220B702A60A0
:102B0000FFF764B8694F3B78002B3FF4E4A9684EA7
:102B1000307801F009F9674B1B78002B00F0BC827C
:102B200033887E2B00F2B882634A0133108899B251
:102B30003180002800F0C082C9B2C0B25F4E03F0FD
:102B400051FA3B783370FFF741B83A68A2E6DBB23E
:102B50001846137003F024FA594B4B491A464B4B55
:102B6000184600230B703B7013700370FFF7BCB85E
:102B70000123FFF7FBB880265249534B534A09887B
:102B80001B8812680B44B2EB630FBFF634A9474BA6
:102B90001B78002B40F0F181B9F800304C4AB34269
:102BA0003FF429A94B4B168001221A70FFF723B975
:102BB000FDF752FDF7E4484B01931B8863BB334B91
:102BC0000393354B0293334E33787BB3DFF80C819C
:102BD000DFF8BCA04FF0000B09E003F17300C0B2B6
:102BE00003F050FA33780BF1010B5B451EDD58F80A
:102BF000043F99F800001844A0F17F038AFB0321E9
:102C0000DA17C2EB610202EB42027F28A3EB8203D8
:102C1000E3DCFDF721FDE2E71C4B03931E4B02931F
:102C200003F030FA009B1B78002BCCD1039B1B7860
:102C3000002B3FF463AC99F80030A3F10C007F281F
:102C400040F3D68112488B3B80FB0320DA17C2EB9E
:102C5000600000EB4000A3EB800303F17300C0B2FF
:102C600003F010FA009B1B78002B00F0A881094E9E
:102C70003378002B00F0AA82DFF86080DFF810A024
:102C80004FF0000B37E000BFC89AFF1FCA9AFF1F22
:102C9000ABAAAA2A3889FF1F9C9AFF1FB69BFF1F69
:102CA000C09BFF1FD49BFF1F729BFF1FE09BFF1F5A
:102CB000CC9AFF1FEC9AFF1FA09AFF1F169BFF1FC5
:102CC0003C9BFF1F269BFF1FB49BFF1F489BFF1FC2
:102CD000A29AFF1F1A9BFF1F1C9BFF1F7889FF1FD3
:102CE00003F17300C0B203F0CDF933780BF1010B9F
:102CF0005B457FF703AC58F8043F99F8000018448F
:102D0000A0F18B038AFB0321DA17C2EB61020C38B6
:102D100002EB42027F28A3EB8203E1DCFDF79CFC7F
:102D2000E0E75046FDF798FCFFF7D1BBFDF794FCB8
:102D3000FFF72FBA00200870B549087840B1B549AF
:102D400000910978002900F0C581009F00213970A9
:102D5000B149097800297FF493A8002E40F0B08093
:102D6000002840F0AD80AD4EAA4F96F800E0AC4E82
:102D70000396AC4E0296AA4EAB493070A94E00970E
:102D8000087038703070BEF1000F7FF48BA8FFF729
:102D900092B8A34B1B78002B42D099F80030A3F1D6
:102DA0000C007F2840F3E081A04A8B3B82FB03218B
:102DB000DA17C2EB610202EB4202A3EB820303F1DA
:102DC0007300C0B203F05EF9009B1B7843B3984ECA
:102DD00033782BB3974FDFF854824FF0000A09E0A5
:102DE00003F17300C0B203F04DF933780AF1010A20
:102DF000534515DD57F8043F99F800001844A0F139
:102E00008B0388FB0321DA17C2EB61020C3802EB5B
:102E100042027F28A3EB8203E2DCFDF71DFCE1E721
:102E2000804B1B78B3B3844B99F800201B88134464
:102E3000A3F118007F2840F394817C4A973B82FBE2
:102E40000321DA17C2EB610202EB4202A3EB820319
:102E500003F17300C0B203F015F9784B784A197882
:102E600099F8003032F811201344A3F118007F289C
:102E700040F374816D4A973B82FB0321DA17C2EB62
:102E8000610202EB4202A3EB820303F17300C0B2C2
:102E900003F0F8F8019B1B88002B00F03781624B90
:102EA0001B78002B40F02D81664B674A19882668F5
:102EB0000020012310602B60F1E4039800210170D1
:102EC0005649097800293EF4F6AF5649029109782F
:102ED000002900F05781029800210170FEF7EBBF36
:102EE000039B1B78002B7FF448AB029B1B78002BC5
:102EF0007FF443AB019B1988FFF745BB243B002BB4
:102F0000B9F8000040F3338198423EF44CAF9BB2D5
:102F10004E48A9F8003001230370FEF744BF4C4B24
:102F20003878197803F086F894E4DFF82481C0B289
:102F300098F8001003F07EF8FFF739BBD8B298F884
:102F4000001003F077F83B68D6E5C0B298F800109F
:102F500003F070F8FFF724B97F21402003F042F816
:102F60003C49334A3B680B600021117032E53A4B13
:102F7000DFF8F0E01978FEF716BF4B2E40F3CE8055
:102F80001836802EB9F80030344AA8BF8026B342E4
:102F90007FF408AEFEF72FBF99F8000003F072F837
:102FA0003188FFF7F0BAFDF757FB9AE42C4B0193F9
:102FB0001B88002B40F08D811A4B02933BE6029B4D
:102FC0001B78002B7FF49DAA039B1B78002B7FF4BA
:102FD000D4AA8FE7FDF740FBFFF7C7BAFDF73CFB2C
:102FE000FFF7A6BAFDF738FB2AE4FDF735FB01E44D
:102FF000FDF732FB33E6FDF72FFB72E5FDF72CFB07
:103000004BE5FDF729FBFBE4FDF726FBFFF7B3B922
:103010006E9BFF1F3C9BFF1FEB9BFF1FE09BFF1F57
:10302000CA9AFF1F9C9AFF1FC89AFF1FABAAAA2A21
:103030003889FF1F7889FF1FB69BFF1FC09BFF1FAA
:10304000D49BFF1FEE9AFF1FE49AFF1F1A9BFF1FDE
:10305000D49AFF1FA09BFF1F399BFF1FA29AFF1F3F
:103060001C9BFF1FCF9BFF1F9B4E307800F05CFE28
:103070009A4B1B781BB133887E2B40F28F80984B84
:103080001B7823B13388944A002B40F09380954EEF
:103090003B783370FEF79ABD914B1B78002BF6D02E
:1030A00033888D4A002BF2D08F49013B088899B2B2
:1030B000118000287FF440ADC8B28A4E03F006F8B4
:1030C0003B783370FEF782BD7F20FFF7EAB97F209F
:1030D000FFF7E5B8854F864902974FF0000C81F85D
:1030E00000C0009F02994FF0010E87F800E081F8C0
:1030F00000C02DE60120FFF7D4B902F0C3FFFFF7AF
:1031000043B90021402002F06DFFCDE699F80000A0
:1031100002F0B8FFC3E60120FFF7C1B8243E002E3D
:10312000B9F8003035DDB3423EF465AEB6B2714B4E
:10313000A9F8006001221A70FEF75DBE6E4B019384
:103140001B88002B3FF4DAA96AE56C4A8342A8BFCA
:1031500003461360FFF706B8164618E5FDF77CFA3C
:1031600095E6FDF779FA75E6FDF776FA29E6012886
:103170003EF419AE0123CBE699F8000002F082FF7D
:10318000FFF773BB5E4800905E4859490390FEF715
:1031900089BE012B3EF42FAE0126C8E701339BB256
:1031A0003380D9B205204F4E02F01CFF3B783370BC
:1031B000FEF70CBD013B9BB2D9B20520494E1380EE
:1031C00002F010FF3B783370FEF700BD029B1B78C6
:1031D000002B7FF496A9FFF7D0B94B4B1B782BB38C
:1031E0004A4B1B78002B7EF406AE494B1B78002B14
:1031F0003EF401AEB9F800303E490A33A9F8003078
:103200000A70FEF7F8BD414B1B78002B7EF4F3AD3E
:103210003F4B1B78002B3EF4EEADB9F8003035493A
:10322000013BA9F800300A70FEF7E5BD374B1B786B
:10323000002B7FF448AA364B1B78002B3EF4DBAD05
:10324000B9F800302B490133A9F800300A70FEF7B5
:10325000D2BD304B00227F2107201A8002F0C2FE2F
:103260007F210B2002F0BEFEFFF760BA2A4B01223D
:103270007F2107201A8002F0B5FE7F210B2002F08B
:10328000B1FEFFF74BBA254B04227F2107201A809D
:1032900002F0A8FE00210B2002F0A4FEFFF737BACF
:1032A0001E4B02227F2107201A8002F09BFE7F2105
:1032B0000B2002F097FEFFF725BA184B00210720DC
:1032C0001E8002F08FFE7F210B2002F08BFEFFF7A5
:1032D00014BA064B0293A3E4CC9AFF1FEC9AFF1F8B
:1032E0006E9BFF1F169BFF1FA09AFF1F9C9AFF1F3C
:1032F000C89AFF1F1A9BFF1F1C9BFF1FE49AFF1F0A
:103300003C9BFF1FCA9AFF1FEC9BFF1FED9BFF1FFB
:10331000E89AFF1F509BFF1F709BFF1F849AFF1F9F
:1033200038B506F0A1FB0B4804F0D8FA00234FF0A3
:103330007E5201210848FDF799F8084B084A0949CF
:10334000802400251C7118461D60BDE838400AF035
:103350004DB800BF889BFF1FF49AFF1F2C9BFF1FD7
:103360001C89FF1FFD05000043682A20198802F010
:10337000BDBF00BF10B5044622206368198802F063
:10338000B5FFE36824201988BDE8104002F0AEBF05
:1033900010B504460A206368198802F0A7FFE368A5
:1033A0000C201988BDE8104002F0A0BF10B50446FB
:1033B00006206368198802F099FFE36808201988DD
:1033C000BDE8104002F092BF10B5044602206368C9
:1033D000198802F08BFFE36804201988BDE81040CB
:1033E00002F084BF70B50E4C84B012250422012374
:1033F00006460390029320468DE8240014231021F2
:1034000005F070FC062209230293039601952046DD
:1034100000921423102105F065FC04B070BD00BFBC
:10342000149CFF1F2DE9F041224D82B0012602B20B
:1034300084B20092284601967823192105F098FB62
:1034400004F10C0212B28DE844002846A719782333
:10345000192104F1020805F08BFB3FB20FFA88F83E
:1034600019233A46284619460196CDF8008005F002
:103470007FFB78233A4628461946CDF8008001960E
:1034800004F10A070B3405F073FB3FB224B2782332
:103490003A46284619468DE8500005F069FB192385
:1034A00000943A4601962846194605F061FB02B0A1
:1034B000BDE8F081149CFF1F2DE9F0411E4682B04B
:1034C0001446002A6AD0099B4D4A00EBC305012C23
:1034D0006F8929896868A7EB010382FB03E21A441C
:1034E0004FEAE373C3EBA21302887BD0042C38D1DC
:1034F00012FA83F3994203DC9F423946A8BF19466A
:10350000089A0180B6F90030BDF920803D48971D2A
:103510004FF0000E3FB2194642460097CDF804E046
:1035200005F026FB29896A896B68521A1B885C2A78
:10353000A3EB010359DD03EB43030132C3EB431358
:1035400093FBF2F303F11B0213B201203280194600
:103550004246019000972B4805F00AFB2A4B0022B7
:103560001A702A4B022CB3F9001045D0082C31D127
:1035700000221A8091422DD0089AB6F900302148D5
:103580000632012412B2009219460194BDF920209E
:1035900005F0EEFA204602B0BDE8F0811C4D1D4A50
:1035A0002B681268CB1A93420F4617D9164A3388F4
:1035B00011781448012918BF01241470089A0632A2
:1035C0001BB212B28DE814001946BDF9202005F097
:1035D000CFFA2F60012002B0BDE8F081204602B092
:1035E000BDE8F0819BB2D31A84E75C2101FB03F3B1
:1035F00093FBF2F21B32A7E74A1C12B21A80B9E71A
:10360000C94216B2149CFF1F8D9CFF1F069CFF1F12
:10361000889CFF1F9CED000030B583B000230C4652
:1036200005B2009326225B231C210C4804F0F0FF16
:10363000294601232622094804F0FAFA002C24B274
:1036400005DB214601232622044804F0F1FA044A4E
:10365000044B15801C8003B030BD00BF149CFF1FBD
:10366000AC89FF1FAE89FF1F70B5944C237882B0E0
:103670001BB1934B4FF6FF721A80924BB3F9003097
:10368000C3B9914A8E4B1068B3F9002080F30C0047
:103690005B2303FB00F000131C3082425AD04FF032
:1036A000FF31FFF7B9FF894805F016F800232370B2
:1036B00002B070BD012B32D0022B6AD0032B4FD049
:1036C000042BF3D1272200258DE8240076231C212A
:1036D0007E487F4E05F04CFA17E0B0F5AF7FA8BFEB
:1036E0004FF4AF70323803FB00F386FB0321DB1786
:1036F000C3EB61111C3109B201231D442722734819
:1037000004F096FA0C2D00F08180E9B2714804F0C3
:103710004DF931284FF05B03DFDC1C21ECE76E4BE9
:103720001A68B2F52F7F32DB41F25C239342A8BFC7
:103730001346A3F52F735B22684802FB03F380FB5B
:103740000320DB17C3EBA0201C305D4BB3F9003026
:103750008342A4D1624BB3F9003001339FD1A5E776
:10376000604B1B68B3F5FA7F11DBB3F57A6FA8BF26
:103770004FF47A63A3F5FA725B485B2303FB02F311
:1037800080FB0320DB17C3EB20201C30DDE71C206F
:10379000DBE7564B1B68B3F5FA7F33DBB3F57A6F83
:1037A000A8BF4FF47A63A3F5FA724F485B2303FB7B
:1037B00002F380FB0320DB17C3EB20201C304C4BB3
:1037C0001B68B3F5FA7F1FDBB3F57A6FA8BF4FF420
:1037D0007A63A3F5FA7244495B2303FB02F381FB8E
:1037E0000321DB17C3EB21211C31354BB3F900302A
:1037F00083427FF456AF3A4BB3F900308B427FF4EB
:1038000050AF53E71C20DAE71C21EEE7012006F059
:10381000D3FF6FF495733238364A03FB00F082FB16
:103820000023C017C0EB632303F5AF73312B3ADDE0
:10383000B3F5AF7FA8BF4FF4AF735B22323B244D8B
:1038400002FB03F385FB0325DB17C3EB65151C3572
:10385000002006F0B1FF6FF495733238254A03FB60
:1038600000F082FB0023C017C0EB632303F5AF73A6
:10387000312B1ADDB3F5AF7FA8BF4FF4AF735B22D6
:10388000323B134902FB03F381FB0321DB17C3EB3C
:1038900061111C310A4BB3F90030AB4207D0284606
:1038A000FFF7BAFEFFE61C25D2E71C21F2E70C4B1E
:1038B000B3F900308B42F2D1F5E600BFFC9BFF1F4D
:1038C000AC89FF1F029CFF1F889AFF1F149CFF1FDB
:1038D0004B48371B889BFF1FC49BFF1FD3058541A7
:1038E000AE89FF1F489BFF1F011FB8127C9AFF1F64
:1038F000449BFF1F67BBCF462DE9F04FDFF8EC82FA
:10390000B74CB8F900604D7854F8264087B082462D
:10391000039305B10D78DFF8FCB2002A34D19BF88F
:1039200000308BBBAF4EB6F90000002800F0CE800F
:10393000012800F02481012032232A4601900093BF
:103940005146A94B2046FFF7B7FD00250746B6F9BB
:103950000030022B40F3F48000233380B8F90030AC
:10396000A24A002BC0F2F880042BC4BF00231380AE
:10397000039B002B40F0F680002D0CBF38464FF023
:10398000FF3007B0BDE8F08F964EE3682268984894
:1039900004930027059237808BF8007004F090FDA7
:1039A0001120FFF73FFD4FF0010919232821CDF821
:1039B00004900091242219468D4805F0D9F8782307
:1039C00028212422CDF8049000918948194605F059
:1039D000CFF84946864805F061FC02221921844847
:1039E00005F058FCDDF8149048460AF0C9FA49463B
:1039F00002467F4805F0E8FD7D4805F0FBFD3946AD
:103A000014227B4805F046FC03227A49784805F0E9
:103A1000DBFD774805F0EEFD39462322744805F0BA
:103A200039FC03227449724805F0CEFD704805F058
:103A3000E1FD049B002B72D10123704A18461370DC
:103A4000FFF7D0FC208963896768191A5C293A88D6
:103A50005BDC131A5C2202FB03F292FBF1F31B33D3
:103A6000674A6348138001271BB21A2219468DE862
:103A70008400142205F07CF8049BDBB1218A638A60
:103A8000E768581A5C283A886FDD521A02EB420246
:103A9000C2EB4212431C92FBF3F31B33524A5448CD
:103AA0001380012738221BB28DE884001946322288
:103AB00005F05EF8534A544BB6F90000012111702D
:103AC0004FF6FF721A8000287FF432AFDFF848917A
:103AD0004E4AD9F800301268C3EB0A0393424CD91E
:103AE000464B1A78012A18BF012018700127FFF7EA
:103AF00079FCC9F800A0012D4ED0042D59D0022D1B
:103B000060D0082D64D0002521E7121A02EB420292
:103B1000C2EB42124B1C92FBF3F31B33A0E72F20A6
:103B2000FFF780FC39463222314805F0B3FB03220F
:103B300037492F4805F048FD2D4805F05BFD7BE730
:103B40007FF40CAFE368002B3FF406AFB8F9003008
:103B5000264A002BBFF608AF04231380039B002BDB
:103B60003FF40AAFFFF780FD06E7511A5C2202FB23
:103B700001F292FBF0F31B3390E70746BBE7002707
:103B800014238DE888002A4651461D4B2046FFF736
:103B900093FC3D460746DAE6B8F800308BF8005053
:103BA0000133A8F80030636983B1002520469847A7
:103BB000CDE6B8F800300122013BA8F800308BF8C0
:103BC0000020F0E7012333800025C7E61D46BEE64E
:103BD0006369002232804FF0FF35002BE6D1BDE64D
:103BE000B089FF1F069CFF1F009CFF1F029CFF1F48
:103BF000149CFF1F58E700005CE700008D9CFF1F2E
:103C0000FE9BFF1FFC9BFF1FAC89FF1F9CED00006C
:103C100060E70000049CFF1F889CFF1F01210D200E
:103C200006F09CBB00210D2006F098BB01460D203C
:103C300006F094BB08B50D2006F096FBB0FA80F1B3
:103C400049090D20BDE8084006F088BB10B50021E9
:103C500044080D2006F082FB204606F0BBFB0D2039
:103C6000012106F07BFB2046BDE8104006F0B2BB08
:103C700008B54FF49670FFF7E9FF4FF49670BDE872
:103C80000840FFF7E3BF00BF08B5214A214B128867
:103C90001868824234DA204B1B88991A8342A8BFE5
:103CA0000346B1F5F87FA3EB020321DAC3EB03135C
:103CB00003EB431393FBF1F105310A2006F0BEF943
:103CC000164B1978F1B1164B16491B6883F307039D
:103CD000C3EB031303EB431381FB03211944DB17ED
:103CE000C3EBA11105310920BDE8084006F0A6B9D3
:103CF000C3EB43131B01013193FBF1F10531DCE709
:103D00000021DAE70920BDE8084006F097B900BFB6
:103D1000EE9AFF1FE49AFF1FFA9BFF1FB89BFF1F3D
:103D2000849BFF1F090402817F2838B5A8BF7F202C
:103D30000D4D4FF4FA7303FB00F485FB0423234479
:103D4000E117C1EBA3110A2006F078F9A4F5784039
:103D50000C3885FB00310144C017A0EBA111BDE870
:103D60003840092006F06AB909040281024B10208C
:103D7000198802F0BBBA00BF3A9BFF1F024B4E20CE
:103D8000198802F0B3BA00BF1C9BFF1F024B4420EE
:103D9000198802F0ABBA00BFB69BFF1F024B2C2064
:103DA000198802F0A3BA00BF5E9BFF1F024B1E20C2
:103DB000198802F09BBA00BF369BFF1FC3680E2014
:103DC000198802F093BA00BF024B2820198802F02C
:103DD0008DBA00BF189BFF1F024B6220198802F0AA
:103DE00085BA00BF529BFF1F024B6420198802F066
:103DF0007DBA00BF5A9BFF1F024B5A20198802F060
:103E000075BA00BF9E9AFF1F024B1620198802F058
:103E10006DBA00BF509BFF1F024B2E20198802F085
:103E200065BA00BF749BFF1F024B3020198802F057
:103E30005DBA00BF809AFF1F024B1820198802F05C
:103E400055BA00BF249BFF1F024B1A20198802F0AD
:103E50004DBA00BF829BFF1F024B1C20198802F045
:103E600045BA00BFAE9BFF1F024B6620198802F0C7
:103E70003DBA00BF709AFF1F024B2020198802F044
:103E800035BA00BFF89BFF1F024B3220198802F0A1
:103E90002DBA00BFF09AFF1F024B6820198802F06C
:103EA00025BA00BFA09AFF1F024B5220198802F0CA
:103EB0001DBA00BFAA89FF1F024B5020198802F0CB
:103EC00015BA00BF7889FF1F024B5420198802F0F1
:103ED0000DBA00BFA089FF1F024B5C20198802F0B9
:103EE00005BA00BF7A89FF1F024B5E20198802F0D5
:103EF000FDB900BFA889FF1F024B6020198802F09E
:103F0000F5B900BF829AFF1F024B5620198802F0B4
:103F1000EDB900BFF69BFF1F064B074A10B41C8883
:103F2000064B0846002C14BF11461946042210BC4B
:103F30000AF0E4B8B09BFF1F84EE000088EE00009A
:103F4000064B074A10B41C88064B0846002C14BFC9
:103F500011461946042210BC0AF0D0B8149BFF1F6A
:103F600084EE000088EE0000064B074A10B41C885F
:103F7000064B0846002C14BF11461946042210BCFB
:103F80000AF0BCB8A89AFF1F84EE000088EE00007B
:103F9000064B074A10B41C88064B0846002C14BF79
:103FA00011461946042210BC0AF0A8B8809BFF1FD6
:103FB00084EE000088EE0000064B074A10B41C880F
:103FC000064B0846002C14BF11461946042210BCAB
:103FD0000AF094B8B29BFF1F84EE000088EE000048
:103FE000064B074A10B41C88064B0846002C14BF29
:103FF00011461946042210BC0AF080B8EE9BFF1F40
:1040000084EE000088EE0000064B074A10B41C88BE
:10401000064B0846002C14BF11461946042210BC5A
:104020000AF06CB8709BFF1F84EE000088EE000061
:1040300070B5284E05460FCE86B06C460FC496E884
:10404000030044F8040B2320218005F071FC40F6A6
:10405000B833984230DC204B40F6F50219889B7843
:10406000ADF80D1090428DF80F302DDD00EB4000C3
:104070001A4B1B491B4E00EB0010C21783FB004379
:10408000C2EB632381FB0314D917C1EBA40101EB3D
:10409000810186FB0040C2EB6030A3EB410330306E
:1040A00030338DF811008DF81330694628461622FA
:1040B0000AF024F806B070BD0B4B1A889B78ADF857
:1040C0000D208DF80F30D1E7084B1868CDF811009E
:1040D000EBE700BF9CEE00008CEE0000976A3E2BE1
:1040E000676666668BAA304598EE000090EE000089
:1040F00038B5094D4624204602F012F935F8021B66
:1041000000B28842204601D002F0F0F80234A4B296
:104110004E2CF0D138BD00BFD49BFF1FF8B5174C13
:10412000174E2278174D33782F888E46003218BFED
:10413000012201467046FFF7DFFB002398423370EF
:10414000237015DB14BF012000202B889F420ED066
:1041500040F23A72A3F5AF730B490C4C02FB03F328
:1041600081FB0312DB17A3EB621332332360F8BD2C
:104170000749012218460A702270E6E75C8BFF1F90
:10418000AA9CFF1F5C9BFF1FB5814E1BA489FF1FCC
:104190000C9CFF1F014B187802F040B8A09CFF1F39
:1041A000014B187802F054B8C88CFF1F134BB3F9B9
:1041B000003030B583EAE374A4EBE374002BA0B2C3
:1041C00018DB012300E0134603EB83025200944204
:1041D000F9DA0B4D90FBF3F285FB03E403FB1200CD
:1041E000DB173032D3EBA40380B201F8012BF1D1FD
:1041F0000B7030BD2D230B700131E2E7C88CFF1F1F
:1042000067666666144BB3F9003070B583EAE375F0
:10421000A5EBE375002BACB21ADB012300E00346EB
:1042200003EB830040008542F9DA0C4E94FBF3F077
:1042300086FB03E503FB1044DB173030D3EBA5030B
:10424000A4B201F8010BF1D105480B70106070BDEC
:104250002D230B700131E0E79E9AFF1F67666666AB
:10426000B4EE0000134BB3F9003030B583EAE374C9
:10427000A4EBE374002BA0B218DB012300E013468B
:1042800003EB830252009442F9DA0B4D90FBF3F2F8
:1042900085FB03E403FB1200DB173032D3EBA403EE
:1042A00080B201F8012BF1D10B7030BD2D230B70C2
:1042B0000131E2E7AA89FF1F67666666134BB3F90F
:1042C000003030B583EAE374A4EBE374002BA0B2B2
:1042D00018DB012300E0134603EB830252009442F3
:1042E000F9DA0B4D90FBF3F285FB03E403FB1200BC
:1042F000DB173032D3EBA40380B201F8012BF1D1EC
:104300000B7030BD2D230B700131E2E77889FF1F60
:1043100067666666134BB3F9003030B583EAE37421
:10432000A4EBE374002BA0B218DB012300E01346DA
:1043300003EB830252009442F9DA0B4D90FBF3F247
:1043400085FB03E403FB1200DB173032D3EBA4033D
:1043500080B201F8012BF1D10B7030BD2D230B7011
:104360000131E2E7A089FF1F67666666134BB3F968
:10437000003030B583EAE374A4EBE374002BA0B201
:1043800018DB012300E0134603EB83025200944242
:10439000F9DA0B4D90FBF3F285FB03E403FB12000B
:1043A000DB173032D3EBA40380B201F8012BF1D13B
:1043B0000B7030BD2D230B700131E2E77A89FF1FAE
:1043C00067666666134BB3F9003030B583EAE37471
:1043D000A4EBE374002BA0B218DB012300E013462A
:1043E00003EB830252009442F9DA0B4D90FBF3F297
:1043F00085FB03E403FB1200DB173032D3EBA4038D
:1044000080B201F8012BF1D10B7030BD2D230B7060
:104410000131E2E7A889FF1F6766666638B5FDF7D8
:1044200055FA0D4B1B7833B90C4B1020198801F04D
:104430005DFF012038BD0A4D0A4C2B782288B3FA63
:1044400083F382F008025B09114642202B70228020
:1044500001F04CFF002038BDE09BFF1F3A9BFF1F7F
:10446000CC9BFF1FB49AFF1F10B40A4B0A4C0A469C
:1044700093E8030083B0238802AC04E9030004EB53
:104480008303104653F8081C052203B010BC09F042
:1044900035BE00BFE8E700005A9BFF1FF0B40C4D8B
:1044A0000C4F0E460FCD8CB001AC0FC40FCD0FC416
:1044B00095E807003B8884E807000CAA02EB830319
:1044C000304653F82C1C04220CB0F0BC09F016BE88
:1044D000F0E70000849AFF1F30B40A4B0A4D0C46E7
:1044E00093E8070084B02B8804AD05E9070005EBCD
:1044F0008303204653F80C1C042204B030BC09F09E
:10450000FDBD00BF1CE80000249BFF1FF0B40A4D56
:104510000A4F0E460FCD86B001AC0FC42A683B8807
:10452000226006AA02EB8303304653F8141C0C22C7
:1045300006B0F0BC09F0E2BD28E80000AE9BFF1F0A
:10454000164B1B880BB31BB283EAE370A0EBE3703E
:10455000002B30B584B21DDB012300E0134603EBD2
:10456000830252009042F9DA0D4894FBF3F280FB8B
:1045700003E503FB1244DB173032D3EBA503A4B2EF
:1045800001F8012BF1D10B7030BD0846042205491A
:1045900009F0B4BD2D230B700131DDE7A09AFF1F98
:1045A00067666666B8EE0000054B1B881BB9054BB5
:1045B000186808607047044B18680860704700BFAF
:1045C0001C9BFF1FC0EE0000BCEE0000164B1B88BA
:1045D0000BB31BB230B583EAE374A4EBE374002B96
:1045E000A0B21CDB012300E0134603EB8302520060
:1045F0009442F9DA0D4D90FBF3F285FB03E403FBE3
:104600001200DB173032D3EBA40380B201F8012B88
:10461000F1D10B7030BD064B1868086070472D2330
:104620000B700131DEE700BF369BFF1F67666666D1
:1046300088EE0000164B1B880BB31BB230B583EA23
:10464000E374A4EBE374002BA0B21CDB012300E0B5
:10465000134603EB830252009442F9DA0D4D90FBAE
:10466000F3F285FB03E403FB1200DB173032D3EBDC
:10467000A40380B201F8012BF1D10B7030BD064BC1
:104680001868086070472D230B700131DEE700BF0A
:104690007C9BFF1F6766666688EE0000164B1B88D2
:1046A0000BB31BB230B583EAE374A4EBE374002BC5
:1046B000A0B21CDB012300E0134603EB830252008F
:1046C0009442F9DA0D4D90FBF3F285FB03E403FB12
:1046D0001200DB173032D3EBA40380B201F8012BB8
:1046E000F1D10B7030BD064B1868086070472D2360
:1046F0000B700131DEE700BF509BFF1F67666666E7
:10470000C4EE0000174B1B881BB31BB270B583EAC5
:10471000E375A5EBE375002BACB21EDB012300E0D3
:10472000034603EB830040008542F9DA0E4E94FB0A
:10473000F3F086FB03E503FB1044DB173030D3EBCB
:10474000A503A4B201F8010BF1D108480B70106069
:1047500070BD074B1868086070472D230B7001313E
:10476000DCE700BF749BFF1F6766666694EE00007F
:1047700088EE0000164B1B880BB31BB230B583EAE2
:10478000E374A4EBE374002BA0B21CDB012300E074
:10479000134603EB830252009442F9DA0D4D90FB6D
:1047A000F3F285FB03E403FB1200DB173032D3EB9B
:1047B000A40380B201F8012BF1D10B7030BD064B80
:1047C0001868086070472D230B700131DEE700BFC9
:1047D000809AFF1F6766666688EE0000184B1A888D
:1047E00052B3184A128830B50A80B3F90030002B52
:1047F00083EAE374A4EBE374BCBF2D238B70A0B2F7
:10480000ACBF02310331012300E0134603EB830206
:1048100052009442F9DA0C4D90FBF3F285FB03E46D
:1048200003FB1200DB173032D3EBA40380B201F894
:10483000012BF1D10B7030BD044B18680860704734
:10484000829BFF1FC8EE00006766666688EE000068
:10485000164B1B880BB31BB230B583EAE374A4EB91
:10486000E374002BA0B21CDB012300E0134603EB32
:10487000830252009442F9DA0D4D90FBF3F285FB6E
:1048800003E403FB1200DB173032D3EBA40380B246
:1048900001F8012BF1D10B7030BD064B1868086090
:1048A00070472D230B700131DEE700BF709AFF1FA8
:1048B0006766666688EE0000174B1B881BB31BB249
:1048C00070B583EAE375A5EBE375002BACB21EDB94
:1048D000012300E0034603EB830040008542F9DA40
:1048E0000E4E94FBF3F086FB03E503FB1044DB174D
:1048F0003030D3EBA503A4B201F8010BF1D1084885
:104900000B70106070BD074B1868086070472D234E
:104910000B700131DCE700BFF89BFF1F676666661E
:10492000CCEE000088EE0000074B1B88022B06D05F
:10493000012B0CBF054B064B186808607047054BF0
:1049400018680860704700BF829AFF1FD4EE00000D
:10495000D8EE0000D0EE0000054B1B881BB1054BC4
:10496000186808607047044B18680860704700BFFB
:10497000F69BFF1FE0EE0000DCEE0000F8B55D4D99
:104980002B780646002B37D11C4673780BB920468E
:10499000F8BDFCF79BFF584A5849594B594F30789E
:1049A000097812781B883E7802EB4102411E06FB13
:1049B00003230E29EBD801A252F821F0494A000046
:1049C0006B4A00008F490000494A00008F490000EF
:1049D0008F4900008F490000134A00008F490000F2
:1049E0008F4900008F4900008F4900008F49000067
:1049F0008F4900000F4A0000AE21434803F010FB2E
:104A0000414803F05DFD00232B700124BDE705F054
:104A1000F3FF3E4B3E491B78002B3DD03D4B3E4AB9
:104A200009881B8812680B44B2EB630F59DA3B4BC1
:104A30001B78002B4BD0AF21334803F0F1FA384AF2
:104A4000012313702B70A2E783B9364E33880428F4
:104A50004FF6FF7103F1FF320CBF01230B461344E5
:104A600003F07F03013333800FE073B1013B2E4A23
:104A700032F813304BB12B4E2C482D492D4A338040
:104A80000123002606700B701370254A02210123B2
:104A900011702B702046F8BD1E4B1F4A09881B88D9
:104AA00012680B44B2EB630FC5DB234E234D3388F2
:104AB0002A88B3FA83F382F002025B09338011463D
:104AC00042202A8001F012FCFFF7D2F85FE7AF2105
:104AD0000D4803F0A5FA124A0621012311702B702C
:104AE00055E7174E154D33882A88B3FA83F382F0C1
:104AF0000402E2E75C8BFF1F6E9BFF1FEC9AFF1F17
:104B0000529BFF1FF49BFF1F149CFF1FE09BFF1F86
:104B1000B49BFF1F269BFF1F489BFF1FC99AFF1FC7
:104B20000C9CFF1FA29AFF1F609BFF1FCD9BFF1FC6
:104B30001A9BFF1F819CFF1FB09BFF1FB49AFF1F92
:104B4000149BFF1F10B5064B064C1A882046012106
:104B500001F0BAFB21884220BDE8104001F0C6BB3D
:104B6000B09BFF1FB49AFF1F10B5064B064C1A8866
:104B70002046022101F0A8FB21884220BDE8104018
:104B800001F0B4BB149BFF1FB49AFF1F10B5064B76
:104B9000064C1A882046042101F096FB2188422009
:104BA000BDE8104001F0A2BBA89AFF1FB49AFF1FF6
:104BB00010B5064B064C1A882046052101F084FBEF
:104BC00021884220BDE8104001F090BB809BFF1F70
:104BD000B49AFF1F10B5064B064C1A8820460621D2
:104BE00001F072FB21884220BDE8104001F07EBB3D
:104BF000B29BFF1FB49AFF1F10B5064B064C1A88D4
:104C00002046002101F060FB21884220BDE81040D1
:104C100001F06CBBEE9BFF1FB49AFF1F08B512207A
:104C200001F07EFB054B1988884206D0122001F066
:104C30005DFBBDE8084001F071BA08BD849AFF1F12
:104C400008B5582001F06CFB054B1988884206D046
:104C5000582001F04BFBBDE8084001F05FBA08BDE9
:104C60007C9BFF1F08B5142001F05AFB054B1988E7
:104C7000884206D0142001F039FBBDE8084001F05D
:104C80004DBA08BD709BFF1FF0B480EAE075A5EB3C
:104C9000E0750028ACB21FDB1DBF2B230B704E1C30
:104CA0000E46012300E0134603EB830252009542B7
:104CB000F9DA0B4F94FBF3F287FB030503FB124475
:104CC000DB173032D3EBA503A4B206F8012BF1D1E8
:104CD00033700846F0BC70472D230B704E1CE0E784
:104CE00067666666144B18880C2811D0192813D0F3
:104CF0001A2815D01B2817D01C2819D01D2803D01E
:104D00000C3800B2FFF7C0BF0C4A1068086070474B
:104D10000B4A1068086070470A4A106808607047BC
:104D2000094A106808607047084A106808607047B0
:104D3000074A106808607047F09AFF1FF8EE0000FD
:104D4000E4EE0000E8EE0000ECEE0000F0EE000003
:104D5000F4EE0000024B1888183800B2FFF794BF39
:104D6000B69BFF1FC3681888183800B2FFF78CBFC6
:104D7000034B1888A0EB8000400000B2FFF784BF0F
:104D8000A09CFF1F024BB3F90000FFF77DBF00BFDF
:104D9000529BFF1F024B1888033800B2FFF774BF05
:104DA000189BFF1F024B18880C3800B2FFF76CBF2E
:104DB000C29BFF1F30B5134C85B001252B463C220A
:104DC00002212046009503F0A1F9204603F078FB6C
:104DD00000224021802320460191009311460A4B76
:104DE000029504F01BF8204603F076FC07480849BA
:104DF000084A0023036083800B608B8013609380DC
:104E000005B030BD149CFF1F94E80000749CFF1F88
:104E1000A49CFF1F909CFF1F10B500EBC00000F189
:104E20000F02D2B293B284B09C1E981C3D23039112
:104E30008DE819003921024803F054FF04B010BD79
:104E4000149CFF1F014B01221A707047AA9CFF1F80
:104E5000F0B585B05E4C5F4B02935F4A019204232C
:104E6000009320465D4B5E4F5E4E5F4D4022802199
:104E700002F054FF20465D4C5D4A5E4908F0B6FAE8
:104E8000A7615D485D4FE7615D4F87615D495E4F9A
:104E9000C7615E4F8F615E4A5E4FCF615E4F976123
:104EA0005E4B5F4FD7615F4F9F615F4FDF615F4F29
:104EB000B7615F4FF7615F4FAF615F4C5F4FEF616D
:104EC0005F4FA7615F48604FE761604F876160494E
:104ED000604FC761604F614A8F61614FCF61614F21
:104EE000614B9761614FD761614F624E9F61624F25
:104EF000DF61624F624DB761624FF761624F634C91
:104F0000AF61634FEF61634F6348A761634FE76130
:104F1000634F64498761644FC761644F8F61644A1E
:104F2000644FCF61644F9761644B654FD761654FA4
:104F30009F61654E654FDF61654FB761654D664F97
:104F4000F761664FAF61664C664FEF61664FA761D0
:104F50006648674FE761674F87616749674FC76179
:104F6000674F8F61674A684FCF61684F9761684BA1
:104F7000684FD761684F9F61684E694FDF61694F25
:104F8000694DB761694FF761694F6A4CAF616A4F0C
:104F90006A486B49EF616B4F6B4DA761E5616B4FE1
:104FA0006B4D6C4CDFF8D0E16B4A6C4B8761C5618F
:104FB0008C61C1F81CE06A4E6A4F6B4D6B4C6C48BB
:104FC0006C499761D5619C61D861B16005B0F0BD55
:104FD000149CFF1FA0860100801A0600548FFF1F3B
:104FE000A54D0000808CFF1F308AFF1FA48CFF1F7F
:104FF0001C89FF1F757D0000388BFF1FBD3D000021
:10500000954D0000E889FF1FC93D0000193F0000D1
:10501000388DFF1F454B0000413F0000888BFF1F6C
:10502000694B0000693F00008D4B0000913F00007C
:10503000B14B0000854D0000F08AFF1FD93D0000F4
:10504000B93F0000648EFF1FD54B0000694400008B
:10505000D08EFF1FE93D0000E13F00000C8AFF1FDA
:10506000F94B0000714D0000CC8CFF1F95410000F2
:10507000AD410000E48DFF1FA14100009D440000F0
:10508000D08BFF1F1D4C000035460000A88AFF1F73
:10509000414C000005420000608AFF1FF93D0000FE
:1050A00009400000188FFF1F654C00009D4600005E
:1050B000F48BFF1F093E000005470000848AFF1F94
:1050C000193E000075470000AC8BFF1F293E000011
:1050D000D9440000148BFF1F393E0000DD4700005B
:1050E000148DFF1F493E00000D450000888EFF1FF4
:1050F000593E0000514800003C8CFF1F693E0000F3
:10510000B9480000208EFF1F793E0000E54C0000EA
:10511000AC8EFF1F893E000041450000CC8AFF1F76
:10512000993E000065420000188CFF1FA93E000058
:10513000BD420000C489FF1FB93E00009C8DFF1FC7
:10514000C08DFF1F15430000C93E00006D430000E5
:10515000D93E0000C5430000F48EFF1FF08CFF1FF6
:10516000548AFF1F29490000F93E000059490000F8
:10517000093F0000E9540000E93E00002DE9F04F2E
:105180002F4DDFF8CCB0DFF8C4A0DFF8C8900FCD0A
:1051900091B003AC0FC40FCD0FC40FCD0FC42B685B
:1051A00023600025A8462F462E4600E09846BAF810
:1051B000003024495BF8232028461123FBF7D4FB59
:1051C00000EBC00400EB840089FB00340444C017EA
:1051D000C0EB6434C4F13C00C6F13C0207F141016C
:1051E000012600B208F1410300901BB2019612B2F1
:1051F00009B2154803F0BCFC08EB060305F21115D3
:105200003C2B2646ADB24746D0D134226B210E4806
:1052100004F040F800210C4804F040F80B4B1B88C8
:1052200010AA02EB830353F8344C204608F0A8FE82
:1052300002460548214611B0BDE8F04F04F0C4B95C
:105240003CE8000004E50000149CFF1F5E9BFF1F6C
:1052500048E60000090002802DE9F043804685B051
:10526000002956D10121304804F018F82F4998F848
:10527000062098F8083011F80290994522DA4FEA92
:1052800089064D460C24D8F80C3027489B595F6896
:1052900022B2002103F0FEFF384608F071FE3946C5
:1052A0000246214804F090F91F4804F0A3F998F849
:1052B000083001350934AB42A4B206F1040601DD21
:1052C000422CE0D1B9F1000F13D109F1060999453B
:1052D0000CDA3C2301213B220391029300930192BB
:1052E00039233F223A21104803F0FCFC05B0BDE809
:1052F000F0830F2301213B2203910293009301923B
:1053000039230C223A21084803F0ECFC98F80830C5
:10531000DBE700213423009301913F230C22024854
:1053200003F0F4FB9EE700BF149CFF1FA49CFF1F2B
:1053300010B5104C0121204603F0B6FF2046012194
:1053400003F0ACFF20463422552103F0A3FF204692
:105350000222094904F038F920460522074904F0E1
:1053600033F9204604F046F92046BDE8104003F02A
:10537000B3B900BF149CFF1FFCEE000000EF00005B
:1053800070B50D46064608F0FBFD00EB40008400BA
:10539000002D36D0284608F0F3FD00EB4000400019
:1053A00023185B1003F16001091A282209B217487B
:1053B000C3F1600403F06EFF0121144803F06EFF97
:1053C000284608F0DDFD29460246104804F0FCF8A6
:1053D0000E4804F00FF902210C4803F05FFF21B2E0
:1053E00021220A4803F056FF304608F0C9FD314635
:1053F0000246064804F0E8F80448BDE8704004F0AE
:10540000F9B86410C4F16004E5E700BF149CFF1F05
:10541000214B70B5B3F9003083EAE374A4EBE37475
:10542000002B82B0A1B22FDB68466D46012300E05D
:10543000134603EB830252009442F9DA174E91FBB4
:10544000F3F286FB03E403FB1211DB173032D3EBDC
:10545000A40389B205F8012BF1D119462B70FFF78F
:105460008FFF0F4B1B786BB101210E4803F016FF25
:10547000332274210B4803F00DFF01220A49094829
:1054800004F0A2F802B070BD2D238DF800300DF1AC
:1054900001056846CAE700BF3A9BFF1F676666665C
:1054A000CC9BFF1F149CFF1F18F1000010B50D4B83
:1054B0001B5C51F82340237884B013B1012004B061
:1054C00010BD04AA01A942F8103D2046A3699847DF
:1054D000A38A9B07F2D401A80099FFF751FF01208E
:1054E00004B010BD749CFF1FF8B51F4D287840B95B
:1054F0001E4B1B68994203D31D4A012313702B7066
:10550000F8BD0C4600261B48184F02F0D9FF04F6E0
:10551000B833324617483B6031212E7003F0BAFE93
:105520000121144803F0C0FE3146124803F0B6FED4
:10553000052211490F4804F047F80E4804F05AF8C4
:105540000C2210210B4803F0A5FE0B220B49094841
:1055500004F03AF805220A49064804F035F80548EF
:1055600004F048F80120F8BD5C8BFF1F7C9CFF1FF6
:105570000C9CFF1F149CFF1F08EF000010EF0000A1
:1055800000EF000010B5424C424882B002F098FF94
:105590002378C3B906213F4803F080FE2378012B0E
:1055A00037D90A22022B11463A486BD003F072FE1B
:1055B00039490322374804F007F8364802B0BDE8FD
:1055C000104004F017B8354B1A7801210523002A42
:1055D00035D10191009311462E4803F019FB304B51
:1055E0001A78002A36D00523012201920093002266
:1055F0000A21284803F08AFA2A4B1A78002A35D162
:1056000001210523019100931421224803F000FB9E
:10561000C0E7254C2388092B32D9632B8CBF0A2184
:105620001F210A221B4803F035FE2188194804F087
:1056300031F8184802B0BDE8104003F0DBBF00228B
:10564000019100931146134803F060FA144B1A7845
:10565000002AC8D105230121019100930A210D4898
:1056600003F0D6FA0F4B1A78002AC9D0012205237D
:105670000192009300221421064803F047FA89E7BB
:105680003021CEE703F006FE0322084992E700BF6F
:10569000819CFF1F149CFF1F20EF00006E9BFF1FCB
:1056A000EC9AFF1FF49BFF1FA29AFF1F1CEF000044
:1056B0002DE9F041764C2278002A05460F4614BFAA
:1056C0004FF001084FF0000850D1724E3368CB1AEA
:1056D000B3F5FA6F04D86B78A3B94046BDE8F08102
:1056E0006D4B6E486E49DFF8D8E11A7001230370E4
:1056F0000988237026208EF8002000F0F7FD6B78D3
:10570000002BEAD03760FCF7E1F8664A664B674940
:10571000674812782D781B780988007802EB4303DC
:105720006A1E00FB01330E2AD7D801A151F822F0DE
:1057300021580000ED570000DB5600002158000002
:10574000DB560000DB560000DB560000D55700009A
:10575000DB56000087570000DB560000DB560000D8
:10576000DB560000DB56000083570000AF21514894
:10577000484E02F055FCFFF705FF00233760237009
:10578000A9E705F039F94B4802F09AFE0221494891
:1057900003F084FD0F222321464803F07BFD052200
:1057A0004549444803F010FF424803F023FF1E22FE
:1057B0002321404803F06EFD052240493D4803F097
:1057C00003FF3C4803F016FF3A4802F085FF00F063
:1057D000B1FC82E73A4D2B78012B50D9304B262073
:1057E000198800F083FD00232B7076E7002B3FF42F
:1057F00074AF013B334A32F81330002B3FF46DAFE6
:10580000274C314825492E4A23804FF001080023B8
:10581000037081F8008082F80080FFF7B3FE5CE738
:1058200093B1013B274A32F8131019B31C4B264D94
:105830001A4C234A19800026012326202E7023703B
:10584000137000F053FD15E0154C1F4922880B70B2
:10585000042D4FF6FF7002F1FF310CBF012202460A
:105860000A440E4F164E02F07F02013201212280BF
:1058700039703370FFF786FE4FF001082DE70649B7
:10588000064A01230020087013702370A6E700BFAA
:105890005C8BFF1F9C9CFF1F0C9CFF1F1A9BFF1F14
:1058A000A29AFF1F6E9BFF1FEC9AFF1F529BFF1FC8
:1058B000F49BFF1F149CFF1F24EF00002CEF00003F
:1058C000819CFF1F609BFF1FCD9BFF1F2DE9F04FA9
:1058D00005468BB00F46AE480121164603F0E4FCA6
:1058E000AA8812F0010440F0B280DFF8D48298F860
:1058F0000030002B7FD1AB79A64AD15CA1B9DFF88B
:10590000C4A279781AF8039041B33978013907298C
:1059100000F2B980DFE811F0F3005801B700700120
:10592000B700B700B700EB007C78002C00F0CC800B
:105930000139EC68387854F82170FC68411EB4F8DD
:105940000080072900F2A980DFE811F078015D01ED
:10595000A7007001A700A700A700A100DFF85CA2C4
:10596000DAF80020B21AB2F5967F77D98A4A107811
:1059700001281ABF012010701170884A18BF014613
:10598000D05CC0EB0900C0B2FFF746FA0124CAF8A8
:105990000060AB889B0772D57B78002B6FD0FBF73C
:1059A00095FF7F4B7F4A804D80481B78127839786D
:1059B0002E780088022515FB02320A2906FB0023F7
:1059C00000F050810C295AD1002B58D003F1190056
:1059D000774E784A013B0021400080B226F8131030
:1059E0000123157088F8003000F080FC724B032210
:1059F00020461A702FE0664802F062FD01216448DB
:105A000003F04CFC62482246214603F043FCAB887D
:105A1000580725D42C68204608F0B2FA21460246E1
:105A20005B4803F0D1FD5A4803F0E4FD092201234D
:105A30008DE80C0000217F23554803F099F80021E0
:105A40002846FFF709FC002388F8003053E7AB68CD
:105A50003146384698470BB0BDE8F08F0846FAE764
:105A60002B6804A8984704A808F08AFA04A90246FB
:105A7000474803F0A9FD464803F0BCFDD6E72046A1
:105A80000BB0BDE8F08F00240AF8039081E70021F5
:105A9000D1543846FB699847FC68A4F80080002779
:105AA00025223C238DE8840041211822384803F048
:105AB0002DF8E968A879FFF7F9FC374A3F4B1770D2
:105AC0001E600BB0BDE8F08F3C490A68B21AB2F50F
:105AD000967FD4D9304F0E603E78012E00F0B6800C
:105AE000E968184601233B70FFF7E0FCB3E7314A51
:105AF000E9791170012288F800200024C4E72A7A8D
:105B0000013A4A45BFDD09F10106F6B2B145BAD006
:105B1000224A039212F803B0CBEB0900C0B2002175
:105B2000FFF77AF92B7A052B5C461BD9CBEB0601E4
:105B30000429039A40F3AE80A6F1040BBBF1000FD9
:105B4000C0F2B080063B9B45A8BF9B465FFA8BF432
:105B5000AB791248D25C5A4504D0C454012128467E
:105B6000FFF77AFB301BC0B201210B4CFFF754F951
:105B700000213423019100930548217040230B221A
:105B80003F2102F0C3FFB1460124AB797CE700BF9F
:105B9000149CFF1F909CFF1F8D9CFF1FA49CFF1F48
:105BA0006E9BFF1FEC9AFF1FF49BFF1F529BFF1F72
:105BB000609BFF1F0C9CFF1F819CFF1F889CFF1F89
:105BC0005C8BFF1F749CFF1F0FFA89F1E8685F4C24
:105BD00050F821602168049134785D490498086088
:105BE000002C70D0012C7FF44EAF5A4A317A88F8DD
:105BF00000401170002447E7B9F1000F50D009F1BF
:105C0000FF36F6B282E7B98A01F0040189B20029B1
:105C10003FF43EAF3B6A03929847039A00283FF453
:105C20003BAFAB79FC680021D15436E77B8A434512
:105C30003BD908F101081FFA88F82EE73B8A434553
:105C40003AD208F1FF381FFA88F826E725238DE8B5
:105C5000180041483C703C231822412102F056FFB5
:105C60003046F8E6002B3FF40AAF3C4A3C4E118820
:105C7000384A03F11900013B400080B226F81310A6
:105C8000012388F80030157000F030FB354B2046BA
:105C90001D70E0E600293FF755AF06F1FF3B4DE7E9
:105CA0004C46F1E60024A34652E7BB8ADA077FF5AB
:105CB000F4AEB7F81080F0E6BB8AD9077FF5EDAEF9
:105CC000B7F81280E9E62849C85CC0EB090009F181
:105CD000010EC0B201214FF0340B02F803E0FFF7D0
:105CE0009BF8B6681C48019440230B223F210124F5
:105CF000CDF800B002F00AFF40230B223F211648E6
:105D0000CDF800B0019402F083FF2146124803F061
:105D1000C5FA304608F034F9A0EB800000F15F01CD
:105D200009B20F220C4803F0B5FA304608F028F902
:105D300031460246084803F047FC074803F05AFC86
:105D4000E968A879FFF7B2FBAB799DE6E09CFF1FFD
:105D5000889CFF1F0C9CFF1F149CFF1FA29AFF1F13
:105D6000609BFF1F819CFF1FA49CFF1F2DE9F04734
:105D7000DFF808926D4B99F800601B68DFF800A20D
:105D800082B0003601934FF0030018BF0126019F37
:105D90009AF8008004F0E8FA0546042004F0E4FADA
:105DA0000446052004F0E0FA800040EA440406209E
:105DB00004F0DAFA2C4364B25D4944EAC0000A7880
:105DC00080F00F03DBB29A425A4A3CD0176000229F
:105DD00059480B7003788DF800808DF8012053B37B
:105DE000564A12684EF66021BA1A8A4219D8022B16
:105DF00059D0012B5FD0062B48D0032B63D0042B46
:105E000069D0052B77D0072B7DD0082B00F083803D
:105E1000092B68D016B14A4802F05EFC02B0BDE81A
:105E2000F087484A484C0023012123700370136017
:105E3000938089F800103A4669464448FFF746FDCA
:105E40003043C6B2E6E71268BA1A1E2A6BD99AF82E
:105E50000020934222D0394C3D488AF80030012B73
:105E6000276082EA030207609846B1D0042BAFD1C5
:105E700037480068381AB0F5C87FA9D9354C206872
:105E8000381A3228A4D927601A46A1E73A4669464B
:105E90003148FFF71BFD3043C6B2BBE7012B4FF083
:105EA0000002E3D1E4E73A4669462C48FFF70EFDCD
:105EB0003043C6B2AEE73A4669462948FFF706FDC9
:105EC0003043C6B2A6E73A4669462648FFF7FEFCCD
:105ED0003043C6B29EE73A4669462348FFF7F6FCD0
:105EE0003043C6B296E73A4669462048FFF7EEFCD3
:105EF0003043C6B28EE73A4669461D48FFF7E6FCD6
:105F00003043C6B286E73A4669461A48FFF7DEFCD8
:105F10003043C6B27EE73A4669461748FFF7D6FCDB
:105F20003043C6B276E7002252E700BFE09CFF1F75
:105F30008C9CFF1F089CFF1F0C9CFF1F849CFF1F55
:105F4000149CFF1F909CFF1F7A9CFF1F68EE0000AF
:105F5000989CFF1F109CFF1FB0ED0000C0ED0000DB
:105F6000A0ED000060ED0000DCED0000CCED0000D5
:105F700074EE000010EE0000548AFF1F5C8BFF1FC0
:105F8000809CFF1F28B11028044BA8BF1020186068
:105F90007047024B01201860704700BFAC9CFF1F88
:105FA00038B50F4D2B78013B01381B02C4B203F406
:105FB0007063200443F4404343F00C0300F4FE00FC
:105FC000184305F039FB2868013860F03F00C0B283
:105FD00004F060FB2046BDE8384004F05BBB00BF26
:105FE000AC9CFF1F70B5124D2B78013B1B0203F4D4
:105FF0007063064643F430430806320400F0FE4066
:1060000043F00B03034302F4FE0018430C4605F073
:1060100013FB2868013860F04F00C0B204F03AFB6F
:10602000304604F037FB2046BDE8704004F032BB38
:10603000AC9CFF1F70B5124D2B78013B1B0203F483
:106040007063064643F410430806320400F0FE4035
:1060500043F00903034302F4FE0018430C4605F025
:10606000EBFA2868013860F06F00C0B204F012FB50
:10607000304604F00FFB2046BDE8704004F00ABB38
:10608000AC9CFF1F38B5104D2B78013B1B0203F46D
:106090007063044643F41043000443F0090300F422
:1060A000FE00184305F0C8FA2868013860F06F0058
:1060B000C0B204F0EFFA204604F0ECFA0020BDE88C
:1060C000384004F0E7BA00BFAC9CFF1F38B50E4D56
:1060D0002B78013B1B0203F47063044643F45043E6
:1060E000000443F00D0300F4FE00184305F0A4FA89
:1060F0002868013860F02F00C0B204F0CBFA2046C7
:10610000BDE8384004F0C6BAAC9CFF1F08B50020BB
:1061100005F05CFB0028FAD108BD00BF08B564217A
:106120000720FFF75FFF7F210B20BDE80840FFF746
:1061300059BF00BF10B500217B20FFF753FF00249B
:10614000E0B2FFF79FFF0134022004F043F9802CF6
:10615000F6D110BD10B504464FF4406004F04AFA81
:1061600004F0A2FA2CB1102C044BA8BF10241C6020
:1061700010BD024B01241C6010BD00BFAC9CFF1F72
:1061800010B5044641F0E00004F084FA04F07F000A
:1061900004F080FAC4F3C610BDE8104004F07ABAE7
:1061A00038B5134D2B78044641F6FF72A0F5005028
:1061B000824203F1FF33A8BF02461B0202F50052E0
:1061C00003F47063100443F4604343F00E0300F4DF
:1061D000FE005204184302F0FE42104305F02CFA70
:1061E000296801392046C9B2BDE83840FFF7C8BF69
:1061F000AC9CFF1F38B504460D46F02004F04AFA67
:1062000035B1254414F8010B04F044FAAC42F9D13D
:10621000F720BDE8384004F03DBA00BF00B50B4B95
:1062200083B00246998818680090032AADF80410DC
:1062300002D903B05DF804FB684606218DF80520FD
:10624000FFF7D8FF03B05DF804FB00BF14F20000B5
:1062500000B50B4B024683B0186899880090131F55
:106260004C2BADF8041002D903B05DF804FB68466E
:1062700006218DF80520FFF7BDFF03B05DF804FB94
:106280001CF20000030203F4FE43C0F3C6101843DF
:10629000704700BF03784078DB0103F47E5300F0C1
:1062A0007F001843704700BF82B002AA114642F82F
:1062B000040D002012F8013B03F07F03914243EAF2
:1062C0000020F7D102B07047003210B403884FF0BD
:1062D000010404FA01F418BF012202FA01F123EAD1
:1062E00004020A43028010BC704700BF70B5CEB2F2
:1062F0000C46054603F000FC864203D03146284692
:1063000003F014FC0135284603F0F6FB240A84420E
:1063100005D021462846BDE8704003F007BC70BD9B
:1063200038B5054603F0E8FB4FF0000460F30704BE
:10633000681C03F0E1FB60F30F24A0B238BD00BF7E
:10634000F8B504460020FFF7EBFF002C00F0F580C5
:106350004FF4AF610220FFF7C9FF04204FF47A61C8
:10636000FFF7C4FF0B2003F0FFFF002840F061841B
:106370004FF496610620FFF7B9FF4FF4FA61082049
:10638000FFF7B4FF4FF4AF610A20FFF7AFFF40F60D
:10639000FC010C20FFF7AAFF4FF496612220FFF7C3
:1063A000A5FF4FF416612420FFF7A0FF7D212A20CE
:1063B000FFF79CFF0C210E20FFF798FF0121102012
:1063C000FFF794FF02211220FFF790FF0021142015
:1063D000FFF78CFF00211620FFF788FF022118200D
:1063E000FFF784FF01211A20FFF780FF02211C2004
:1063F000FFF77CFF04211E20FFF778FF14212020E7
:10640000FFF774FF01212620FFF770FF03212820EA
:10641000FFF76CFF04212C20FFF768FF0F212E20CF
:10642000FFF764FF00213020FFF760FF0C213220CE
:10643000FFF75CFF00213420FFF758FF00213620D2
:10644000FFF754FF00213820FFF750FF00213A20CA
:10645000FFF74CFF00213C20FFF748FF00213E20C2
:10646000FFF744FF00214020FFF740FF00214220BA
:10647000FFF73CFF1F214420FFF738FF1321462080
:10648000FFF734FF0E214820FFF730FF11214A208B
:10649000FFF72CFF0A214C20FFF728FF00214E2098
:1064A000FFF724FF06215020FFF720FF0221522092
:1064B000FFF71CFF0C215420FFF718FF0021562086
:1064C000FFF714FF00215820FFF710FF01215A2089
:1064D000FFF70CFF03215C20FFF708FF0A215E2075
:1064E000FFF704FF00216020FFF700FF0421622076
:1064F000FFF7FCFE01216420FFF7F8FE0021662073
:10650000FFF7F4FE0B216820FFF7F0FE7F216A20E1
:10651000FFF7ECFE21210020FFF7E8FE0220FFF745
:10652000FFFEB0F5805F034616D34FF4AF61022043
:10653000FFF7DCFE4FF4AF630EE04FF6FF739842B7
:106540003FF406AF212840F0AB830220FFF7E8FEBE
:10655000B0F5805F0346E8D2D24A04201380FFF7EB
:10656000DFFEB0F5805F034680F09B82CE4A0620B6
:106570001380FFF7D5FEA0F52F739BB2B3F57A6FAA
:10658000024606D940F628210620FFF7AFFE40F666
:106590002822C64B08201A80FFF7C2FEA0F52F73F1
:1065A0009BB2B3F57A6F024606D940F6E441082063
:1065B000FFF79CFE40F6E442BD4B0A201A80FFF72D
:1065C000AFFEA0F5FA739BB240F6AC518B42024687
:1065D00006D94FF4AF610A20FFF788FE4FF4AF628F
:1065E000B44B0C201A80FFF79BFEA0F5FA739BB208
:1065F00040F6AC518B42024606D940F6FC010C2015
:10660000FFF774FE40F6FC02AB4B0E201A80FFF73A
:1066100087FE1828034600F27682A84A10201380CD
:10662000FFF77EFE431E9BB20F2B024604D90121C9
:106630001020FFF75BFE0122A14B12201A80FFF70A
:106640006FFE0A28034600F258829E4A14201380E7
:10665000FFF766FE0128034604D900211420FFF746
:1066600045FE0023984A16201380FFF759FE7F2825
:10667000034600F23C82954A18201380FFF750FE33
:106680000228034600F22D82914A1A201380FFF758
:1066900047FE0C28034600F266828E4A1C201380B7
:1066A000FFF73EFE0428034600F257828A4A1E2066
:1066B0001380FFF735FE0928034600F24882874A17
:1066C00020201380FFF72CFE4628034600F2398273
:1066D000834A22201380FFF723FEA0F5FA739BB2B2
:1066E00040F6AC518B42024606D94FF49661222007
:1066F000FFF7FCFD4FF496627A4B24201A80FFF7D7
:106700000FFEA0F5FA739BB240F6AC518B420246E5
:1067100006D94FF416612420FFF7E8FD4FF4166206
:10672000714B26201A80FFF7FBFD7F28034600F2FD
:1067300002826E4A28201380FFF7F2FD06280346E6
:1067400000F2F3816A4A2A201380FFF7E9FDA0F1E5
:1067500032039BB2B3F5967F024604D97D212A20ED
:10676000FFF7C4FD7D22634B2C201A80FFF7D8FD74
:106770000C28034600F2D3815F4A2E201380FFF7D6
:10678000CFFD1E28034600F2C4815C4A30201380EE
:10679000FFF7C6FD0928034600F24582584A322019
:1067A0001380FFF7BDFD1D28034600F23682554ACF
:1067B00034201380FFF7B4FD7F28034600F22782C0
:1067C000514C36202380FFF7ABFD7F28034600F2B3
:1067D000188238206380FFF7A3FD7F28034600F26C
:1067E0000A823A20A380FFF79BFD7F28034600F230
:1067F000FC813C20E380FFF793FD7F28034600F2F5
:10680000EE813E202381FFF78BFD7F28034600F2B7
:10681000E08140206381FFF783FD7F28034600F27B
:10682000D2814220A381FFF77BFD384D2880442090
:10683000FFF776FD3028034600F2BF81344A462038
:106840001380FFF76DFD3028034600F2B081314C14
:1068500048202380FFF764FD3028034600F2A18121
:106860004A206380FFF75CFD3028034600F29381E5
:106870004C20A380FFF754FD3028034600F28581A9
:106880004E20E380FFF74CFD0128034604D9002188
:106890004E20FFF72BFD00231F4A50201380FFF7E7
:1068A0003FFD3BE0EE9AFF1FFA9BFF1F949BFF1FEB
:1068B000EA9AFF1FE89BFF1F589BFF1FC29BFF1F09
:1068C0003A9BFF1F849AFF1F709BFF1F509BFF1F67
:1068D000249BFF1F829BFF1FAE9BFF1F369BFF1F4A
:1068E000F89BFF1FB49BFF1F269BFF1FA29AFF1F51
:1068F000189BFF1F5C9BFF1F5E9BFF1F749BFF1F6E
:10690000809AFF1FF09AFF1F609BFF1FB49AFF1F22
:10691000B69BFF1FD49BFF1F1C9BFF1F431E9BB2F8
:106920000B2B024604D906215020FFF7DFFC06227C
:10693000C64B52201A80FFF7F3FC0428034600F2EE
:106940001E81C34A54201380FFF7EAFC431E9BB20A
:106950001D2B024604D90C215420FFF7C7FC0C2242
:10696000BC4B56201A80FFF7DBFC0128034604D9F4
:1069700000215620FFF7BAFC0023B74A58201380A5
:10698000FFF7CEFC7F28034600F2F380B34A5A207B
:106990001380FFF7C5FC431E9BB2092B024604D9A6
:1069A00001215A20FFF7A2FC0122AD4B5C201A8086
:1069B000FFF7B6FC431E9BB2102B024604D90321FD
:1069C0005C20FFF793FC0322A64B5E201A80FFF7A2
:1069D000A7FC431E9BB21D2B024604D90A215E2050
:1069E000FFF784FC0A22A04B60201A80FFF798FC76
:1069F000022803465DD89D4A64201380FFF790FC6F
:106A00000128034604D901216420FFF76FFC01230C
:106A1000974A62201380FFF783FCC31E9BB2012BB1
:106A2000024604D904216220FFF760FC0422914B46
:106A300066201A80FFF774FC7F2803464BD88E4AE5
:106A400068201380FFF76CFC7F2803463DD88B4AF3
:106A50006A201380FFF764FC7F2830D82B88DFF88A
:106A60003CE2874F874A884D884E894C894903F01C
:106A7000010CAEF800C0C3F3400EA7F800E0C3F36A
:106A800080071780C3F3C007834A2F70C3F3001732
:106A9000C3F34015C3F38013378025800B8010802B
:106AA000F8BD4FF47A610420FFF720FC4FF47A63BD
:106AB0005CE500216020FFF719FC00239BE76A20BA
:106AC0007F21FFF713FC7F20C8E70B216820FFF729
:106AD0000DFC0B23BBE700216620FFF707FC00231A
:106AE000ADE702211820FFF701FC0223CCE50021CD
:106AF0001620FFF7FBFB0023BDE502211220FFF764
:106B0000F5FB0223A1E50C210E20FFF7EFFB0C2380
:106B100083E50F212E20FFF7E9FB0F2335E6042143
:106B20002C20FFF7E3FB042326E603212820FFF7B0
:106B3000DDFB032306E601212620FFF7D7FB012317
:106B4000F7E514212020FFF7D1FB1423C0E5042131
:106B50001E20FFF7CBFB0423B1E502211C20FFF729
:106B6000C5FB0223A2E501211A20FFF7BFFB012389
:106B700093E500215820FFF7B9FB002306E7022127
:106B80005220FFF7B3FB0223DBE60A214C20FFF77C
:106B9000ADFB0A2374E611214A20FFF7A7FB11235E
:106BA00066E60E214820FFF7A1FB0E2358E61321CD
:106BB0004620FFF79BFB132349E61F214420FFF7E4
:106BC00095FB1F233AE600214020FFF78FFB0023AF
:106BD00027E600213E20FFF789FB002319E600216C
:106BE0003C20FFF783FB00230BE600213A20FFF750
:106BF0007DFB0023FDE500213820FFF777FB002314
:106C0000EFE500213620FFF771FB0023E1E50021CD
:106C10003420FFF76BFB0023D2E50C213220FFF775
:106C200065FB0C23C3E500213020FFF75FFB002349
:106C3000B4E540F628210620FFF758FB40F6E44172
:106C40000820FFF753FBFFF79DBB00BF7889FF1FAC
:106C5000AA89FF1FA089FF1FF69BFF1F7C9BFF1FB8
:106C60009E9AFF1F7A89FF1FA889FF1F829AFF1F24
:106C70005A9BFF1F529BFF1F709AFF1FA09AFF1F76
:106C8000B09BFF1F149BFF1FCC9BFF1FA89AFF1FE9
:106C9000809BFF1FB29BFF1FCC9AFF1FEE9BFF1F25
:106CA00017287FF655AB19287FF6C4AB1B287FF653
:106CB000E1AB1C283FF4F6AB1E287FF6FBAB1F2888
:106CC0003FF400AC20287FF425AC17E4F8B577201A
:106CD00006F0C6FB204B214A054603CB1368C5F8D6
:106CE00003001A0C6620C5F807102B80AA70FFF766
:106CF000C9FA2E46002426F80B0FA0B2FFF710FBAE
:106D0000FFF7C0FA0234662C26F8020FF5D16C1E8C
:106D100005F172064FF0FF3014F8013F0827584084
:106D20000F4B40F300017A1E0B4012F0FF0783EA7D
:106D30005000F5D1B442EFD1C043FFF7B5FA3A465F
:106D4000C5F873007721284604F0C4FC2846BDE846
:106D5000F84006F08DBB00BF28F2000024F20000CE
:106D60002083B8EDF0B50E4B0E4C054693E80700B6
:106D700085B024682E88AD7801AB83E80700270C26
:106D8000184600220B21ADF804408DF80670ADF8CE
:106D90000C608DF80E5004F09DFC05B0F0BD00BFF6
:106DA00034F2000024F20000F0B5124B124D1E68C0
:106DB000124F0FCD87B06C460FC495E8030044F81E
:106DC000040B38683B79CDF80D00320C212021806E
:106DD0008DF802208DF81130ADF80060FFF752FAFF
:106DE0000022ADF80B001221684604F073FC07B0D6
:106DF000F0BD00BF24F2000040F2000000EF0000F0
:106E0000002004F0E3BC00BF02F02EBE70B5124CAF
:106E100082B000254023064629462046009301956E
:106E20008023202201F072FE20222946204602F013
:106E300031FA2046012102F037FA304607F0A0F877
:106E400031460246204602F0BFFB204602B0BDE8B4
:106E5000704001F041BC00BF149CFF1FF0B57629C3
:106E600083B075D90546441E00F172064FF0FF301D
:106E700014F8012F08275040404A40F300017B1EC0
:106E80000A4013F0FF0782EA5000F5D1B442EFD177
:106E9000C043FFF709FA0146D5F873000190019A43
:106EA000914202D0B2F17F2F0BD105F10B00FFF719
:106EB000F1F966280BD03248FFF7A8FF002003B095
:106EC000F0BD3048FFF7A2FF384603B0F0BD05F132
:106ED0000D00FFF7DFF9212840D1002440F6AC5621
:106EE00013E004281AD0062821D008281FD00A2829
:106EF00028D00C2822D1A1F5FA7292B2B24201D860
:106F0000FFF7F4F90234662C0ED004F10D0028448A
:106F1000FFF7C0F9022C0146A0B2E2D1B1F5805FC3
:106F2000EED30234662CF0D1012003B0F0BDA1F500
:106F30002F7292B2B2F57A6FE4D8E1E7222801D03D
:106F4000242811D1A1F5FA7292B2B242DAD8D7E769
:106F50000D48FFF75BFF002003B0F0BD0B48FFF7C3
:106F600055FF002003B0F0BD2A28C9D1A1F132029B
:106F700092B2B2F5967FC5D8C2E700BF2083B8EDC4
:106F800084F2000070F2000058F2000098F2000055
:106F900003290CD970B5461C82B005460C46304614
:106FA00003222A4907F05AF810B102B070BD7047A9
:106FB0000B2C05D905222649281D07F04FF840B1B2
:106FC0002448FFF723FF244802B0BDE87040FFF7D4
:106FD000C9BE05F10901032201A807F08FF801A835
:106FE00003221E4907F03AF8D8B103221C4901A830
:106FF00007F034F808B301A803221A4907F02EF865
:10700000B0B91948FFF702FFA11E89B23046FFF759
:1070100025FF0028C9D0154802B0BDE87040FFF731
:10702000F5BE1348FFF7F2FEFFF750FE1148F3E7F5
:107030001148FFF7EBFE1148C6E71148FFF7E6FEDF
:1070400002B0BDE87040FFF7AFBE00BF24F2000001
:1070500008EF0000B0F20000C4F20000C8F2000027
:10706000F0F2000008F300000CF3000020F3000031
:10707000CCF20000E0F2000034F3000048F300001E
:10708000F4F200002DE9F043174D2B6883B08146E0
:107090000F469046F3B1154E34880A1992B218463D
:1070A0001146328006F05AFD28603A46494620448F
:1070B00002F06CFDB8F1000F09D031882868FFF7A5
:1070C00067FF286806F0D4F900232B60338003B0F3
:1070D000BDE8F083054E01930846318006F0C0F903
:1070E000019B28601C46E0E7B49CFF1FB09CFF1F7B
:1070F00010B51F4C4FF4FA70FCF7A8FD204601F0C4
:10710000DFF900221146204602F0C4F82046012192
:1071100002F0CAF82046002102F0C0F80B221549FF
:10712000204602F051FA204602F064FA0F2212497A
:10713000204602F049FA204602F05CFA0F49072285
:10714000204602F041FA204602F054FA204601F0AF
:10715000C3FA0B4B0B4A1A604FF4FA70FCF776FD3A
:10716000FFF722FE0848BDE81040FFF74FBE00BF02
:10717000149CFF1F4CF3000058F3000068F300005C
:107180006C9EFF1F8570000070F3000000207047A8
:1071900090F8392090F83800101A704790F838307D
:1071A00090F839209A4205D95A1C034480F83820B7
:1071B000187E70474FF0FF30704700BF90F83830AE
:1071C00090F839209A4286BF1B18187E4FF0FF3086
:1071D000704700BF704700BF38B50546B0F85E0085
:1071E00090B195F85D301446C3F1210294420CD859
:1071F00005F13B001844224602F0C8FC95F85D30CA
:10720000234485F85D30204638BD0120144628719E
:10721000EEE700BFB0F85E306BB190F85D30202B28
:1072200007D8C218013380F85D30012082F83B1086
:107230007047012303710020704700BF002342699B
:1072400080F8383080F8393080F85C3080F85D3074
:1072500080F85E3080F85F3006CA30B40D6804698B
:1072600043662A4383660A60A370426990F86130DE
:107270001649146813441D7A5B7B01EBC5051B029C
:107280006D6803F4E06343F064032B6090F86230B0
:1072900013449D7CDB7D01EBC5011B02496803F4AF
:1072A000E06343F064030B6021685368194205D022
:1072B000036927225A70036904229A710369202204
:1072C0005A71036980229A7030BC7047A4FE000096
:1072D00043690CCB12681A420CD0094B99420AD967
:1072E000084B9942036994BF1A220D225A70036910
:1072F00004229A717047036927225A70F7E700BF8A
:107300007F1A06003F420F0010B50269D378DBB246
:10731000D90604463DD510215806D17038D503F062
:10732000040303F0FF02002B51D03D49626E00239D
:107330000B7084F85D30002A5BD0904794F85D3084
:10734000002B56D02369D0229A70236994F83B20F1
:107350001A712369012284F85C200222DA7010BDC0
:10736000304B84F860009C424AD02F4B9C4252D054
:1073700094F8391013791F29DBB207D82848007810
:1073800020B16018013184F8391003760223D370DC
:1073900010BD5906C3D4917801F0100101F0FF002F
:1073A0000029DDD013F001031ED194F85C1094F88D
:1073B0005D00884281BF4B1C091984F85C3091F84C
:1073C0003B3013712369D0229A702269DEE723696A
:1073D00084F83920C0229A702369114A1979012151
:1073E00011700222DA7010BDC023937022691379E4
:1073F000CCE70122002384F85D2084F83B30A1E72C
:10740000626994F86130094913440322187A02F042
:1074100043FD2269ACE7626994F861300449F3E7FF
:10742000B89CFF1F548FFF1FC08FFF1F9174000077
:107430009D7400000369DB7803F0200373B190F8BA
:1074400060300133DBB2012B80F860301AD9426919
:1074500090F861301344187A02F09ABD70B5426911
:1074600003F0FF0590F8613013440446187A02F0E7
:107470008FFDA36E5BB184F8385094F83900BDE8F5
:107480007040184790F85F30002BE0D0704770BD17
:107490000148FFF7CFBF00BF548FFF1F0148FFF720
:1074A000C9BF00BFC08FFF1F2DE9F047374FDFF87E
:1074B000E0903B68026982B006460093DDF80080E8
:1074C0000021A025D3789B065BD53B680193019BE7
:1074D000C8EB03030F2BF5D949B1102BF2D00020D4
:1074E0009070336980229A7002B0BDE8F0877269AB
:1074F00096F8613013440521187A02F043FF72694F
:1075000096F861301344012193F812A0504602F01E
:1075100039FF09240021504602F020FF2B46013B91
:10752000FDD10121504602F019FF2B46013BFDD150
:10753000013CEFD1706996F8611001444FF4A072DC
:107540000C7A4B7B09EBC4011B02496803F4E0632E
:1075500043F064030B6096F862300344997CDB7D52
:1075600009EBC1011B02496803F4E06343F06403C3
:107570000B60013AFDD13269D3789B064FF00101CF
:10758000A3D4012002B0BDE8F08700BFE09CFF1F3C
:10759000A4FE0000F0B503691222DA700269937844
:1075A00003F0200385B004460D46002B5ED0B423C3
:1075B00093703C4922690B680093009E05E00B68BC
:1075C0000193019B9B1B042B42D8D37803F020032B
:1075D00003F0FF00002BF2D094F85D30002B31D087
:1075E0004FF0000E4FF0020C04EB0E0393F83B300B
:1075F00013710B680393039F206907E09B060DD569
:107600000B680293029BDB1B052B28D8C378DBB2E7
:1076100003F0020202F0FF06002AEFD080F803C058
:107620002669F378DBB2DF0632462DD49F062BD5D0
:10763000DB0731D40EF1010E94F85D305FFA8EFE57
:107640007345D1D800201DBB002384F85E3004E0D0
:107650009070236980229A70042005B0F0BD867076
:107660002369802204209A7005B0F0BD03F0FF0664
:10767000FFF71AFF10B9042005B0F0BD236984F8A4
:107680005F60B0229A7094E78023B3700420DAE739
:1076900026698023B370D7E7BEF1000F0CBF02202C
:1076A0000320F6E7E09CFF1F2DE9F0410669002565
:1076B000122780F8385080F83950F770D0F810C091
:1076C0009CF802E00EF0200E88B00446884615466D
:1076D0001E46BEF1000F49D0B4238CF80230784B1F
:1076E00021691A680092DDF800E006E01A6801924C
:1076F0000198CEEB0000042830D8C87800F02000B4
:1077000000F0FF070028F1D04FEA480242F00102E2
:10771000D2B20A711A680292DDF808E0206906E028
:107720001A6803920399CEEB010105292AD8C17882
:1077300001F0020101F0FF070029F1D04FF0020C27
:1077400080F803C02269D17811F0110722D12DBB36
:10775000002E0CBFA0238023937003E08F70236959
:1077600080229A70384608B0BDE8F0810EF0FF071D
:10777000FFF79AFE0028F5D0236984F85F70B022E5
:107780009A70ACE787702369802238469A7008B0F7
:10779000BDE8F081802393700027E3E7012D75D0C9
:1077A000A021917021690A79BE4667464FF0A80C66
:1077B0001A680492049805E01A680592059A121A4C
:1077C000052A4AD8CA7802F0020202F0FF08002A0D
:1077D000F2D0CF702169CA78D2B212F0100F0846E9
:1077E0005AD1920658D5013DEDB2012D49D0BEF1D6
:1077F0001F0F3BD90A79012DDAD11A680692069D2E
:1078000005E01A680792079A521B052A46D8C278E3
:1078100002F0020202F0FF01002AF2D00223C3703C
:107820002269D378DBB2D9063AD49B0634D5B0238B
:10783000BEF11F0F93703FD8226904EB0E0312793B
:107840001A760EF1010E5FFA8EFE16B123698022C0
:107850009A7084F839E0774684E781F802802369DA
:1078600080229A70774684F839E07BE704EB0E02B9
:1078700091F8048082F818800EF1010E5FFA8EFEF6
:10788000B9E781F802C021690846B0E7A8219170E4
:107890002069BE460279B0E7774663E78170DEE78C
:1078A0001021A023D170013BFDD12269937803F010
:1078B000F7037746937055E723691B79C5E700BF47
:1078C000E09CFF1F0148FFF71FBD00BF548FFF1F43
:1078D0000148FFF719BD00BFC08FFF1F704700BFF1
:1078E00038B5144C037801225B000546204684F825
:1078F0003B3084F85E2084F85D20FFF78BFC204647
:107900000021FFF747FE0B4C2978012320461A4639
:10791000FFF7CAFE0128F6D194F8383094F83920E0
:107920009A4205D9E218013384F83830107E38BD08
:10793000FF2038BD548FFF1F38B51B4C0378012240
:107940005B000546204684F83B3084F85E2084F8CE
:107950005D20FFF75FFC20460021FFF71BFE124C65
:107960002978204601230222FFF79EFE0228F6D145
:1079700094F8382094F839108A420FD2531CDBB2A5
:10798000A018994284F83830007E0AD92344023284
:107990001B7E84F8382040EA032038BD4FF6FF7084
:1079A00038BD40F47F4038BD548FFF1F0C2901D9EA
:1079B000002070470231490001F0FE01FFF7BCBF13
:1079C00070B50C4C0378164601255B00204684F800
:1079D0003B3084F85E5084F85D50FFF71BFC314665
:1079E0002046FFF717FC29462046BDE87040FFF708
:1079F000D1BD00BF548FFF1FF8B505460F46164690
:107A0000412421463A462846FFF7DAFF611C02343A
:107A1000C9B232462846E4B2FFF7D2FF592CF0D162
:107A2000F8BD00BF38B504460D463548FFF706FCE3
:107A30006322802120462570FFF7C2FF012002F05B
:107A4000C9FC204600225E21FFF7BAFF20465D21D7
:107A5000FFF746FF242801D0002038BD204606222B
:107A60000C21FFF7C9FF204601222B21FFF7A8FFB9
:107A7000204601222C21FFF7A3FF20460E222D21B4
:107A8000FFF79EFF204600222E21FFF799FF204698
:107A900001222F21FFF794FF204605223021FFF716
:107AA0008FFF204601223121FFF78AFF2046002266
:107AB0003221FFF785FF204600223321FFF780FFA8
:107AC000204600223421FFF77BFF2046002235218B
:107AD000FFF776FF204600225B21FFF771FF20466B
:107AE00010225C21FFF76CFF204620225D21FFF76A
:107AF00067FF20468F225E21FFF762FF012038BD1D
:107B0000548FFF1F10B4047F4160022CC26002D06A
:107B100010BC01F0D7BB836810BC184790E80C007C
:107B2000F0B41C6859682568164F174E2943216028
:107B3000164D17491760D66015611160417A154AD4
:107B40005C180A3194F8244053F8215002EBC40128
:107B500049680D60017A5C1803EB8101247ECD69D0
:107B600002EBC40149680D60817A581803EB810368
:107B700090F83000596B02EBC002F0BC53681960FA
:107B8000704700BF01401F0001100038011000784D
:107B900000001F80A4FE0000704700BFF0B50C1E5F
:107BA000BDF8146034DBB0F906701919B942C4BFCE
:107BB0003B1B1BB2002BA6461CDD002A1146B8BF9A
:107BC000D11D02F00705CC10826A012007FB04E1F9
:107BD000A840012E0A44C0B21ED00CD3022E09D1F7
:107BE000013B12FA83F3013A12F8011F41409A4215
:107BF0001170F9D1F0BDC043013B12FA83F3C0B25A
:107C0000013A12F8011F014093421170F9D1F0BD01
:107C100023441BB20024C6E7013B12FA83F3013A66
:107C200012F8011F01439A421170F9D1F0BD00BF53
:107C3000F8B50D1E0EDB14461F46064601F03AFB52
:107C4000A84207DD002C05DB304601F037FBA042DF
:107C500001DCF8BDF8BD304601F02AFB022853D004
:107C600003284BD0012806D16540F3886C4065405D
:107C7000013B5D1B2DB2012F03D02AD3022F14D05C
:107C8000F8BD002C2246B6F90630B06AB8BFE21D36
:107C900042F3CF0202FB035504F00704435D0121C8
:107CA00001FA04F41C434455F8BD002C2246B6F9F1
:107CB0000630B06AB8BFE21D42F3CF0202FB0355A3
:107CC00004F00704435D012101FA04F45C404455CB
:107CD000F8BD002C2246B6F90630B06AB8BFE21DE6
:107CE00042F3CF0202FB035504F00704435D012178
:107CF00001FA04F423EA04044455F8BD3389013B36
:107D0000591B25460CB2B6E7F18832890139013A90
:107D10004D1B141B2DB224B2ADE700BF2DE9F0417D
:107D2000079E9DF91880089D04461F4600F0C0FF7D
:107D30000D4B0E480E4984F83380FF22002F08BFF8
:107D40001F4684F82F20002384F8302084F8312047
:107D500084F832202060A665E5656762616523626C
:107D6000A3622046BDE8F081548FFF1FFCF30000A2
:107D70000110013810B50446806A034B236008B136
:107D800005F076FB204610BDFCF30000F8B5436A11
:107D9000DBB190F82C200125AA4083F83B2083F822
:107DA0005E5083F85D500446406A03680E461B68C7
:107DB00000219847606A036831461B689847294646
:107DC000606ABDE8F840FFF7E5BBC26BC56C13689D
:107DD000046A23EA050313604CB122684FF00043A4
:107DE000D3625163D36A002BFCDA936BF8BD836BCB
:107DF000466B0825802410E03768426C3A433260B5
:107E00001F68826C3A431A601A68876C013D22EA47
:107E100007024FEA54041A6007D02142ECD13268BD
:107E2000476C22EA07023260EAE7F8BD70B5044603
:107E3000406A0D4600282BD0A16DFFF749FA002DAE
:107E400020460CBFA621A721FFF7A0FF606A20B142
:107E5000E16DBDE87040FFF73BBA216C226D086808
:107E6000236A02430A6093B1DA7A82B1D00703D55C
:107E7000224A99691160DA7A910703D5204AD969B3
:107E80001160DA7A520702D51E4A1B6A136070BD70
:107E9000236A002B2BD0D97A626DE1B172B6D97A00
:107EA000CE0706D51848D968066831409961016047
:107EB000D97A880706D51548196906683140D9610D
:107EC0000160D97A4E0705D51148596906683140D5
:107ED0001962016062B61B68D968914207D00D48EB
:107EE00018600D49DA6042F0804018611960226C18
:107EF000216D136823EA01031360A0E700E100E0AD
:107F000004E100E008E100E080E100E084E100E05D
:107F100088E100E001403F0000003F80436A2DE916
:107F2000F04105460E469046002B3ED090F82C10AE
:107F30000124A14083F83B1083F85E4083F85D4044
:107F4000406A036800211B6808F1FF379847FFB2B9
:107F5000B8F1000F23D03744A046013E686A16F8F6
:107F6000011F03681B6898470134B742E4B216D07A
:107F7000202CF3D10121686AFFF70CFB95F82C2027
:107F80006B6A520083F83B2083F85E8083F85D8043
:107F9000686A036800211B6898470124DEE7686A65
:107FA0000121BDE8F041FFF7F5BAC26BC16C13685F
:107FB00023EA010306EB080413604FF00048A642D1
:107FC0000ED02B6A16F801EB63B11A68C2F82C8048
:107FD000C2F834E0D36A002BFCDAA642936BF0D1EE
:107FE000BDE8F081AB6BD5F834C008208021DCF807
:107FF00000206F6C1EEA010F14BF3A43BA43CCF85D
:1080000000201A68AF6C3A431A601A68AF6C0138E6
:1080100022EA07024FEA51011A60E8D1CFE700BF18
:1080200070B50446406A0D46002828D0A16DFFF7C0
:108030004FF920462946FFF7A9FE606A20B1E16D9D
:10804000BDE87040FFF744B9216C226D0868236ACF
:1080500002430A6093B1DA7A82B1D00703D5234A8A
:1080600099691160DA7A910703D5214AD9691160BB
:10807000DA7A520702D51F4A1B6A136070BD236A61
:10808000002B2BD0D97A626DE1B172B6D97ACE07C6
:1080900006D51948D9680668314099610160D97AD6
:1080A000880706D51548196906683140D96101600D
:1080B000D97A4E0705D512485969066831401962C8
:1080C000016062B61B68D968914207D00D481860FC
:1080D0000D49DA6042F0804018611960226C216D10
:1080E000136823EA01031360A3E700BF00E100E087
:1080F00004E100E008E100E080E100E084E100E06C
:1081000088E100E001403F0000003F802DE9F041A0
:10811000044686B0806A9DF830801E460F4615469C
:10812000B4F90830002800F04281DA1D48BF03F19D
:108130000E02B4F90630D21003FB02F2002105F062
:10814000BBFCB4F90820202A00F39280B4F9061091
:10815000A34B0120203A733902EBD27201EBD171AB
:108160004FF0200E029073208DE8014042F34F0241
:1081700041F34F01204600F051FE606A84F82D70F3
:10818000002800F04D81002D40F08A80B4F90830BD
:10819000202B14BF3D253C2584F82C50B8F1000F4E
:1081A00040F0858006B394F93300002818DBC0B294
:1081B000012102F0E7F8012194F8330002F0CEF833
:1081C000012002F007F9002194F8330002F0C6F80C
:1081D0000A2002F0FFF8012194F8330002F0BEF803
:1081E000606A002800F08280A16DFFF771F8042218
:1081F0007C492046FFF792FE217A0139C9B2204618
:10820000FFF7C4FD784904222046FFF787FE94F962
:108210002D30012B14BF142110212046FFF7B6FD8D
:10822000042272492046FFF779FEB4F90630802B0C
:1082300000F09280602B00F0A680D9212046FFF745
:10824000A5FD94F92D30012B14BFF12122212046E8
:10825000FFF79CFD204606226549FFF75FFE606A36
:1082600050B3E16DFFF734F8012006B0BDE8F081AE
:10827000B4F906105F4B0120403A52394FF0400EDE
:10828000029002EBD272522001EBD1718DE80140D5
:1082900042F34F0241F34F01204600F0BFFD6CE76F
:1082A0006DB284F82C50B8F1000F3FF47BAFFEF7AD
:1082B000C5FF002E94D076E7216C226D0868236AF2
:1082C00002430A6073B1DA7A62B1D00703D54A4A31
:1082D00099691160DA7A91077CD4520702D5474A2E
:1082E0001B6A1360012006B0BDE8F081236A002BF1
:1082F0002BD0D97A626DE1B172B6D97ACF0706D5A3
:108300003F48D9680568294099610160D97A8E078C
:1083100006D53C48196905682940D9610160D97AB8
:108320004D0705D53848596905682940196201602B
:1083300062B61B68D968914207D034481860344946
:10834000DA6042F0804018611960226C216D136878
:1083500023EA010313604AE7B4F90830202B00F048
:108360008680402B7FF469AF2A4920460322FFF71D
:10837000D5FD94F92D30012B14BFCF219F2120462C
:10838000FFF704FD59E7B4F90830102B7FF455AF1F
:10839000214920460322FFF7C1FD94F92D30012B1E
:1083A00014BFAF2110212046FFF7F0FC45E7DA1D8E
:1083B00048BF03F10E02B4F90630D21003FB02F2FB
:1083C0001046059205F04CF8A06200283FF44DAF2E
:1083D000059AB3E6114AD9691160DA7A7DE700BFE0
:1083E00054F4000034F6000038F600003CF60000BB
:1083F00040F6000048F6000000E100E008E100E07F
:1084000080E100E084E100E088E100E001403F001D
:1084100000003F8050F4000008F9000004E100E093
:10842000012194F83100244F01F0ACFF94F83200A0
:10843000012101F0A7FF94F9312094F9323057F867
:108440003220E26357F83330206A23640125E56463
:1084500025651A682A431A6078B1B8F1000F3FF415
:1084600028AFFFF75BFB002E3FF4BAAE9BE6042279
:1084700012492046FFF752FDDFE6294694F82F0007
:1084800001F080FF294694F8300001F07BFF94F959
:108490002F2094F9303057F83220626357F8333088
:1084A0006564A5641A68A36322F001021A60002EB5
:1084B0003FF496AE77E600BFA4FE00004CF4000047
:1084C000B0F90820D31D48BF02F10E03B0F9062011
:1084D000806ADB1002FB03F2002105F0EDBA00BF59
:1084E000F0B50029BDF814502EDBB0F90660B1429A
:1084F0002ADA002A59DBB0F9087014461C44BC4241
:10850000C4BFBB1A1BB2002B1EDDD2B2D408D0F8F8
:1085100028E016FB041112F00702DBB20EEB010497
:1085200021D0C2F10807FAB2374F9342BF5C0CD298
:10853000C3EB020CFF2646FA0CF6012D07EA0607EC
:108540003FD005D3022D36D0F0BD012D39D030D229
:108550001EF8016026EA07070EF801709342F3D374
:10856000B0F906100C449A1AD2B2072A10D9022D7B
:1085700036D0002D14BFFF26002613462670083B78
:10858000B0F90610DBB2072B0C44F7D802F0070253
:10859000002AD9D01D4B012D9B5C1DD017D3022D75
:1085A000D2D1227853402370F0BD13441BB2002275
:1085B000A1E7022D25D11EF8016077400EF8017069
:1085C000CCE71EF8016037430EF80170C6E7227849
:1085D00022EA03032370F0BD227813432370F0BD19
:1085E00011462378DB4323700839B0F90630C9B24D
:1085F00007291C44F5D812F00702A5D0034B9B5C59
:10860000CFE73444AFE700BFECF30000DCF3000039
:1086100070B4C47DBDF80C50022C18D0032C1FD0B0
:10862000012C0BD0002A03DBB0F90840944201DC96
:1086300070BC7047039570BCFFF7B0BAC48803954F
:10864000013CA41A0A4621B270BCFFF749BF068953
:10865000C488013E641AB21AE41A12B221B2E1E7E8
:1086600004890395E41A641A114622B270BCFFF71C
:1086700037BF00BF70B4C57DBDF80C60022D1AD0A5
:10868000032D12D0012D03D0039670BCFFF728BF35
:10869000C488E41AA41A0A4621B2002A03DBB0F9FE
:1086A0000840944213DC70BC70470489013C641A92
:1086B000114622B2F1E7C48805890396013CAD1A40
:1086C000ED1A621A11B22AB270BCFFF709BF039605
:1086D00070BCFFF763BA00BF2DE9F8430446406A57
:1086E000002863D0A16DFEF7F3FD052274492046F2
:1086F000FFF714FCA1790139C9B22046FFF746FB08
:10870000B4F90820E588A66AD31D48BF02F10E031C
:10871000DB10626A15FB03F51FFA85F8002A7BD08F
:1087200094F82C300125AB4082F83B3082F85E5043
:1087300082F85D50606A036840211B6808F1FF37CA
:108740009847BFB2B8F1000F23D03744A846013E86
:10875000606A16F8011F03681B6898470135B74225
:10876000EDB216D0202DF3D10121606AFEF712FF81
:1087700094F82C20636A520083F83B2083F85E80D3
:1087800083F85D80606A036840211B689847012573
:10879000DEE70121606AFEF7FDFE606A002800F056
:1087A0008D80E16DBDE8F843FEF792BD236A002B92
:1087B0002BD0D97A626DE1B172B6D97ACE0706D5DF
:1087C0004048D9680568294099610160D97A8D07C8
:1087D00006D53D48196905682940D9610160D97AF3
:1087E000480705D53948596905682940196201606B
:1087F00062B61B68D968914207D035481860354980
:10880000DA6042F0804018611960226C216D1368B3
:1088100023EA0103136068E7E26BE36C1168276ADF
:108820000B4306EB080913604FF0004E4E450DD088
:1088300016F801CB2FB33A68C2F82CE0C2F834C066
:10884000D36A002BFCDA4E45936BF1D1226C236D79
:1088500011680B43136097B1FB7A83B1D90703D535
:108860001D4BBA691A60FB7A9A0703D51B4BFA694C
:108870001A60FB7A5B0702D5194B3A6A1A60BDE8A9
:10888000F883A36BD4F8348008208021D8F8002026
:10889000656C1CEA010F14BF2A43AA43C8F80020E4
:1088A0001A68A56C2A431A601A68A56C013822EA76
:1088B00005024FEA51011A60E8D1B7E7276AC5E718
:1088C000E4F3000080E100E084E100E088E100E002
:1088D00001403F0000003F8000E100E004E100E0D3
:1088E00008E100E02DE9F04F85B09946BDF93870F8
:1088F000BDF83CA0BB1AC1EB090B002BB8BF5B4213
:10890000BBF1000FB8BFCBF1000B5B450D4616461F
:108910000093804648DC4D453A4633464CDC1946C8
:1089200013460A46C5EB09019B1A89B2002B0CB20B
:10893000B8BF5B4204EBD474BE42ACBF4FF0FF3211
:1089400001224D45039102924FEA640429DC9BB257
:1089500001930DE0D8F80070BF69B847019BE41A95
:10896000A3B21CB20135002C2DB211DBA94518DBD6
:10897000009B5B452A46534631464046EADCD8F820
:10898000002053469769294632464046B847E5E7F6
:10899000029A1644039AA94502EB030436B224B2A4
:1089A000E6DA05B0BDE8F08F4A462B46B9463546B3
:1089B0004D4517461E46B2DD304629463E464D46D9
:1089C00007468946AEE700BF10B404682469A44690
:1089D00010BC604730B40468BDF808500295A46B21
:1089E000A44630BC604700BF30B40468BDF80850EE
:1089F0000295E46BA44630BC604700BF70B40468C5
:108A0000BDF90C60BDF8105003960495246CA44683
:108A100070BC6047704700BF10B582B0B0F90C2041
:108A200001910168009200220C6CB0F90A301146E5
:108A3000A04702B010BD00BF704700BF01F00301A6
:108A40000129C17506D0032904D0C2880389428157
:108A5000838170470289C38842818381704700BF48
:108A60002DE9F0410568134E6F6986B0B7420446A0
:108A7000BDF8308010D1013B13441BB20093CDF8F8
:108A800004800B46AD6A2046A8472368DB6AB342E0
:108A90000AD106B0BDE8F081059304920391B8476E
:108AA00003A925680EC9E6E7204606B0BDE8F041F7
:108AB000184700BF158A00002DE9F0410568124EE5
:108AC0006F6986B0B7420446BDF830800FD1013BD4
:108AD000CDF804800B4400921BB2AD6A2046A84733
:108AE0002368DB6AB3420AD106B0BDE8F081059382
:108AF00004920391B84703A925680EC9E7E7204609
:108B000006B0BDE8F0411847158A00002DE9F04F86
:108B10000568DFF858B06F6985B05F450646BDF956
:108B20003890BDF83CA00C46904615D11F19BC42A8
:108B30000CDACDF800A0214601342D6A4B4642469E
:108B4000304624B2A847BC423568F2DBEB6A5B458D
:108B500007D105B0BDE8F08F0393B8473568039B94
:108B6000E4E7304605B0BDE8F04F1847158A00002D
:108B70002DE9F04387B099420546BDF93840BDF86C
:108B80003C6025D0A24212D00768DFF88080D7F879
:108B90001490C14532D18DE850002846BC6AA047E8
:108BA0002B68DB6A434524D107B0BDE8F0839942C6
:108BB00002DD08461946034628680E96C46B013349
:108BC0005B1A1BB22846A44607B0BDE8F0436047D5
:108BD000A24202DD134622461C4628680E96631CFC
:108BE000846B9B1A1BB22846A44607B0BDE8F0432D
:108BF0006047284607B0BDE8F04318470593049244
:108C00000391C84703A92F680EC9C4E7158A00005D
:108C10002DE9F04FD0F800E0DFF89090DEF814B0C6
:108C200083B0CB450446BDF93080BDF834A00D4675
:108C300017461E4631D1CDF800A0DEF824B02946F3
:108C400033463A462046D8472368CDF800A008F1BD
:108C5000FF323A44D3F824B0294612B233462046B4
:108C6000D8472368CDF800A02946D3F820B03A466B
:108C700043462046D8472068CDF800A0711E2944FD
:108C80004346056A09B23A462046A8472368DB6A8C
:108C90004B4506D103B0BDE8F08FD847D4F800E0CB
:108CA000C9E7204603B0BDE8F04F1847158A000019
:108CB000F0B4002401264FF6FF75094F07600471D8
:108CC000C475C48104824476C46186750676858243
:108CD0004582C180028141818281F0BC704700BF22
:108CE00014F900002DE9F04F85B00668BDF8445036
:108CF000BDF93880CDF8008004460195D6F848B01B
:108D00000392BDF93C60BDF9407089469A46D84748
:108D100023680195009742465146D3F84880204683
:108D20003346C0472068039B0E930F95856C4B46D6
:108D30003A4631462046AC4605B0BDE8F04F6047A4
:108D40002DE9F04F87B01746BDF940400091254608
:108D5000E91D059344BF2B4603F10E010268BDF8DF
:108D6000486053690294C91003912B49BDF94440EE
:108D700001968B42824645D1002C3CDD029B3C444F
:108D80005E1EB6B24FF0000923B2049301364D4681
:108D9000029B002B28DD059B002403EB090806E05D
:108DA000EDB22B0604F1010411D4A6421CD0A1B2ED
:108DB00011F0070F23B24FEA4505F1D1002BB8BFE0
:108DC0000733DB10013418F803502B06EDD5009B58
:108DD000D2F818B019443A4609B2019B5046D84718
:108DE000A642DAF80020E2D1039B01379944049BA4
:108DF0003FB2BB42CCD1D36A074A934206D107B0F7
:108E0000BDE8F08F9847DAF80020B5E7504607B084
:108E1000BDE8F04F184700BF158A000070B4BDF9D7
:108E20000C60BDF91050BDF81440039604950594EC
:108E300070BCFFF785BF00BF2DE9F04F93B090469F
:108E40000591C1691090BDF870000790BDF874904D
:108E50009DF878A00493002900F0CD800A7A0AC911
:108E6000894604998A1AD2B203EBC203BAF1010F00
:108E7000DA780B9293F905201E8893F802B00F92CE
:108E800093F9064079D913B2099323B20C93109B3E
:108E90001A68A94B1193194653698B4240F0A6807A
:108EA0000B9B002B55D01FFA88F300210D93C84669
:108EB0002344DDF8409006910E930F460C46BBF11B
:108EC000000F3FD0BDF818100C9B03971FFA8AF0D3
:108ED000CB1813FB00F304900E9801440D98034443
:108EE00009B21BB20A910893002505E00135EBB2E7
:108EF00064009B45E4B222D9039B2B44590703D15C
:108F0000731C18F806409EB22306EFD5099BBDF8E6
:108F10001000E91811FB00F10598BAF1010F0FFAE2
:108F20008AF301441CD0079801900093D26909B2DA
:108F300017464846089AB847D9F80020D6E7039F55
:108F40005F44FFB2069B0B9901330693DBB2994253
:108F5000B5D8D36A119A934243D113B0BDE8F08FCC
:108F60000F9B191893690A9A29441F4609B2079B57
:108F70004846B847D9F80020B8E700230C93099376
:108F800085E70A9A0D9B0132013B52B213F0FF03B1
:108F90000A920D936FD1DDF81890079BDDF83C80A5
:108FA000DDF820A04B4517D0BAF1010F00F0C880C2
:108FB0000B9A109DCDF804900BEB8B014FEACB037D
:108FC0000A4400931146DEF81C405346424609B25B
:108FD0002846A047D5F800E0DEF82C30119A9342DD
:108FE000BBD0109813B0BDE8F04F1847109D28462D
:108FF00098472A6854E7109A0598B2F90A308342D4
:10900000ABDDB2F90C304345A7DD062313FB0A03A1
:10901000002BA2DD08EBCA03002B9EDD537E2BB98B
:10902000049BAF2B02D90133DBB20493109BD3F81E
:1090300000E0414B11931A46DEF81430934240F0A1
:109040008E801FFA88F30E9308339BB2BDF814206C
:10905000059305230D9300230A93CDF83C800FFA66
:109060008AF3DDF84080CDF818900B921FFA8AFB46
:10907000CDF820A099460A9ABDF810000B9C0E9DD1
:109080000523194611FB00232C481146C75C0397A2
:1090900002FB0B4214FA81F312B21BB209920C9339
:1090A0002C462E461CE0089B0999012B2AB24B4600
:1090B00040462DD0079F0197CDF80090DEF81CA008
:1090C000D047D8F800E0039B5B0801340393059B6D
:1090D000A4B25D445E44A342ADB2B6B23FF451AF18
:1090E000039BD807DFD4079B069A9342EBD0089BDB
:1090F000012B16D0069B0193CDF80090DEF81CA042
:1091000009994B4632B24046D047D8F800E0DAE73A
:10911000DEF818A0079B0C9922B2D047D8F800E0DF
:10912000D1E7DEF818A00C991346404622B2D0478A
:10913000D8F800E0C7E700BF158A000064F9000016
:109140000B99109DCDF800900531DEF8204009B252
:10915000424608232846A047D5F800E03CE7109C8B
:1091600020469847D4F800E06BE700BFF0B5C3692C
:1091700085B004462BB30A2968D00D294AD01A7A43
:10918000914247D3587A884244D35D688A1A05EBE6
:10919000C205AA78002A50D0E87800284DD0207E59
:1091A00000283AD095F905E0B4F90E00A67DB4F98F
:1091B0000A70724406FB0202BA4262DCB4F9102063
:1091C00030E00A2956D00D2924D0027E002A4BD047
:1091D000B0F90E00A57DB4F90A60062212FB050263
:1091E000B2423EDD228AE38102EBC50212B218468A
:1091F0002282A78A668A02950B468DE8C000014646
:109200002046FFF719FEA37DE28903EB430302EB3F
:109210004303E381012005B0F0BDA67DB4F90E0043
:10922000B4F91020B4F814E0678A02960B468DE872
:10923000804001462046FFF7FFFD2979E389A27DA2
:10924000012001FB0233E38105B0F0BD0022C281A1
:109250009A7A817D038A01FB02330382012005B0E3
:10926000F0BDB4F91020C4E7857DB4F91020B0F941
:109270000E00BEE7028A817DC38102EBC103038237
:10928000C8E70020E0819B7A228A03FB062212B203
:109290002282C7E7C1810282704700BF002908BF50
:1092A00001218175704700BF81824182704700BFF4
:1092B000C07D7047B0F90A00704700BFB0F90C00DC
:1092C000704700BF10B4EFF3108272B6437F33B91A
:1092D000017F012907D003290FD00123437702B969
:1092E00062B610BC7047124C2168A1B111494361AC
:1092F0000B68836108605861EFE70F4C216881B10A
:109300000E4943610B688361086058610C4B4FF054
:1093100080511960E1E7074B41618161206018606D
:10932000DBE7064B4161816120601860EEE700BF1A
:10933000CC9CFF1FC89CFF1FBC9CFF1FC09CFF1F35
:1093400004ED00E070B5EFF3108272B60C4C2068AB
:1093500080B10C4E00254369236073B19D6102B951
:1093600062B6457783689847EFF3108272B620683B
:109370000028F0D102B962B670BD3360EFE700BFDC
:10938000BC9CFF1FC09CFF1FFFF7DCBF184A30B416
:109390001468002C27D0036821688B420ED2CB1AA8
:1093A00000218460C1602360E060106002230375C7
:1093B00030BC704711688B42144608D3A2685B1A10
:1093C0000360002AF6D18260C460A060EEE7D26834
:1093D000C2608460E060C568CB1A0222A860236086
:1093E000027530BC70478460C4601060DEE700BF67
:1093F000C49CFF1FF8B5224E34682CB32368002BA1
:109400003AD1204F1D4604E03468ECB12368002BAC
:1094100032D1A36803B1DD6020693360036825752C
:109420001B68BB4221D1037F4560022BC46020D062
:10943000FFF748FF6368002BE6D023602046FFF764
:10944000A5FF3468002CE1D1EFF3108372B60E4A09
:1094500000211068116003B962B628B18468FFF773
:1094600095FF20460028F9D1F8BD224600219847F3
:10947000E0E783689847DDE7013B2360E4E700BF4E
:10948000C49CFF1F057B0000D49CFF1F024A136889
:1094900001331360FFF7AEBFE09CFF1F704700BFB2
:1094A0000368F0B4FBB1002501249D60DC601B4C17
:1094B0001A601C44241104F144056A110326920029
:1094C0009E60174F0679174B47F8241002F160424F
:1094D00002F5614205F01F05012000FA05F5E6548A
:1094E0001560F0BC7047104C236843F40003236000
:1094F00000BF0E4B0E4DA4F58734A4F59E740126D3
:109500001E60234604609C68002CD0D01033AB4210
:109510000360F8D1002303601846E2E7008FFCBF28
:109520002C90FF1F44E400E03C80044000700340A6
:10953000407103400168A9B10B4BF0B40B441B11FF
:109540000A4E0B4F0B4D46F8237003F1440202F014
:109550001F0401235211A340002445F822308C60DF
:109560000460F0BC704700BF008FFCBF2C90FF1F51
:109570009D94000080E100E0024A034B012111604C
:109580001B6818470C7103402C90FF1F024A034BC5
:10959000012111605B6818471C7103402C90FF1F6C
:1095A000024A034B012111609B6818472C7103404C
:1095B0002C90FF1F024A034B01211160DB68184702
:1095C0003C7103402C90FF1FF8B50E4671B17AB183
:1095D0000746144600253B6816F8011B1B683846F1
:1095E0009847013C0544F6D12846F8BD0846F8BD29
:1095F0001046F8BD00B5064A036812885B6883B060
:1096000001A9ADF804200222984703B05DF804FBDD
:1096100064FE0000F0B507468BB0002A33D0012A63
:1096200008BF0A2251B3212400E0F4B2B1FBF2F5E5
:1096300002FB1511C8B2092900F1300198BFC8B268
:109640000AA988BF3730214488BFC0B201F8240C72
:10965000661E2946002DE8D133B1013CE4B20AABC5
:1096600023442D2203F8242C3B6801AA11195B68BE
:109670003846C4F1220298470BB0F0BD30228DF875
:1096800025202124E8E70368C9B21B6898470BB07E
:10969000F0BD00BF0029BABF49422D2300230A2292
:1096A000FFF7B8BF374A384913681B06FCD40B686C
:1096B00013F08003F8D172B634490A78002A5FD0DB
:1096C000334A3448F0B4344C176806682568D468C7
:1096D0000C303E44143200681268304F35442C443C
:1096E00020440244C2F34E022D4E2E482E4D2F4CE4
:1096F00042F400423A60376806682D682C4A2468B4
:109700000C303E44006812682A4F35442C442044F3
:109710000244C2F34E02284E2848294D294C42F4F7
:1097200000423A60376806682D68274A24680C3082
:109730003E4400681268254F35442C4420440244BE
:10974000C2F34E02224E2348234D244C42F40042E1
:109750003A60376806682D68214A24680C303E4418
:109760000068126835442C4420440244C2F34E027F
:109770001C4842F4004202600B7062B6F0BC7047B5
:1097800062B6704724B0034024B00B40D99CFF1F41
:1097900038B003403CB0034040B003402CB003401D
:1097A00058B003405CB0034060B0034064B0034075
:1097B0006CB0034030B0034038B00B403CB00B40BD
:1097C00040B00B4044B00B404CB00B402CB00B40B1
:1097D00058B00B405CB00B4060B00B4064B00B4025
:1097E0006CB00B4030B00B4030B42948294A2A4BAA
:1097F0002A4D6024E121047011701B78284C082B3D
:1098000030D00A2B2748284937D00C2B0CBF3522E3
:109810003D2212232A60236002600B60234B2449FF
:109820001B78244ABBB101230B601360224B2349F0
:109830001B78234A012B26D9042B0FD9082B1ED9BC
:10984000102B94BF862387230B6013601D4B0122CE
:109850001A7030BC70470B601360E7E784230B601D
:109860001360F3E700F58E200F490830012213231F
:109870002A60236002600B60D0E73922F7E7852376
:109880000B601360E2E780230B601360DEE700BF2C
:1098900000400740014007403C90FF1F08B00340D4
:1098A0000CB0034008B00B400CB00B40DC9CFF1F19
:1098B00020B0034020B00B403D90FF1F24B0034078
:1098C00024B00B40D99CFF1F0C2830B417D91023AB
:1098D000984228BF18461C46104A114D1178181A94
:1098E0008C42287018D00F4913700B7823B10E49A1
:1098F0000E4A00230B60136030BCFFF775BF0A28C7
:1099000002D90C231C46E7E7082802D90A231C4683
:10991000E2E708231C46DFE730BC70473C90FF1F9E
:10992000D89CFF1FD99CFF1F24B0034024B00B40DC
:1099300028282FD8334B2DE9F0411E5CFF2E2BD069
:10994000314B1B78002B2AD132062CD472B62F4D06
:109950002F4C2F46012326602B7062B672B6236807
:109960001B060CD43B781BB9F4E72B78002BF1D005
:1099700062B602F09BF972B623681806F5D5254B3E
:109980001B6800222A7062B6234A107843FA00F05E
:10999000BDE8F081002070470020BDE8F081FFF7AE
:1099A00081FE3206D2D572B61C4DDFF87C801C4C8D
:1099B00006F04007FFB206F03F06D8F80030DFB1EE
:1099C00023F01003C8F8003001232660134A2B70DF
:1099D00062B672B6236819060CD413781BB9ECE78B
:1099E0002B78002BE9D062B602F060F972B62368DA
:1099F0001B06F5D50B4BC3E743F01003C8F8003046
:109A0000E2E700BF68FE0000D99CFF1FDB9CFF1F40
:109A100000B0034010B00340D89CFF1FDA9CFF1F2A
:109A200000B00B4010B00B400CB00B400A4A0B4981
:109A3000136843F4805313600B7843B9084BC0227A
:109A40001A70084B80F30C0000B218807047044B6A
:109A500080221A70F5E700BF2C800440DC9CFF1FB9
:109A600021C00C4000C00C40F0B51B4B1B4E596888
:109A700018689A68DB6885B06C460FC4337899071C
:109A80001DD5174A174C1378174913F0700318BFE8
:109A90001370164A164B80271770002633200322B6
:109AA00026706D4608701A7072B6043C45F00105C8
:109AB0002046A84762B6237813F0700309D10D4BF6
:109AC000064901E0013B02D00A78D207FAD505B079
:109AD000F0BD237005B0F0BD94FE0000010002400F
:109AE00000000240040002400B0002400700024058
:109AF0000A000240410D0300B0F5006F0AD210B514
:109B0000094B1B78DB07044606D504F1A05000780A
:109B1000C0B210BD00207047FFF7A6FF04F1A050AF
:109B20000078C0B210BD00BF01000240B0F5006F68
:109B300017D238B50F4B1B78DA070D46044611D5FE
:109B400004F1A0500378AB420AD00B4A137813F00B
:109B5000700318BF1370074A05701378DB07FCD534
:109B600038BD7047FFF780FF04F1A0500378AB4287
:109B7000EBD1F5E7010002400000024008B5F6F71E
:109B80007DFDF7F7FDFF02F091F8FAE7844641EA20
:109B9000000313F003036DD1403A41D351F8043B65
:109BA00040F8043B51F8043B40F8043B51F8043BB7
:109BB00040F8043B51F8043B40F8043B51F8043BA7
:109BC00040F8043B51F8043B40F8043B51F8043B97
:109BD00040F8043B51F8043B40F8043B51F8043B87
:109BE00040F8043B51F8043B40F8043B51F8043B77
:109BF00040F8043B51F8043B40F8043B51F8043B67
:109C000040F8043B51F8043B40F8043B51F8043B56
:109C100040F8043B51F8043B40F8043B403ABDD2C5
:109C2000303211D351F8043B40F8043B51F8043B67
:109C300040F8043B51F8043B40F8043B51F8043B26
:109C400040F8043B103AEDD20C3205D351F8043BF6
:109C500040F8043B043AF9D2043208D0D2071CBFC2
:109C600011F8013B00F8013B01D30B8803806046EB
:109C7000704700BF082A13D38B078DD010F0030361
:109C80008AD0C3F10403D21ADB071CBF11F8013BD1
:109C900000F8013B80D331F8023B20F8023B7BE720
:109CA000043AD9D3013A11F8013B00F8013BF9D24B
:109CB0000B7803704B7843708B78837060467047E5
:109CC00008B5104C08E0236859050DD423681A051F
:109CD0000FD42368DB0411D423685803F3D500F0B4
:109CE0008DFE23685905F1D502F044F823681A0562
:109CF000EFD502F0D5F82368DB04EDD500F0F0FCD9
:109D0000EAE700BF3480044008B5FFF7D9FF00BF81
:109D1000014B10221A80704700200540704700BF99
:109D2000094908B50B6830B16A461844A2F580525B
:109D3000904202D20860184608BD03F063FB0C2372
:109D400003604FF0FF3008BD4090FF1FFEE700BFEB
:109D5000EFF3138070B9EFF310836BB9EFF3058263
:109D60005AB94FF48070EFF311832BB1984228BF9A
:109D7000184670474FF0FF3070470F2A01D8184639
:109D8000F1E7014BD05CEEE7F0E300E0F0B44D1EEC
:109D90002E46002400E00134B0FBF2F302FB130076
:109DA000092800F130078ABF3730F8B2C0B206F890
:109DB000010F1846002BEED10A1953704CB11078E0
:109DC00015F8016F28700133E01A834202F8016927
:109DD000F5DB0846F0BC7047704700BF10B40F4B6E
:109DE00053F8302092F880422CB1012369B182F8F7
:109DF000803010BC704703EBC0035B681A6841B940
:109E000022F002021A6010BC704782F8003110BCC8
:109E1000704742F003021A6010BC7047A4FE0000B5
:109E20001C4A02EBC00301295B6811D004291BD036
:109E300052F83000002280F8802229B1022920D077
:109E4000032922D01A6070474FF480721A6070475D
:109E500052F830004FF4A27280F880121A601A682B
:109E600022F020021A60704752F830104FF4A272AC
:109E7000012081F880021A601A6842F020021A60FC
:109E8000704740F203121A6070474FF481721A60F3
:109E9000704700BFA4FE0000212848D8F8B5042A66
:109EA00044D8DFE802F0484B4E0345004FF410263B
:109EB0002B4B03EBC0030D465C68216811F4E06195
:109EC00048D0284B284A2949C3F89C2104F1404234
:109ED0002748C3F8A411A2F59221264FC3F8A00188
:109EE0007C292548C3F8A871C3F8AC012CD9A2F588
:109EF00094237C2B2AD9A2F596237C2B28D9A2F572
:109F000098237C2B29D9A2F59A227C2A27D81B4892
:109F100072B6236823F4702343F08072C4F3840183
:109F20001643236040F82150266062B6F8BD7047A2
:109F30004FF43026BCE74FF40026B9E74FF4402633
:109F4000B6E74FF42026B3E70D48E1E70D48DFE719
:109F50000D48DDE7FFF764FFB3E70C48D8E7F8BD2D
:109F6000A4FE00000082FF1FF188FF1F9988FF1FD9
:109F7000C588FF1F6D88FF1F4188FF1F1C91FF1FB1
:109F80004490FF1F7C90FF1FCC90FF1FFC90FF1F91
:109F90001A4B03EBC00010B4426802F14043A3F532
:109FA00092217C2923D9A3F594217C290DD9A3F5ED
:109FB00096217C291FD9A3F598217C2919D9A3F5CD
:109FC0009A237C2B11D80E4C00E00E4C72B613680D
:109FD0000D4823F08773C2F3840123F4803343F0E8
:109FE0008073136044F8210062B610BC7047074CC0
:109FF000ECE7074CEAE7074CE8E700BFA4FE0000E7
:10A000001C91FF1F7C90FF1FD99D00004490FF1FF3
:10A01000FC90FF1FCC90FF1F30B4054B054D064C44
:10A02000002210211A602A602060196030BC70473D
:10A0300014D0034004D0034000D00340282838B592
:10A040002ED0002904464FDD5F4B1B78012505FA11
:10A0500003F28A4202D8212837D938BD0338C2B268
:10A06000012A3AD9202C4AD0192C48D0574A1268D4
:10A0700002FB011222FA03F31D2800F29B80DFE8A5
:10A0800000F0928B847D9999766F99999999999915
:10A0900099999968615A53994C99999999999945BF
:10A0A000494B1B780B2B08D90C2B1CBF0C3B1941BF
:10A0B0000846BDE83840FFF7B9BCC3F10C0399402E
:10A0C0000846BDE83840FFF7B1BC2946FFF786FED9
:10A0D0002946BDE83840FFF7A3BE3D4A126802FB9F
:10A0E000011222FA03F3C7E72128B6D80021FFF7AF
:10A0F00075FE20460121BDE83840FFF791BE354A84
:10A10000126802FB011222FA03F3B5E73249334A1F
:10A110000B604FF45173136038BD3149314A0B6005
:10A120004FF45173136038BD2F49304A0B6040F231
:10A130004443136038BD2E492E4A0B6040F244431D
:10A14000136038BD2C492D4A0B6040F24443136024
:10A1500038BD2B492B4A0B6040F24443136038BD95
:10A1600029492A4A0B6040F24443136038BD28490C
:10A17000284A0B6040F24443136038BD2649274A01
:10A180000B6040F24443136038BD2549254A0B60FB
:10A1900040F24443136038BD2349244A0B604FF416
:10A1A0005173136038BD2249224A0B604FF451733A
:10A1B000136038BD212C3FF650AF7F29D4BF00215A
:10A1C0000121204693E700BF2491FF1F0880034030
:10A1D0000890034008800B4010800B4048A00440CA
:10A1E00018800B404CA004401880034008B0044085
:10A1F0001080034004B004404080034018C0044075
:10A200003880034014C004402880034010B004404C
:10A21000208003400CB004403080034010C0044054
:10A22000488003401CC00440189003403490044010
:10A23000109003403090044038B1102828BF1020FF
:10A24000044AC3B2107813707047024A0123107891
:10A25000137070472491FF1F2DE9F8430E46804686
:10A260003249334D304603F053F847F612230028A5
:10A270001ABF1D464FF002094FF00109002425FACC
:10A2800004F002F04FFE4FF05E51074602F0A2FECE
:10A290000146304603F050F830B90134072CEED1B6
:10A2A000E80902F03FFE07463146384602F046FF15
:10A2B0004FF07C5102F084FD03F078F84FF6FF7206
:10A2C0009042A8F1030328BF1046012B29D9B8F109
:10A2D000170F17D8174B23FA08F303F0010383F085
:10A2E000010223B9B8F1190F0FD0BDE8F883124B62
:10A2F000124D13491A6044EAC9042A6008601C60C0
:10A30000BDE8F883B8F1200FECD10E4B0E4D0F498C
:10A31000002244EAC9041A602A6008601C60BDE893
:10A32000F8830B4B0B4D0C49F2E700BF001BB74005
:10A33000006CDC026006F0000080034004800340F3
:10A340000880034000800B4004800B4008800B40D5
:10A35000009003400490034008900340212801D856
:10A36000FFF73CBD704700BF212806D8044B53F8C7
:10A37000303093F80002C0B270470020704700BF31
:10A38000A4FE0000212801D8FFF74ABD704700BF96
:10A3900072B60C490C4B0D4A1B680868126862B60D
:10A3A000520102D5322B88BF01300949C3F5BB33B6
:10A3B0004FF47A72FF33A1FB031302FB00F000EBB2
:10A3C00093107047E09CFF1F18E000E004ED00E0F0
:10A3D000ABAAAAAA2DE9F843054672B6204F214B35
:10A3E000214A1B683C68126862B6520102D5322BC2
:10A3F00088BF013495B3C3F5BB331C4EDFF86490BE
:10A40000DFF86480FF334FF47A72A6FB031302FB7C
:10A4100004F404EB931472B6D9F800103A68D8F833
:10A4200000E062B6C1F5BB33FF33A6FB03031EF0A9
:10A43000806FC4EB93134FF47A7002D0322988BF37
:10A44000013200FB0233B3F57A7F04D3013D05D01E
:10A4500004F57A74DFE701F029FCDCE7BDE8F88356
:10A46000E09CFF1F18E000E004ED00E0ABAAAAAA00
:10A47000F8B52D4B2D49DFF8D0E0DFF8D0C02C4ED9
:10A480002C4D2D4C2D4A2E4F4FF4000018604FF0EC
:10A49000807018604FF0007018604FF08060186096
:10A4A0004FF0006018600020086028234BF6FF7111
:10A4B000CCF80010CEF80030336013602B602360BE
:10A4C0003B60B3629362092245F8242CC4F8D80F8C
:10A4D00005F57F65C7F8D41F07F5FF2707F5FA676D
:10A4E000C6F8F83F2B6006F5FF26C4F8D42F05F513
:10A4F000FD2504F5FF24386006F2F476114831603A
:10A5000005F5FF6504F5FD642B6023600260FFF72D
:10A510006BF91920FFF75EFF00F0B6FF40F2131051
:10A52000BDE8F840FFF756BF08E100E004800340B3
:10A5300014800340248003402C8003401C8003408F
:10A540003480034000800B400C80034008800340AF
:10A550002DE9F84F214B1B6807460BB101221A70F9
:10A56000DFF888901E4D99F80040DFF884801D4E7A
:10A570000134272C8ABF4FF0000A5FFA84FA544650
:10A58000AB462B78A34216D1FFF7E2FB40281FDC35
:10A5900033791B06F5D59BF800300133272B86BF96
:10A5A00000221346DAB218F80330DBB2F3712A70D6
:10A5B0002B78A342E8D00C490A4BFFB208F804708C
:10A5C0000120AC22087089F800A0DA70BDE8F88F8D
:10A5D000FF28D6DD01F06AFBD3E700BF589DFF1FBF
:10A5E000559DFF1F00C00640549DFF1F5C9DFF1F2F
:10A5F000EC9CFF1F1C4BDFF894C01A681B49F0B598
:10A6000042F480521A4D1A60DFF884E0194F1A4E56
:10A610001A4C00238CF800304FF451722B701F2815
:10A6200040F213358EF800303B70337025600A60BD
:10A6300012D819460124124A124D11701248547052
:10A6400000212C27402693724FF40034917011742E
:10A65000D7702E700460F0BDC0F34431C0F34714CE
:10A6600000F01F03E7E700BF348004400CC0044043
:10A67000E99CFF1F559DFF1F549DFF1F08C004400C
:10A6800000C0064031E400E004E100E0E89CFF1F68
:10A690005C9DFF1F034B1B68DB0401D5FFF758BF10
:10A6A000704700BF3480044010B5044C237823B1B8
:10A6B00001F0FCFA2378002BFAD110BD549DFF1F46
:10A6C000054A064B10781B78C0B2DBB2984238BFFF
:10A6D0004030C01A704700BFE89CFF1FE99CFF1F75
:10A6E00030B42B4B1A7994061FD52A48DA790378AF
:10A6F000294901333F2B0978C8BF00238B42D2B2CE
:10A7000003D0264CD9B2E2540170254A116861B1D8
:10A71000244A1278D2B2934236BFC2F140029B1A49
:10A720009B18272BC4BF01230B70194AD378DBB2C7
:10A73000180611D45A060DD5154B1B795B0609D5A1
:10A74000194B1A491B6800220A7003B11A70104B8A
:10A750002C22DA7030BC704711790906EAD5144909
:10A7600010480C780178C9B28C420DD04A1C272AB7
:10A7700084BF00210A460F4D054C98BFD1B2AA5C98
:10A78000D2B2E2710170D5E76C21D170D2E700BF7F
:10A7900000C00640E89CFF1FE99CFF1F149DFF1F9F
:10A7A000E49CFF1F559DFF1F589DFF1F549DFF1FD9
:10A7B0005C9DFF1FEC9CFF1F21282FD8184B195CB4
:10A7C000FF292BD0174B184ADFF870C003EBC000ED
:10A7D000F0B54368DFF868E0144F154D154E0024BE
:10A7E0001C60DEF80030012043F020038840CEF8E2
:10A7F000003014604FF4A07338602E60C2F800C0BF
:10A80000013BFDD113689B05FCD42023013BFDD106
:10A81000094B09B233F8110080B2F0BD0020704737
:10A82000B4FF0000A4FE00000050044008500440A3
:10A8300004500440000002030051044080014A001B
:10A8400038800440431E032B14D872B60A4951F8CD
:10A85000230068B170B4094C058834F813204668A9
:10A8600041F82360521B24F8132062B670BC704775
:10A8700062B6704700207047B89DFF1FFC9FFF1F06
:10A88000013803280BD872B6074B53F8203043B178
:10A8900000205B680130002BFBD162B670470020BE
:10A8A00070471846F9E700BF0C9EFF1F30B472B620
:10A8B0002B4A13781D0706D52A4B196A002936D072
:10A8C000996A002941D053781C0706D5254B196C8D
:10A8D00000293ED0996C002939D09378190705D505
:10A8E000204B196E002936D0996E89B1D3781B0799
:10A8F00007D51C4BD3F880207AB3D3F888201121D8
:10A900003AB162B6184B00221A7030BC00F04ABE51
:10A910000D21154C154D227843F8315003EBC1033E
:10A920000830013A5860227062B630BC7047042289
:10A930000D4C0F4D217843F8325003EBC203083021
:10A940004A1E5860227062B6EFE70521E1E709214F
:10A95000DFE70822ECE70C22EAE71022E8E700BF75
:10A96000D8FF00000080FF1F359EFF1FC800400079
:10A9700088004000431E032B1DD81B4A400140F0B5
:10A98000100030B4104472B6184CE25C032A1BD895
:10A99000DFE802F00212151703220D88E25410F0CE
:10A9A000080F14BFC823882343EA05430831036016
:10A9B000416062B630BC704708300222EDE70522E4
:10A9C000EBE708300422E8E7094A52F8230038B1DF
:10A9D000084A52F82300416042F8231062B6E9E7C2
:10A9E00042F82310034AF7E70080FF1F449EFF1F31
:10A9F0000C9EFF1F1C9EFF1F00BE70472DE9F04FED
:10AA0000DFF818B3DFF818A387B044E0AD4F4FEA82
:10AA1000930807EBC809013ED9F8042003F00803A6
:10AA2000F6B2A2F1080003F0FF04002B40F0018110
:10AA300057F838301B0C99B222F8081C002B00F094
:10AA4000EF80A14B22F8064C42F8044C53F8262024
:10AA5000002A00F0CF819D4D55F8263058609C4C5F
:10AA600045F8260034F81630194424F8161000F082
:10AA700079FD002800F0C281964A974B19F0080F23
:10AA800000F1080018BF1346C9F8040047F8383031
:10AA900008238BF800309BF80040E4B265071CD512
:10AAA0008E4B1B78B3B18E490A7802F0FF0322B1B6
:10AAB000013BDBB20B7003B900BE8A490A7802F091
:10AAC000FF032AB1013BDBB20B70002B00F0688161
:10AAD00000F066FE04238BF8003004F0080303F056
:10AAE000FF02002B00F0C9809AF80030DBB21E098B
:10AAF0008CD19A08DFF8CC9159F8321009EBC200DA
:10AB0000C1F38301013940680C2900F28580DFE838
:10AB100001F07A7A83838383838346838383070068
:10AB20000168714D4068714F714E6860296088B24C
:10AB300040F281610024674B49F832304FF0010E3A
:10AB400088423C60C9F81040C9F8184086F800E017
:10AB50005C4A00F2E780B0F5D06F80F01B82B0F560
:10AB6000817F00F0D98100F26981802800F02A827B
:10AB7000822840F0D781A98801F07F01042900F2E2
:10AB8000D1815C485C4A8900084414705470017893
:10AB90008C0740F1608382F800E0022173E1534F9B
:10ABA0003A682AB3554B524E55481988347805787F
:10ABB00040298E4645F0020828BF4FF0400E002C79
:10ABC00084F001043470CEEB01010CBF8824C8244A
:10ABD00009EBC80689B285F0010544EA0E447260AB
:10ABE000198049F8384072440570002965D03A60F0
:10ABF0003D4B1A88B2F5A06F0ED100219A7859709A
:10AC0000404B1A7008E038493F4C0D68A54200F0EF
:10AC10009880304949F832103C4A0123137037E7D5
:10AC20002C4A2D4B19F0080F18BF134647F838303F
:10AC30002EE700F0B7FC364A364952F82630002B92
:10AC400000F0E38058688C5D42F8260003F10802AA
:10AC5000C9F80420032C05D8DFE804F02C022926CB
:10AC600002228A551A8819F0080F0CBF8823C823BE
:10AC700043EA024347F838300AE7E00700F19380DF
:10AC8000210600F1D180A20706D5234A2349137873
:10AC90000220DBB213700870E30602D51F4B1022AE
:10ACA0001A7007B0BDE8F08F04228A55DAE7052252
:10ACB0008A55D7E703228A55D4E7BEF1400F18BF63
:10ACC000002294E70080FF1FB89DFF1F649DFF1FB7
:10ACD000FC9FFF1FC800400088004000409EFF1FEF
:10ACE000C99DFF1FB49EFF1F2C9EFF1F609DFF1F6D
:10ACF000C89DFF1FC0200740389EFF1F749DFF1F87
:10AD0000349EFF1F9820074021090003942007402C
:10AD10000C9EFF1F449EFF1F882007408020074095
:10AD200090200740B0F5106F00F07C8140F2A380C6
:10AD300040F62112904240F07B82A54A0123137015
:10AD40006AE74C68A3498C427FF463AF0178A92974
:10AD50007FF45FAF417845297FF45BAF8178C229EA
:10AD60007FF457AFC1786B297FF453AF9A489B4E5D
:10AD70000178347881F00105002C41F00201057062
:10AD80000CBF8820C82084F0010449F8310009EB89
:10AD9000C10193483470002505244D60047038E7E4
:10ADA00000F064FF94E68F4B89488B491A614FF09D
:10ADB000020E80F800E08C4F0A708C49196099608F
:10ADC0008B4E8C4D8C4C9A610D213970FF21317066
:10ADD000DFF84CE229702270884D894A8EF8001005
:10ADE0009F27012406F8047C5D600470DA6007B0D8
:10ADF000BDE8F08F43F82600824D30E6824A47F8DE
:10AE0000380013780133137042E68B5D032B00F298
:10AE1000BA8001A252F823F091AA000091AA000082
:10AE200071AE00006BAE00006F49724B80220D20A6
:10AE300008701A70A2077FF52FAF26E740F20232A2
:10AE4000904240F0ED81AA8802F07F02042A69D87E
:10AE50006D88002D66D16449CDF804E0920011445C
:10AE60000A7842F002020A70C1E101238B550FE615
:10AE700000238B550CE6B0F5086F53D16349644A43
:10AE8000097811707146ED888D4280F0E882524851
:10AE90000478402DAE4644F0020C28BF4FF0400E1F
:10AEA00002EB0E0309EBCC01029301234A604FEA47
:10AEB0000E48CEEB050101930025C82242EA0803A3
:10AEC00084F0010249F83C3035700270DFF814C19B
:10AED000424BDFF8048149BBBEF1400F7FF42DAF38
:10AEE00042F0020C09EBCC03029ADFF8F8E05A605A
:10AEF0008DBB0D0445F088059DF804304EF83C509C
:10AF00000A4433700470134640297FF416AF0021C1
:10AF1000404A3B60118010E7AA8802F07F02042AB1
:10AF200040F28B81304A0F23137006E74029D7D9AE
:10AF300042F002020CEBC200029E4660BDB19DF8D9
:10AF4000045035481D703346403988F8004040337E
:10AF50004CF83200DCE79DF8043033700D04029B9E
:10AF6000047045F0C8050B444EF83C50CCE79DF802
:10AF700004501D70029B1D4888F800404039403342
:10AF80004CF83200C4E719F0080F0CBF022303236A
:10AF90008B557DE521494A68002AC3D06C88B5F8F5
:10AFA00004E003E00C314A68002ABBD00B88A342BE
:10AFB000F8D14B887345F5D1240A032C0CBF1178C6
:10AFC000098960E7124A0221147054705BE700BFE0
:10AFD0009420074001000400349EFF1FC89DFF1FFE
:10AFE000C99DFF1F0080FF1FC02007408800400050
:10AFF000882007408020074098200740789DFF1F49
:10B00000CC9DFF1F649DFF1F359EFF1F409EFF1FAD
:10B01000389EFF1F749DFF1FC8004000DCFF00002A
:10B020008C200740B248116AAC7804700C0600F11D
:10B030009881D9F82820AF49100600F1DB81D9F8B2
:10B040003020AC49120600F1D081D9F83820A94946
:10B05000130600F1C581D9F84020A649150600F174
:10B06000BA81D9F84820A349140600F1AF81D9F874
:10B070005020A049100600F1A481D9F858209D491C
:10B08000120600F19981D9F860209A49130600F15F
:10B090008E81D9F868209749150600F18381D9F887
:10B0A00070209449140600F17881D9F878209149EC
:10B0B000100600F16D81D9F880208E49120600F14A
:10B0C0006181D9F888208B49130600F15581D9F8A0
:10B0D00090208849150600F14981D9F898208549C2
:10B0E000140600F1FF808448844A85490190854810
:10B0F000854D864C049700230596029580460F46A1
:10B1000016461D460394306828B1446800F04AFA98
:10B110002046002CF9D100233360029B38681A4680
:10B12000002342F8253028B1446800F03BFA20465D
:10B13000002CF9D100223A60019A98F800301146AB
:10B14000002241F8042B039A0191023B4FF00001C9
:10B1500022F81510032B07D8DFE803F05D025D022B
:10B160004FF0010388F800300135042D06F1040684
:10B1700007F1040708F10108C5D1654C654D227837
:10B18000654B049F059E0021100729701A7000F17D
:10B190009280624962780A700021C9F83010C9F8BB
:10B1A00038101107DFF84C816ED4A2785C49DFF8C3
:10B1B00044810A7000211207C9F85010C9F85810CC
:10B1C0004BD4E27857494B4C0A7013074FF00001FB
:10B1D000C9F87010C9F8781000F1AE803378019387
:10B1E000002283F00105C9F89020C9F898200021B9
:10B1F000029188468E460A464B48047844F0020C79
:10B2000009EBCC030393019B002B039B5A600CBFFB
:10B210008822C82252E64FF0000388F80030A3E7E6
:10B22000B0F5A06F7FF47EAE012300250193DEE729
:10B2300040F621229042F7D074E66D88002D7FF40D
:10B2400071AE3A49CDF804E0920011440A7822F038
:10B2500002020A70CBE7022115E600F083F900280C
:10B2600000F0EB800830324AC8F86400C8F860206B
:10B2700000F078F9002800F0DA8008302D4AC9F88B
:10B280006C00C9F868209CE700F06CF9002800F019
:10B29000E0800830264AC8F84400C8F8402000F092
:10B2A00061F9002800F0CF800830224AC9F84C002C
:10B2B000C9F8482079E700F055F9002800F0A5808A
:10B2C00008301B4AC9F82400C9F8202000F04AF9C8
:10B2D000002800F094800830164AC9F82C00C9F8FC
:10B2E000282056E7D1F89C00083800F05BF9FAE610
:10B2F000409EFF1F0080FF1F1C9EFF1FB89DFF1F69
:10B300000C9EFF1F449EFF1F649DFF1FFC9FFF1F9D
:10B31000D8FF0000359EFF1FC4200740C82007400B
:10B32000CC200740D0200740349EFF1FC02007409C
:10B3300088004000C800400000F014F9002870D0D8
:10B3400008304F4AC4F88400C4F8802000F00AF99D
:10B35000002860D008304B4AC9F88C00C9F8882012
:10B360003CE7506A083800F01DF962E6D1F8940015
:10B37000083800F017F9B0E6D1F88C00083800F072
:10B3800011F9A4E6D1F88400083800F00BF998E62A
:10B39000C86F083800F006F98DE6486F083800F0ED
:10B3A00001F982E6C86E083800F0FCF877E6486ECE
:10B3B000083800F0F7F86CE6C86D083800F0F2F8CD
:10B3C00061E6486D083800F0EDF856E6C86C0838BC
:10B3D00000F0E8F84BE6486C083800F0E3F840E687
:10B3E000C86B083800F0DEF835E6486B083800F026
:10B3F000D9F82AE6C86A083800F0D4F81FE62A7897
:10B40000C9F8280001322A70C3E62A78C9F820005A
:10B4100001322A705AE72A78C9F8880001322A7066
:10B42000DCE62A78C4F8800001322A708EE72A7898
:10B43000C9F8680001322A70C3E62A78C8F86000AB
:10B4400001322A7014E72A78C9F8480001322A70BC
:10B45000ABE62A78C8F8400001322A701FE740297D
:10B460008E4628BF4FF0400E02EB0E0302930123DD
:10B47000CEEB01014FEA0E4800250193BCE600BF68
:10B4800088004000C8004000F8B500F08FFD294B4F
:10B4900029482A4C2A4F2B4DDFF8BCC0DFF8BCE00E
:10B4A000294E00221A605A609A60DA601A615A6165
:10B4B0009A61DA611A625A629A62DA621A635A63AC
:10B4C0009A63DA631A645A649A64DA641A655A658C
:10B4D0009A65DA651A665A669A66DA661A675A676C
:10B4E0009A67DA67C3F880200168C3F8842041F4C2
:10B4F00080210160C3F307212170C3F30740134982
:10B5000038701B0E2B70FF238CF80030104D8EF816
:10B51000003010480B700123337084F864207026CB
:10B520004FF40074102207F82C3C2E70046081F850
:10B53000F820F8BD0080FF1F348004409C200740A5
:10B54000B0200740B4200740942007401020074057
:10B5500049E400E008E100E080200740882007403F
:10B56000704700BF72B60D480268B2FA82F30F2B23
:10B5700010DC4FF00041D94022EA0102026062B6BD
:10B58000074803EBC303DB00C2180021C15010467B
:10B590005160704762B60020704700BF2891FF1FBE
:10B5A000BC83FF1F0D4B0E4AC31AA2FB03231B09CA
:10B5B0000F2B0CD80B4A127852B972B60A484FF0CA
:10B5C0000041026821FA03F31A43026062B6704731
:10B5D000064A1278002AF0D0FFF768B9BC83FF1F33
:10B5E000398EE338359EFF1F2891FF1F409EFF1FB5
:10B5F00038B50E4B0E4C1B68218805468BB1B1F552
:10B60000917F05D20B4A4B1C55549BB2238038BD09
:10B610000022084898470021064A555401232380F8
:10B6200038BDB1F5917FEDD338BD00BF6C9EFF1FD3
:10B6300006A0FF1F0CA0FF1F2DE9F843214E224F4B
:10B640003168012380463B70B1B1204D4B8801EB3E
:10B650008302013300240F2BC2F808802C7004D819
:10B660004B8000233B70BDE8F88340230B80032010
:10B67000FFF780F93460F4E7DFF8549099F8003070
:10B68000002BF0D0114D45F6215408E0013C12D0BA
:10B690002B7883B900F00AFB99F800307BB10320C6
:10B6A000FFF7EEF80528F1D8FFF75CFF01463060A0
:10B6B0000028EBD0CAE701232B70BDE8F883BDE872
:10B6C000F88300BF889EFF1F5C9EFF1F8C9EFF1F9C
:10B6D000409EFF1F1201F8B5D5B2A1B3012943D096
:10B6E0004378044600781B0643EA004040F470406B
:10B6F00045F004068F1E3043FFF79EFF022F04F132
:10B70000020314D9053414F8023C14F8032C14F87D
:10B71000010C1B0443EA0223334343EA0060033F66
:10B72000FFF78AFF022F234604F10304EBD8022F10
:10B7300023D0012F0DD045F4774040F00500BDE83F
:10B74000F840FFF779BF14482843BDE8F840FFF7F9
:10B7500073BF187845F4770545F0060545EA0020E3
:10B76000BDE8F840FFF768BF03780C4845EA034599
:10B770002843BDE8F840FFF75FBF1A78587845F0D6
:10B78000774545F0070545EA022545EA0040BDE852
:10B79000F840FFF751BF00BF06F0F70007F000F7D1
:10B7A00038B5084B1C7824B9074D296809B14B8876
:10B7B00003B938BD9B000B800320FFF7DBF82C603A
:10B7C00038BD00BF5C9EFF1F889EFF1F2DE9F04122
:10B7D000AD4E33680746002B00F092801D885A88D2
:10B7E000910803EB81010432AA428C6842D25A804C
:10B7F00004F00F064FEA1428A449A6F1080208F045
:10B800000F00C4F30313062A00F101050B701AD9C7
:10B81000B31E012B5FFA88F04ED9052E48D0042EB6
:10B8200000F0A481731F022B7FD90F2E0ED1F728B1
:10B8300042D8F02802D0964B1B883BB1FFF7D8FEC8
:10B840000020BDE8F08127B1BD4202D00020BDE854
:10B85000F081082EC4F3033300F08780092E11D045
:10B860000A2E40F094800A2BF0D18A4B8A4A1B683A
:10B87000A02181E01846FFF795FE0420FEF7E2FFC5
:10B880003060B5E7092BE1D1270E00F07B81834BB7
:10B89000814A1B689021C4F307461170EDB2FCB2D7
:10B8A000002B00F09D80224631462846984797E0BD
:10B8B000F02843D9F72841D0F1380E28C6D801A383
:10B8C00053F820F07BBA00005FBA00004DBA0000C8
:10B8D0004DB800004DB800003FBA00004DB8000060
:10B8E0001FBB00004DB80000E9BA000003BB000018
:10B8F00027BA00004DB800000FBA0000F3B90000ED
:10B90000674B1B78002BA1D00420FEF79BFF03465A
:10B91000306000289AD00588002D7FF460AFFFF7D3
:10B9200041FE35602846BDE8F081FFF761FEC4F3B3
:10B930000740FFF75DFE072E02D1200EFFF758FEED
:10B94000534B584A198858481468584D524A017048
:10B9500000270E0AF0201F802E7010700CB30122F9
:10B960005348A0470120BDE8F081082B7FF46EAF5B
:10B97000504B494A1B688021C4F307461170EDB251
:10B98000240E6BB3284622463146984728E00B2EFA
:10B9900011D10B2B7FF45AAF474B3F4A1B68B021A4
:10B9A000EAE7464B1B68002B00F0FB8040489847B5
:10B9B0000120BDE8F0810C2E40F000810C2B7FF4BB
:10B9C00045AF3F4B344A1B68C0211170EDB2C4F340
:10B9D0000746002B00F0C88028463146240E9847C1
:10B9E0003849314A314B0D7016701C700120BDE88A
:10B9F000F081354B1B68002B00F0D6809847C4F3CC
:10BA00000746254BEDB2240E83F80080E8E72F4B64
:10BA10001B68002BF2D12E4B1B68A3B1FE20984768
:10BA2000C4F30746EDE72B4B1B68002BE6D1284BF0
:10BA30001B6843B1FC209847C4F30746E1E7264B57
:10BA40001B68002BDAD1C4F30746DAE7234B1B68E7
:10BA5000C4F30746002BD4D030469847D1E7204B9B
:10BA60001A68002AEFD0260C630C06F07F0003F45E
:10BA70007E531843F6B29047C3E71A4B1B68C4F3D2
:10BA80000746002BE8D1BCE7949EFF1F0AA0FF1FCA
:10BA900006A0FF1F709EFF1F04A0FF1FA49EFF1F94
:10BAA000409EFF1F6C9EFF1F08A0FF1F09A0FF1FE5
:10BAB0000CA0FF1F9C9EFF1FA09EFF1F849EFF1FC8
:10BAC000609EFF1F0BA0FF1F4C9EFF1F509EFF1F7D
:10BAD000549EFF1F909EFF1F809EFF1F989EFF1F7A
:10BAE000689EFF1F7C9EFF1F3F4B1B68002B85D16C
:10BAF0003E4B1B68002BA6D0FA209847C4F307469C
:10BB00007FE73B4B1B68002B7FF478AF374B1B68FC
:10BB1000002B98D0FB209847C4F3074671E7354BBC
:10BB20001B68002B7FF46AAF304B1B68002B8AD058
:10BB3000F8209847C4F3074663E70E2B7FF486AEE0
:10BB40002D4A2E4B1268E0211970002A47D0260C8E
:10BB5000610C06F07F0301F47E511943EDB2A1F5AB
:10BB6000005128469047F6B2240E39E7FFF740FD12
:10BB7000C4F30740FFF73CFD200EFFF739FD00201E
:10BB8000BDE8F0811E4B1D4A1B6880211170EDB28B
:10BB9000C4F3074683B1314628463A4698473C46A7
:10BBA0001EE70120BDE8F081104B1B68002B3FF41D
:10BBB0004AAFFF20984746E71C4611E70D2EBCD13F
:10BBC0000D2B7FF443AE0F4B0C4A1B68D021117034
:10BBD000EDB2C4F30746002B7FF4FEAEC4E7C4F316
:10BBE0000746EDB2240EFBE6789EFF1F549EFF1F12
:10BBF000589EFF1F489EFF1F649EFF1F04A0FF1F4B
:10BC00009C9EFF1F749EFF1F38B5164D2868E0B13B
:10BC100001884488A14213DD03191B7A83B104F122
:10BC20000803C2180C1B002302E012F8011F21B107
:10BC30000133A342F9D1204638BD1C46204638BD09
:10BC4000FFF7B0FC0020286038BD074B1B780BB90C
:10BC5000002038BD0220FEF7F5FD28600028D7D16E
:10BC6000F6E700BFB09EFF1F409EFF1F0D4B1B78E5
:10BC7000BBB910B50C4C216803F0FF024B883F2B79
:10BC800007DC07330B4401F1470003F8012F83421F
:10BC9000FBD140230B800120FEF76CFE00232360C4
:10BCA00010BD7047A89EFF1FAC9EFF1F38B5224CE9
:10BCB000237803B138BD01232370FFF7A5FF70BBC4
:10BCC00000F048F840BB00F0DBF810BBFEF7F8FCD2
:10BCD000E0B900232370EFF30583002BEAD1EFF3E3
:10BCE000108172B6154B1868E0B1154C2278CAB9AC
:10BCF00045691D6001232370C5B1AA6101B962B60F
:10BD000000254577836898472570D3E700F020F831
:10BD1000DFE700F01BF8D9E700F016F8D3E7FFF7EC
:10BD20001FFCCDE70029C5D162B638BD054B1D60AB
:10BD30000029E5D1E3E700BFB59EFF1FCC9CFF1FA4
:10BD4000D09CFF1FC89CFF1F704700BF704700BFFB
:10BD5000704700BF054A064B10781B78C0B2DBB2B3
:10BD6000984238BF4030C01A704700BFBC9EFF1FCA
:10BD7000BD9EFF1FF0B4384B1A7912F0300F2CD053
:10BD800072B6997D01F0FF0200293DD062B6334FB3
:10BD9000334938780D78334E1C46C0B2EDB2431C9F
:10BDA000402BE17928BF0023AB4202F1FF32C9B238
:10BDB0001CBFF154184612F0FF02F0D12A4B1B6849
:10BDC000C2B23A704BB1A84236BFC5F14005401B24
:10BDD00040192728C4BF01221A701F49CA78D2B25D
:10BDE000150616D452060DD51B4B1B795B0609D5DB
:10BDF0001E4B1F491B6800220A7003B11A70164BB4
:10BE00003C22DA70F0BC70474022D9795A7462B68D
:10BE1000E3E70B791C06E5D5164B174E1C783378F3
:10BE2000E4B2DBB29C420ED0144D01E0A3420AD032
:10BE30000133402B28BF00230879E85CC0B2C871E9
:10BE4000087D0728F2D9DBB2034933700B79180655
:10BE500044BF7C23CB70C5E700A00640BC9EFF1FFB
:10BE6000BD9EFF1F009FFF1FB89EFF1F449FFF1F27
:10BE7000409FFF1F489FFF1F419FFF1FC09EFF1F46
:10BE8000054A064B10781B78C0B2DBB2984238BF27
:10BE90004030C01A704700BFBC9FFF1F519FFF1F5B
:10BEA000F0B4384B1A7912F0300F2CD072B6997D5D
:10BEB00001F0FF0200293DD062B6334F3349387894
:10BEC0000D78334E1C46C0B2EDB2431C402BE179D5
:10BED00028BF0023AB4202F1FF32C9B21CBFF154AC
:10BEE000184612F0FF02F0D12A4B1B68C2B23A701A
:10BEF0004BB1A84236BFC5F14005401B4019272869
:10BF0000C4BF01221A701F49CA78D2B2150616D4CE
:10BF100052060DD51B4B1B795B0609D51E4B1F49DD
:10BF20001B6800220A7003B11A70164B3C22DA70AB
:10BF3000F0BC70474022D9795A7462B6E3E70B79B6
:10BF40001C06E5D5164B174E1C783378E4B2DBB2ED
:10BF50009C420ED0144D01E0A3420AD00133282B9D
:10BF600028BF00230879E85CC0B2C871087D0728A3
:10BF7000F2D9DBB2034933700B79180644BF7C2336
:10BF8000CB70C5E700B00640BC9FFF1F519FFF1F4D
:10BF90007C9FFF1F4C9FFF1FC09FFF1F509FFF1FD5
:10BFA000C49FFF1FBD9FFF1F549FFF1F70B584B02C
:10BFB00072B6194B194D1A48702241260F24802160
:10BFC0001A702E701A460470197013781B06FCD56F
:10BFD000144B186862B6144B144C984298BF00EB8F
:10BFE000800001A998BF40000A22FDF7CFFE01A9F9
:10BFF0002046002311F8012B01333AB10A2B20F817
:10C00000022FF7D11623237004B070BD5B00DBB2A2
:10C01000237004B070BD00BF000002400700024062
:10C0200006000240080002407F969800F491FF1F2E
:10C030002DE9F043DFF8EC808BB006460F4600F0A8
:10C0400073F898F90030013304460D4637D0304676
:10C05000394600F0DFF9002831D02BA3D3E90023C3
:10C060003046394600F026FE814668BB28A3D3E956
:10C0700000233046394600F0FFFD00B398F9003048
:10C08000254ACDF82090042400200021022BCDE980
:10C090000467CDE9026700940192CDE906012CD036
:10C0A000684600F0BDF940B3089B1BB101F0AAF946
:10C0B000089B0360DDE906010BB0BDE8F083204674
:10C0C00029460BB0BDE8F083134A98F9003001927D
:10C0D00003210022CDE90467CDE9026700910892AF
:10C0E0002BB90E4B4FF06042CDE90623D8E70C493F
:10C0F0000020022BCDE90601D2D101F083F92223E1
:10C100000360D1E7AFF30080EF39FAFE422E86409C
:10C1100051302DD5104987C048000100FFFFEF477F
:10C120000000F07F0A92FF1F2DE9F04FB04F21F081
:10C130000042BA4283B00C464FEAD17605460DD98B
:10C14000AC4FBA4225D9C1F31303034340F0EF804B
:10C150000EB10020014603B0BDE8F08FA64B9A4215
:10C1600000F2CC80A54B9A4200F2DE808AA3D3E98C
:10C17000002300F05DF90022A14B00F09BFD002898
:10C1800000F005812846214600229D4B00F050F921
:10C19000E1E783A3D3E9002300F08CFD002840F001
:10C1A000CB802846214680A3D3E9002300F064FD1C
:10C1B0000028CED1934B284603EBC60821467CA32A
:10C1C000D3E9002300F0E6FAD8E9002300F030F9C3
:10C1D00000F07AFD804600F077FA77A3D3E90023D8
:10C1E00006460F4600F0D6FA02460B462846214680
:10C1F00000F01CF972A3D3E90023CDE90001304619
:10C20000394600F0C7FA82468B4652465B46DDE966
:10C21000000100F00BF905460C462A462346284645
:10C22000214600F0B7FA68A3D3E9002306460F467B
:10C2300000F0B0FA66A3D3E9002300F0F7F8324625
:10C240003B4600F0A7FA64A3D3E9002300F0F0F81E
:10C2500032463B4600F09EFA61A3D3E9002300F08A
:10C26000E5F832463B4600F095FA5FA3D3E9002398
:10C2700000F0DEF832463B4600F08CFA02460B46F0
:10C280002846214600F0D2F806460F4628462146A9
:10C2900032463B46B8F1000F56D000F07BFA3246EA
:10C2A00004460D463B4600204FF0804100F0BEF8AA
:10C2B00002460B462046294600F096FB02460B46F6
:10C2C0005046594600F0B2F8DDE9002300F0AEF820
:10C2D0000B4602464A49002000F0A8F86FF47F732D
:10C2E00098454FDA08F57A7801EB085100224FF0B3
:10C2F000B87300F04FFA03B0BDE8F08F424B9A429A
:10C300003FF658AF414BF4002344D3E9002300F03B
:10C310008DF83F4BC6F101081C44CDE90001D4E97A
:10C3200000ABC6EB080870E74FF0000875E702465F
:10C330000B4600F07DF80EE717A3D3E90023104663
:10C34000194600F027FA06E700F024FA002280469A
:10C3500089464FF080433046394600F067F8024680
:10C360000B464046494600F03FFB2A46234600F074
:10C370005DF802460B460020214900F057F803B053
:10C38000BDE8F08F01EB085103B0BDE8F08F8046A7
:10C3900043E700BFAFF300809C7500883CE4377E24
:10C3A000EF39FAFE422E864051302DD5104987C014
:10C3B000FE822B654715F73F0000E0FE422EE63F68
:10C3C000763C7935EF39EA3DD0A4BE726937663ED6
:10C3D000F16BD2C541BDBB3E2CDE25AF6A56113F85
:10C3E00093BDBE166CC1663F3E5555555555C53F6C
:10C3F000412E8640FFFFEF7F422ED63FFFFF2F3EAC
:10C400000000F03F50000100B1A2F03F70000100B9
:10C410006000010041F0004101F58010C00F70473D
:10C420000020704781F0004102E000BF83F000432C
:10C4300030B54FEA41044FEA430594EA050F08BFBF
:10C4400090EA020F1FBF54EA000C55EA020C7FEA83
:10C45000645C7FEA655C00F0E2804FEA5454D4EB00
:10C460005555B8BF6D420CDD2C4480EA020281EACA
:10C47000030382EA000083EA010180EA020281EA02
:10C480000303362D88BF30BD11F0004F4FEA013154
:10C490004FF4801C4CEA113102D0404261EB410163
:10C4A00013F0004F4FEA03334CEA133302D05242E9
:10C4B00063EB430394EA050F00F0A780A4F10104A5
:10C4C000D5F1200E0DDB02FA0EFC22FA05F28018DF
:10C4D00041F1000103FA0EF2801843FA05F35941C5
:10C4E0000EE0A5F120050EF1200E012A03FA0EFC44
:10C4F00028BF4CF0020C43FA05F3C01851EBE3716E
:10C5000001F0004507D54FF0000EDCF1000C7EEB8A
:10C5100000006EEB0101B1F5801F1BD3B1F5001FC8
:10C520000CD349085FEA30004FEA3C0C04F10104E7
:10C530004FEA445212F5800F80F09A80BCF1004F10
:10C5400008BF5FEA500C50F1000041EB045141EA92
:10C55000050130BD5FEA4C0C404141EB010111F493
:10C56000801FA4F10104E9D191F0000F04BF01463E
:10C570000020B1FA81F308BF2033A3F10B03B3F11C
:10C5800020020CDA0C3208DD02F1140CC2F10C02AC
:10C5900001FA0CF021FA02F10CE002F11402D8BF0A
:10C5A000C2F1200C01FA02F120FA0CFCDCBF41EAD6
:10C5B0000C019040E41AA2BF01EB0451294330BDA5
:10C5C0006FEA04041F3C1CDA0C340EDC04F1140482
:10C5D000C4F1200220FA04F001FA02F340EA030059
:10C5E00021FA04F345EA030130BDC4F10C04C4F19F
:10C5F000200220FA02F001FA04F340EA030029467F
:10C6000030BD21FA04F0294630BD94F0000F83F4C8
:10C61000801306BF81F480110134013D4EE77FEAAB
:10C62000645C18BF7FEA655C29D094EA050F08BFF7
:10C6300090EA020F05D054EA000C04BF19461046D8
:10C6400030BD91EA030F1EBF0021002030BD5FEA1C
:10C65000545C05D14000494128BF41F0004130BD44
:10C6600014F580043CBF01F5801130BD01F0004598
:10C6700045F0FE4141F470014FF0000030BD7FEA0B
:10C68000645C1ABF194610467FEA655C1CBF0B4606
:10C69000024650EA013406BF52EA033591EA030F1D
:10C6A00041F4002130BD00BF90F0000F04BF002115
:10C6B000704730B54FF4806404F132044FF0000548
:10C6C0004FF0000150E700BF90F0000F04BF0021C1
:10C6D000704730B54FF4806404F1320410F0004527
:10C6E00048BF40424FF000013EE700BF42004FEA22
:10C6F000E2014FEA31014FEA02701FBF12F07F439F
:10C7000093F07F4F81F06051704792F0000F14BF9B
:10C7100093F07F4F704730B54FF4607401F00045DF
:10C7200021F0004120E700BF50EA010208BF704736
:10C7300030B54FF000050AE050EA010208BF70472B
:10C7400030B511F0004502D5404261EB41014FF494
:10C75000806404F132045FEA915C3FF4DCAE4FF098
:10C7600003025FEADC0C18BF03325FEADC0C18BF7F
:10C77000033202EBDC02C2F1200300FA03FC20FAD0
:10C7800002F001FA03FE40EA0E0021FA02F114441D
:10C79000C1E600BF70B54FF0FF0C4CF4E06C1CEA32
:10C7A00011541DBF1CEA135594EA0C0F95EA0C0FA7
:10C7B00000F0DEF82C4481EA030621EA4C5123EA1A
:10C7C0004C5350EA013518BF52EA033541F4801149
:10C7D00043F4801338D0A0FB02CE4FF00005E1FBFC
:10C7E00002E506F00042E0FB03E54FF00006E1FB46
:10C7F00003569CF0000F18BF4EF0010EA4F1FF0489
:10C80000B6F5007F64F5407404D25FEA4E0E6D41C8
:10C8100046EB060642EAC62141EA55514FEAC520D9
:10C8200040EA5E504FEACE2EB4F1FD0C88BFBCF555
:10C83000E06F1ED8BEF1004F08BF5FEA500E50F106
:10C84000000041EB045170BD06F0004646EA0101CC
:10C8500040EA020081EA0301B4EB5C04C2BFD4EBFE
:10C860000C0541EA045170BD41F480114FF0000EF7
:10C87000013C00F3AB8014F1360FDEBF002001F065
:10C88000004170BDC4F10004203C35DA0C341BDCDF
:10C8900004F11404C4F1200500FA05F320FA04F0B1
:10C8A00001FA05F240EA020001F0004221F00041E5
:10C8B00010EBD37021FA04F642EB06015EEA430E58
:10C8C00008BF20EAD37070BDC4F10C04C4F1200588
:10C8D00000FA04F320FA05F001FA04F240EA02003B
:10C8E00001F0004110EBD37041F100015EEA430E0C
:10C8F00008BF20EAD37070BDC4F1200500FA05F22C
:10C900004EEA020E20FA04F301FA05F243EA0203AA
:10C9100021FA04F001F0004121FA04F220EA0200B9
:10C9200000EBD3705EEA430E08BF20EAD37070BDFF
:10C9300094F0000F0FD101F00046400041EB0101DF
:10C9400011F4801F08BF013CF7D041EA060195F0C1
:10C95000000F18BF704703F00046520043EB03037B
:10C9600013F4801F08BF013DF7D043EA0603704768
:10C9700094EA0C0F0CEA135518BF95EA0C0F0CD073
:10C9800050EA410618BF52EA4306D1D181EA0301B9
:10C9900001F000414FF0000070BD50EA410606BFB3
:10C9A0001046194652EA430619D094EA0C0F02D1F8
:10C9B00050EA013613D195EA0C0F05D152EA03363D
:10C9C0001CBF104619460AD181EA030101F000415B
:10C9D00041F0FE4141F470014FF0000070BD41F0A4
:10C9E000FE4141F4780170BD70B54FF0FF0C4CF47E
:10C9F000E06C1CEA11541DBF1CEA135594EA0C0F9D
:10CA000095EA0C0F00F0A7F8A4EB050481EA030EE9
:10CA100052EA03354FEA013100F088804FEA0333D0
:10CA20004FF0805545EA131343EA12634FEA02229E
:10CA300045EA111545EA10654FEA00260EF000415F
:10CA40009D4208BF964244F1FD0404F5407402D2B1
:10CA50005B084FEA3202B61A65EB03055B084FEA42
:10CA600032024FF480104FF4002CB6EB020E75EB3F
:10CA7000030E22BFB61A754640EA0C005B084FEA67
:10CA80003202B6EB020E75EB030E22BFB61A7546E4
:10CA900040EA5C005B084FEA3202B6EB020E75EB2F
:10CAA000030E22BFB61A754640EA9C005B084FEAA7
:10CAB0003202B6EB020E75EB030E22BFB61A7546B4
:10CAC00040EADC0055EA060E18D04FEA051545EAA3
:10CAD00016754FEA06164FEAC30343EA52734FEA4C
:10CAE000C2025FEA1C1CC0D111F4801F0BD141EAC5
:10CAF00000014FF000004FF0004CB6E711F4801F2A
:10CB000004BF01430020B4F1FD0C88BFBCF5E06F09
:10CB10003FF6AFAEB5EB030C04BFB6EB020C5FEA19
:10CB2000500C50F1000041EB045170BD0EF0004E6E
:10CB30004EEA113114EB5C04C2BFD4EB0C0541EAA0
:10CB4000045170BD41F480114FF0000E013C90E69D
:10CB500045EA060E8DE60CEA135594EA0C0F08BF61
:10CB600095EA0C0F3FF43BAF94EA0C0F0AD150EA60
:10CB700001347FF434AF95EA0C0F7FF425AF1046F3
:10CB800019462CE795EA0C0F06D152EA03353FF41B
:10CB9000FDAE1046194622E750EA410618BF52EA98
:10CBA00043067FF4C5AE50EA41047FF40DAF52EA6C
:10CBB00043057FF4EBAE12E74FF0FF3C06E000BF09
:10CBC0004FF0010C02E000BF4FF0010C4DF804CD16
:10CBD0004FEA410C7FEA6C5C4FEA430C18BF7FEAD6
:10CBE0006C5C1BD001B050EA410C0CBF52EA430C04
:10CBF00091EA030F02BF90EA020F0020704710F184
:10CC0000000F91EA030F58BF994208BF90422CBF12
:10CC1000D8176FEAE37040F0010070474FEA410C0B
:10CC20007FEA6C5C02D150EA013C07D14FEA430C29
:10CC30007FEA6C5CD6D152EA033CD3D05DF8040B9A
:10CC4000704700BF8446104662468C4619466346CC
:10CC500000E000BF01B5FFF7B7FF002848BF10F1A3
:10CC6000000F01BD4DF808EDFFF7F4FF0CBF0120E8
:10CC700000205DF808FB00BF4DF808EDFFF7EAFF64
:10CC800034BF012000205DF808FB00BF4DF808ED1F
:10CC9000FFF7E0FF94BF012000205DF808FB00BF14
:10CCA0004DF808EDFFF7CEFF94BF012000205DF89E
:10CCB00008FB00BF4DF808EDFFF7C4FF34BF0120AB
:10CCC00000205DF808FB00BF4FEA410212F5001298
:10CCD00015D211D56FF47873B3EB625212D94FEAC3
:10CCE000C12343F0004343EA505311F0004F23FAAD
:10CCF00002F018BF404270474FF00000704750EA02
:10CD0000013005D111F0004008BF6FF000407047BE
:10CD10004FF00000704700BF4FEA4102B2F1E0431C
:10CD200024BFB3F5001CDCF1FE5C0DD901F0004C12
:10CD30004FEAC0024CEA5070B2F1004F40EB830062
:10CD400008BF20F00100704711F0804F21D113F18E
:10CD50003872BCBF01F00040704741F480114FEAC7
:10CD60005252C2F11802C2F1200C10FA0CF320FA50
:10CD700002F018BF40F001004FEAC1234FEAD3236D
:10CD800003FA0CFC40EA0C0023FA02F34FEA4303D7
:10CD9000CCE77FEA625307D150EA01331EBF4FF060
:10CDA000FE4040F44000704701F0004040F0FE407B
:10CDB00040F40000704700BF80F0004002E000BF78
:10CDC00081F0004142001FBF5FEA410392EA030F76
:10CDD0007FEA226C7FEA236C6AD04FEA1262D2EBC0
:10CDE0001363C1BFD218414048404140B8BF5B42C5
:10CDF000192B88BF704710F0004F40F4000020F05E
:10CE00007F4018BF404211F0004F41F4000121F073
:10CE10007F4118BF494292EA030F3FD0A2F10102BD
:10CE200041FA03FC10EB0C00C3F1200301FA03F1FB
:10CE300000F0004302D5494260EB4000B0F5000F1E
:10CE400013D3B0F1807F06D340084FEA310102F1DD
:10CE50000102FE2A51D2B1F1004F40EBC25008BF8F
:10CE600020F0010040EA03007047490040EB000059
:10CE700010F4000FA2F10102EDD1B0FA80FCACF188
:10CE8000080CB2EB0C0200FA0CF0AABF00EBC25087
:10CE900052421843BCBFD0401843704792F0000F75
:10CEA00081F4000106BF80F400000132013BB5E7C8
:10CEB0004FEA41037FEA226C18BF7FEA236C21D03E
:10CEC00092EA030F04D092F0000F08BF08467047A3
:10CED00090EA010F1CBF0020704712F07F4F04D171
:10CEE000400028BF40F00040704712F100723CBF84
:10CEF00000F50000704700F0004343F0FE4040F4AE
:10CF0000000070477FEA226216BF08467FEA23636B
:10CF10000146420206BF5FEA412390EA010F40F456
:10CF2000800070474FF0000304E000BF10F00043A2
:10CF300048BF40425FEA000C08BF704743F0964389
:10CF400001464FF000001CE050EA010208BF7047A4
:10CF50004FF000030AE000BF50EA010208BF70472B
:10CF600011F0004302D5404261EB41015FEA010C40
:10CF700002BF84460146002043F0B64308BFA3F138
:10CF80008053A3F50003BCFA8CF2083AA3EBC2531A
:10CF900010DB01FA02FC634400FA02FCC2F1200239
:10CFA000BCF1004F20FA02F243EB020008BF20F070
:10CFB0000100704702F1200201FA02FCC2F12002D6
:10CFC00050EA4C0021FA02F243EB020008BF20EACB
:10CFD000DC7070474FF0FF0C1CEAD0521EBF1CEAF9
:10CFE000D15392EA0C0F93EA0C0F6FD01A4480EAE7
:10CFF000010C400218BF5FEA41211ED04FF00063D0
:10D0000043EA501043EA5111A0FB01310CF00040FB
:10D01000B1F5000F3EBF490041EAD3715B0040EA21
:10D02000010062F17F02FD2A1DD8B3F1004F40EBF1
:10D03000C25008BF20F00100704790F0000F0CF0C4
:10D04000004C08BF49024CEA502040EA51207F3A88
:10D05000C2BFD2F1FF0340EAC250704740F4000063
:10D060004FF00003013A5DDC12F1190FDCBF00F054
:10D0700000407047C2F10002410021FA02F1C2F102
:10D08000200200FA02FC5FEA310040F1000053EA9E
:10D090004C0308BF20EADC70704792F0000F00F0EC
:10D0A000004C02BF400010F4000F013AF9D040EAF2
:10D0B0000C0093F0000F01F0004C02BF490011F486
:10D0C000000F013BF9D041EA0C018FE70CEAD15384
:10D0D00092EA0C0F18BF93EA0C0F0AD030F0004C04
:10D0E00018BF31F0004CD8D180EA010000F00040B8
:10D0F000704790F0000F17BF90F0004F084691F076
:10D10000000F91F0004F14D092EA0C0F01D14202AF
:10D110000FD193EA0C0F03D14B0218BF084608D178
:10D1200080EA010000F0004040F0FE4040F40000C2
:10D13000704740F0FE4040F4400070474FF0FF0C55
:10D140001CEAD0521EBF1CEAD15392EA0C0F93EA9C
:10D150000C0F69D0A2EB030280EA010C49024FEAEE
:10D16000402037D04FF0805343EA111143EA1013A7
:10D170000CF000408B4238BF5B0042F17D024FF45F
:10D18000000C8B4224BF5B1A40EA0C00B3EB510F3A
:10D1900024BFA3EB510340EA5C00B3EB910F24BF23
:10D1A000A3EB910340EA9C00B3EBD10F24BFA3EBA8
:10D1B000D10340EADC001B0118BF5FEA1C1CE0D170
:10D1C000FD2A3FF650AF8B4240EBC25008BF20F023
:10D1D000010070470CF0004C4CEA50207F32C2BF77
:10D1E000D2F1FF0340EAC250704740F400004FF014
:10D1F0000003013A37E792F0000F00F0004C02BF45
:10D20000400010F4000F013AF9D040EA0C0093F00E
:10D21000000F01F0004C02BF490011F4000F013B68
:10D22000F9D041EA0C0195E70CEAD15392EA0C0FD0
:10D2300008D142027FF47DAF93EA0C0F7FF470AF08
:10D24000084676E793EA0C0F04D14B023FF44CAF4B
:10D2500008466EE730F0004C18BF31F0004CCAD1E0
:10D2600030F000427FF45CAF31F000437FF43CAF1C
:10D270005FE700BF4FF0FF3C06E000BF4FF0010C3E
:10D2800002E000BF4FF0010C4DF804CD4FEA400220
:10D290004FEA41037FEA226C18BF7FEA236C11D06A
:10D2A00001B052EA530C18BF90EA010F58BFB2EB1D
:10D2B000030088BFC81738BF6FEAE17018BF40F09D
:10D2C000010070477FEA226C02D15FEA402C05D151
:10D2D0007FEA236CE4D15FEA412CE1D05DF8040BD6
:10D2E000704700BF844608466146FFE70FB5FFF769
:10D2F000C9FF002848BF10F1000F0FBD4DF808ED21
:10D30000FFF7F4FF0CBF012000205DF808FB00BF11
:10D310004DF808EDFFF7EAFF34BF012000205DF86B
:10D3200008FB00BF4DF808EDFFF7E0FF94BF0120B8
:10D3300000205DF808FB00BF4DF808EDFFF7D2FFB5
:10D3400094BF012000205DF808FB00BF4DF808EDF8
:10D35000FFF7C8FF34BF012000205DF808FB00BFC5
:10D360004FEA4002B2F1FE4F0FD34FF09E03B3EBF2
:10D3700012620DD94FEA002343F0004310F0004F32
:10D3800023FA02F018BF404270474FF00000704788
:10D3900012F1610F01D1420205D110F0004008BF27
:10D3A0006FF0004070474FF00000704742000ED20F
:10D3B000B2F1FE4F0BD34FF09E03B3EB126209D4D0
:10D3C0004FEA002343F0004323FA02F070474FF086
:10D3D0000000704712F1610F01D1420202D14FF0FB
:10D3E000FF3070474FF00000704700BF0B4601460A
:10D3F000184600F001B800BF13460A460146022055
:10D4000000F0B0BE014B1868704700BF3896FF1F90
:10D4100070B50F4E0F4D761BB61018BF002405D007
:10D42000013455F8043B9847A642F9D10A4E0B4DFA
:10D43000761B02F027FEB61018BF002406D0013478
:10D4400055F8043B9847A642F9D170BD70BD00BFA6
:10D450009000010090000100A40001009000010074
:10D46000024B0146186800F00BB800BF3896FF1F4A
:10D47000024B0146186800F039BF00BF3896FF1F05
:10D480002DE9F04F01F10B05162D83B0064640F251
:10D490009F8035F0070500F1BF80A94200F2BC80F3
:10D4A00000F058FBB5F5FC7FC0F09C826B0A00F0E1
:10D4B000BA80042B00F28381A80900F1390E4FEAEB
:10D4C0004E033830C44F07EB8303A3F108015C68B7
:10D4D000A14207D1ACE0002A80F2AC80E468A1420E
:10D4E00000F0A680636823F003035A1B0F2AF2DDC5
:10D4F000B9493C6901F1080E744500F0B3816368D5
:10D5000023F003035A1B0F2A00F39981002AC1F864
:10D5100014E0C1F810E080F29E80B3F5007F80F047
:10D520006781DB0803F1010C01229B1002FA03F36F
:10D530004A6851F83C80C4F8088001EBCC091A43D2
:10D54000A9F10803E3604A6041F83C40C8F80C4088
:10D55000831001249C40944200F28A80144206D138
:10D5600020F003006400144200F10400FAD007EB3D
:10D57000C009CC468046DCF80C108C4507D173E11D
:10D58000002A80F28181C9688C4500F06D814B686A
:10D5900023F003035A1B0F2AF2DD0C46D1F80CC00E
:10D5A00054F8088F4B1945F001054D6042F0010118
:10D5B000C8F80CC03046CCF808807B613B61C3F8EA
:10D5C0000CE0C3F808E059609A5000F0C5FA1FE07B
:10D5D000102921D800F0BEFA1025062302207E4F24
:10D5E00007EB8303A3F108025C68944200F04581D5
:10D5F0006368E168A56823F00303234430465A6852
:10D60000E96042F001028D605A6000F0A5FA08342A
:10D61000204603B0BDE8F08F00240C232046336081
:10D6200003B0BDE8F08F80234FF0400E3F2049E764
:10D6300070465DE72344E1685A68A56842F001023C
:10D64000E96030468D605A6000F086FA0834204662
:10D6500003B0BDE8F08F234430465A6842F001021F
:10D660005A6000F079FA0834204603B0BDE8F08F24
:10D67000BC68636823F00308A84504D3C5EB08031E
:10D680000F2B00F38C80554BDFF860911A68D9F8A6
:10D69000003001332A4404EB080A00F0608102F5EF
:10D6A00080520F3222F47F6222F00F021146304680
:10D6B000019200F04BFCB0F1FF3F8346019A00F06D
:10D6C0005881824500F2FC80454B1968DA451144C7
:10D6D000196000F05381D9F80000DFF810E1013043
:10D6E0001BBFCAEB0B0A5144CEF800B019601BF007
:10D6F000070100F01781C1F10800C1F58051834492
:10D7000008315A44C2F30B02C2EB010949463046C4
:10D71000019300F01BFC431C019B00F03F81CBEB0D
:10D7200000024A4442F001021968C7F808B04944AF
:10D73000BC42CBF804201960DFF8A49016D0B8F1F1
:10D740000F0F40F2FD806268A8F10C0323F007037D
:10D75000E01802F001024FF0050E1A430F2B626031
:10D76000C0F804E0C0F808E000F21C811D4BBC6862
:10D770001A68914288BF19601B4B1A68914262680F
:10D7800088BF196022F003029542A2EB050301D87D
:10D790000F2B04DC304600F0DFF9002438E7621973
:10D7A00043F0010345F0010565603046BA605360FF
:10D7B00000F0D2F90834204603B0BDE8F08F142BF6
:10D7C00071D9542B00F2A480280B00F16F0E4FEAA0
:10D7D0004E036E3076E600BF3C96FF1FD09FFF1FC2
:10D7E000D49FFF1FCC9FFF1FC89FFF1F489AFF1F9A
:10D7F0005A0A042A5ED9142A00F2B38002F15C01AD
:10D8000049005B3207EB810C57F82110DFF8DC810F
:10D81000ACF1080C8C4500F088804A6822F00302C5
:10D82000934202D289688C45F7D1D1F80CC07A684E
:10D83000C4F80CC0A160CCF80840CC6088E663193D
:10D8400042F0010745F00105656030464B610B6110
:10D85000C3F80CE0C3F808E05F609A50083400F0A9
:10D860007BF9D5E64A6873E608F1010818F0030F62
:10D870000CF1080C7FF47FAE30E0DC68A34208BFF7
:10D8800002303FF435AEB3E60B440C465A68C96823
:10D8900054F8085F42F001025A603046E9608D603A
:10D8A00000F05AF9B4E603F15C0E03F15B004FEAB5
:10D8B0004E0307E69A0902F1390149003832A1E71F
:10D8C000BC424A4B3FF400AF9C68626822F00302FE
:10D8D0005AE759F80839994540F0828010F0030F53
:10D8E00000F1FF30F5D17B6823EA04037B6064001C
:10D8F0009C423FF6BDAE002C3FF4BAAE1C424046FF
:10D900007FF435AE64001C4200F10400FAD02EE62C
:10D91000B3F5AA7F18D8E80B00F1780E4FEA4E0352
:10D920007730CFE54FF48051EBE60121D8F8043091
:10D93000921001FA02F21A43C8F80420614677E710
:10D940000123CBF8043025E740F25452934220D80B
:10D95000A80C00F17D0E4FEA4E037C30B2E5103288
:10D96000A4E6542A26D81A0B02F16F0149006E3240
:10D9700048E7BC68626822F0030205E7CAF30B00BF
:10D9800000287FF4A8AE4244BB6842F001025A600E
:10D99000ECE6FE234FF07F0E7E2093E501224FF050
:10D9A0000009C1E604F10801304600F09FFCD9F8F7
:10D9B0000010DBE6B2F5AA7F05D8DA0B02F1780198
:10D9C000490077321EE740F254518A4205D89A0C3A
:10D9D00002F17D0149007C3214E7FE217E2211E72D
:10D9E0007B6884E7E808431C5B00F8E53C96FF1F72
:10D9F0008842F0B50DD98B1898420AD28118002AB6
:10DA000051D09A1A13F8014D01F8014D9342F9D102
:10DA1000F0BD0F2A48D941EA00039B0746D100F127
:10DA2000100401F11003154653F8106C44F8106C03
:10DA300053F80C6C44F80C6C53F8086C44F8086C00
:10DA4000103D53F8046C44F8046C0F2D03F11003DF
:10DA500004F11004E8D8A2F1100323F00F0302F040
:10DA60000F0E1033BEF1030F1944034421D91E1FBA
:10DA70000D467446043C55F8047B46F8047F032C9D
:10DA8000F8D8AEF1040424F0030404342344214400
:10DA900002F0030262B1013B0A4411F8014B03F8A2
:10DAA000014F8A42F9D1F0BD0346F3E70346F2E79E
:10DAB000F0BD7246EEE700BF70B4840746D0541E36
:10DAC000002A41D0CDB2034602E0621EE4B3144600
:10DAD00003F8015B9A07F8D1032C2ED9CDB245EAA1
:10DAE00005250F2C45EA054519D903F110022646F4
:10DAF000103E0F2E42F8105C42F80C5C42F8085CB5
:10DB000042F8045C02F11002F2D8A4F1100222F0F3
:10DB10000F0204F00F041032032C13440DD91E46DB
:10DB20002246043A032A46F8045BFAD8221F22F060
:10DB300003020432134404F003042CB1C9B21C44A0
:10DB400003F8011BA342FBD170BC70471446034687
:10DB5000C2E700BF704700BF704700BF024B0A46D4
:10DB60000146186800F002B83896FF1F2DE9F04F03
:10DB7000174683B0002900F0C1800E46814607F1A8
:10DB80000B05FFF7E7FF56F804EC162D2EF0030403
:10DB9000A6F1080840D810221546AF4241D8944259
:10DBA00075DAC94B996808EB04008842416800F0B7
:10DBB000D98021F0010303445B68DB077DD51EF0AB
:10DBC000010F35D039464846FFF75AFC0746E0B109
:10DBD00056F8043C23F001034344A0F108029A42A2
:10DBE00000F04481221F242A00F23181132A00F21E
:10DBF0000481034632461168196051685960926881
:10DC00009A603146484600F071FB4846FFF7A4FF92
:10DC1000384603B0BDE8F08F25F00705002D2A46F1
:10DC2000BBDA0C230020C9F8003003B0BDE8F08F48
:10DC300056F8083CC3EB080ADAF8043023F0030C6A
:10DC400004EB0C039342BDDB5746DAF80C1057F88F
:10DC5000080F221F242AC160886000F21781132A4E
:10DC600040F212813168CAF808107168CAF80C10C5
:10DC70001B2A00F22B8108360AF11002316811606C
:10DC800071685160B16891603E461C46D046631B86
:10DC90000F2B1DD8D8F8043003F00103234344446C
:10DCA000C8F80430636843F0010363604846FFF737
:10DCB00053FF304603B0BDE8F08F21F0030121444B
:10DCC000914221DBC36882680C46D3609A60DEE72C
:10DCD000D8F8042008EB050102F00102154343F0D7
:10DCE00001020B44C8F804504A605A6842F001022D
:10DCF00008315A60484600F0F9FAD7E7114603B0F8
:10DD0000BDE8F04FFFF7BCBB1EF0010F7FF45AAF28
:10DD100056F8083CC3EB080ADAF8043023F0030C89
:10DD200001EB0C0E96458BDBC36882685746D360C7
:10DD30009A6057F8081FDAF80C30CB60221F242AAB
:10DD4000996000F29980132A62D93368CAF80830C2
:10DD50007368CAF80C301B2A00F2A08008360AF15A
:10DD6000100356E021F0030BA34405F11000834596
:10DD700059DA1EF0010F7FF425AF56F8081CC1EBED
:10DD8000080ADAF8041021F0030CE34458453FF781
:10DD900057AF5746DAF80C1057F8080F221F242AFD
:10DDA000C160886000F2B480132A40F2A580316817
:10DDB000CAF808107168CAF80C101B2A00F2AF806C
:10DDC00008360AF110023168116071685160B1685B
:10DDD00091600AEB0501C5EB0B0242F0010299606C
:10DDE0004A60DAF8043003F001031D434846CAF8DC
:10DDF0000450FFF7B1FE38465CE733680360736890
:10DE000043601B2A27D800F1080306F10802F2E656
:10DE10003B4632681A6072685A60B2689A603E4641
:10DE20007446D04633E708EB0501C5EB0B0B4BF00E
:10DE3000010299604A6056F8043C03F001031D4357
:10DE4000484646F8045CFFF787FE304632E7314625
:10DE5000FFF7CEFDD5E6B3688360F368C360242A7C
:10DE600028D000F1100306F11002C4E650F8043C7B
:10DE700023F003031C440AE7314638467446D04673
:10DE8000FFF7B6FD3E4602E73A46F7E6314638462A
:10DE90001C46D046FFF7ACFD3E46F8E6B368CAF82C
:10DEA0001030F368CAF81430242A1BD010360AF157
:10DEB0001803AEE7336903617369436106F1180221
:10DEC00000F1180397E600BF3C96FF1FB168CAF83F
:10DED0001010F168CAF81410242A0FD010360AF175
:10DEE0001802CBE63369CAF818307369CAF81C30D7
:10DEF00018360AF120038CE73A4664E73269CAF81B
:10DF000018207269CAF81C2018360AF12002B5E6FA
:10DF1000314638460193FFF76BFD019B59E7B16825
:10DF2000CAF81010F168CAF81410242A03D0103669
:10DF30000AF1180247E73269CAF818207269CAF86C
:10DF40001C2018360AF120023DE700BF38B5074C07
:10DF50000023054608462360FBF7E2FE431C00D081
:10DF600038BD2368002BFBD02B6038BD30A1FF1FCC
:10DF7000FFFFFFFFFFFFFFFFFFFFFFFFFFFFFFFFB1
:10DF800090F800F06DE9024520F007016FF0000CF9
:10DF900010F0070491F820F040F049804FF00004A1
:10DFA0006FF00700D1E9002391F840F000F108007C
:10DFB00082FA4CF2A4FA8CF283FA4CF3A2FA8CF3B4
:10DFC0004BBBD1E9022382FA4CF200F10800A4FA1B
:10DFD0008CF283FA4CF3A2FA8CF3E3B9D1E904236F
:10DFE00082FA4CF200F10800A4FA8CF283FA4CF3A6
:10DFF000A2FA8CF37BB9D1E9062301F1200182FA60
:10E000004CF200F10800A4FA8CF283FA4CF3A2FA65
:10E010008CF3002BC6D0002A04BF04301A4612BA73
:10E02000B2FA82F2FDE8024500EBD2007047D1E976
:10E03000002304F00305C4F100004FEAC50514F005
:10E04000040F91F840F00CFA05F562EA05021CBFD6
:10E0500063EA050362464FF00004A9E7002A41D0B5
:10E0600040EA010313F00303F0B425D1032A23D9B6
:10E0700004680D68AC421FD1043A35D0A4F10135D3
:10E0800025EA040414F0803F31D1071D0D1D0DE079
:10E0900057F8043B0E68A3F10134B34224EA0304A9
:10E0A0000AD1043A20D014F0803F23D1032A294614
:10E0B000384605F10405EBD803780C789C4202F150
:10E0C000FF320CD182B114B916E06AB17BB110F8FD
:10E0D000013F11F8014FA34202F1FF32F5D0181BA6
:10E0E000F0BC7047104670471046F0BC70471846A9
:10E0F000F0BC70470020F3E72046F1E740EA010357
:10E100009B0770B42BD1032A29D90C46034621461C
:10E1100054F8046BA6F1013525EA060515F0803F99
:10E1200006D1043A032A43F8046B2146EFD8A2B182
:10E130000C781C70013A013301313CB16AB111F81D
:10E14000014B03F8014B013A002CF7D12AB11A44D4
:10E15000002103F8011B9A42FBD170BC70470346B3
:10E16000E5E700BF2DE9F047254C2568D5F8484183
:10E170000646884692469946C4B360681F2817DC55
:10E18000431C76B104EB80050122C5F888A0D4F8C1
:10E19000881182401143022EC4F88811C5F80891F5
:10E1A0001ED00230636044F820800020BDE8F08774
:10E1B000144B03B34FF4C870FFF752F90446D0B1C3
:10E1C000D5F84831002780E88800C5F8484138462E
:10E1D0000123C4F88871C4F88C71002EE1D0D1E716
:10E1E000D4F88C110A43C4F88C21DAE705F5A6743B
:10E1F000C5F84841C1E74FF0FF30BDE8F08700BFE8
:10E200008000010061D40000024B13B1024800F00D
:10E2100005B870470000000029E200000023014615
:10E220001A461846FFF79EBF38B5074D074C2C1B02
:10E23000A41005D0013C55F8043D9847002CF9D1B5
:10E24000BDE8384001F02EBF0000000000000000D3
:10E25000F8B5234F0C460646FFF77CFCBB685D68AB
:10E2600025F00305291B01F6EF7121F47F6121F0F0
:10E270000F01A1F58054B4F5805F07DB0021304623
:10E28000FFF764FEBB682B44984204D03046FFF78A
:10E2900063FC0020F8BD61423046FFF757FE0130B5
:10E2A0000DD0104BBA6819682D1B45F0010530469A
:10E2B000091B55601960FFF74FFC0120F8BD0021D4
:10E2C0003046FFF743FEBA68831A0F2BDEDD064C9B
:10E2D0000449246843F00103001B53600860D5E73C
:10E2E0003C96FF1FD49FFF1F489AFF1F002945D06F
:10E2F0002DE9F0410D468046FFF72CFC55F8047CD3
:10E300006A4927F00103A5F10804E2188E685068F5
:10E31000B24220F0030062D0FE0750600BD455F8E3
:10E32000087CE41B01F1080EA56875453B446FD0DD
:10E33000E768EF60BD6015186D68ED0742D543F0E2
:10E3400001026260E350B3F5007F18D2DB085A1C6B
:10E350004D6851F83270A76001209B1000FA03F35A
:10E3600001EBC2001D430838E0604D6041F83240C7
:10E37000FC604046BDE8F041FFF7EEBB70475A0A2B
:10E38000042A53D89A0902F139077F0002F13805AF
:10E3900001EB870051F827204449083890424DD0BE
:10E3A000516821F003018B4202D292689042F7D16A
:10E3B000D068E060A2608460D4604046BDE8F0416F
:10E3C000FFF7CABB95683A4FBD4203443FD0D068BF
:10E3D000E86043F0010285606260E350B3E7FF0745
:10E3E000034407D455F8082CA41A1344A068E26823
:10E3F000C26090602F4A126843F00100934260604F
:10E400008C60B6D32C4B40461968FFF721FFB0E76C
:10E4100011184968C90744D49168D268CA60034496
:10E4200043F0010091606060E350A2E7142A17D81E
:10E4300002F15C077F0002F15B05A9E7AA104B68B7
:10E44000012505FA02F213434B600246B1E743F09F
:10E4500001024C610C61E560A5606260E35088E7F1
:10E46000542A06D81A0B02F16F077F0002F16E05DD
:10E470008EE7B2F5AA7F06D8DA0B02F178077F00A3
:10E4800002F1770584E740F25450824206D89A0C94
:10E4900002F17D077F0002F17C0579E7FE277E25EA
:10E4A00076E743F001026260E35062E73C96FF1FAB
:10E4B0004496FF1F449AFF1FD09FFF1F0000CC10FF
:10E4C000581BFC21AC26C62A7C2E3831F4334C363E
:10E4D000A438983A5A3C543D803E7A3FFF3FFFFFB4
:10E4E0000000580246056608540BD80E5C127017DF
:10E4F000FC21F82A70305834DC37663A8C3C803E78
:10E50000FF3FFFFF0000FF03FF07FF0BFF0FFF139D
:10E51000FF17FF1BFF1FFF23FF27FF2BFF2FFF33DB
:10E52000FF37FF3BFF3FFFFF0000D007100E8813AF
:10E530003219AA1E282374275C2B442F6432843599
:10E540004038663A8C3C803EFF3FFFFF0000900160
:10E5500020031405D0075A0AAC0DCC10B4146A1865
:10E56000E81C342180252A2B70301437FF3FFFFF31
:10E570000000580246056608540BD80E5C12E015E0
:10E58000FA19141E6022AC265C2B0C30BC34023A03
:10E59000FF3FFFFF0000C800F401840314050807D3
:10E5A0002E091C0CD80EF811AE159619401F1C250B
:10E5B000F22B5834FF3FFFFF00006400C8009001B9
:10E5C000BC021A04DC059E07F609800CA00F241378
:10E5D000A2174C1D5424442FFF3FFFFF0000580298
:10E5E00046056608540BA00FD4172823F82A442F99
:10E5F000643284354038663A8C3C803EFF3FFFFFF2
:10E6000000007805220B0410B4143219B01DFC214F
:10E610004826FE29822D383126344637663A223D77
:10E62000FF3FFFFF0000540BEC13FA1908201C25D4
:10E630003629EC2C0C302C33E8357238663AF63B30
:10E64000863D163FFF3FFFFFBCE4000024E60000CC
:10E6500028E5000000E6000004E5000070E5000089
:10E660004CE5000094E50000B8E50000E0E400009F
:10E67000DCE5000004E700007CE600000000D007B5
:10E68000800CD80E0010C012EC130C17FA19141ECF
:10E690006022AC265C2B0C30BC34023AFF3FFFFFFB
:10E6A00000000000CDCC4C3DCDCCCC3D9A99193E1C
:10E6B000CDCC4C3E0000803E9A99993E3333B33E18
:10E6C000CDCCCC3E6666E63E2C011301FA00E1009B
:10E6D000C800AF0096007D0064004B0032001900B6
:10E6E00040067805B004E80384032003BC02580206
:10E6F000F40190012C01FA00C80096006400320079
:10E700001900FFFF000078053408540B800C3C0F03
:10E710005C12E015FA19141E6022AC265C2B0C303A
:10E72000BC34023AFF3FFFFF98E70000EE9AFF1F5C
:10E730000000FF0FFA9BFF1F0000FF0FC93300000E
:10E7400064E700005C9BFF1F32005E0100000000D8
:10E75000000000006933000054485200534E53003B
:10E760004D415800544F5543482053454E534500A2
:10E77000455854524120434F4E54524F4C4C4552F1
:10E780000000000050495443482042454E440000D8
:10E79000424954450000000042524541544800FFA0
:10E7A00070E70000B49BFF1FF401A00F269BFF1F22
:10E7B000F401A00F7533000090E70000949BFF1F49
:10E7C000BC025C12EA9AFF1FBC025C12AD3300006F
:10E7D00084E70000E89BFF1FF401A00F589BFF1F78
:10E7E000F401A00F9133000068EF000070EF00000B
:10E7F00088EE000034EF000048EF00004CEF00000E
:10E8000050EF000054EF000058EF00005CEF0000F4
:10E8100060EF00003CEF000064EF000088EE0000B5
:10E8200084EE000044EF000088EE000034EF0000AA
:10E8300038EF00003CEF000040EF000078EF0000F0
:10E840007CEF000080EF000084EF000088EF000004
:10E850008CEF000090EF000094EF000098EF0000B4
:10E860009CEF0000A0EF0000A4EF0000A8EF000064
:10E870000000000028F1000010F10000D69BFF1FEF
:10E880000000300000000000654D0000F140000075
:10E890000000000000000000000000000000000078
:10E8A0000000000000000000000000000000000068
:10E8B0000000000000000000000000000000000058
:10E8C0000000000000000000000000000000000048
:10E8D0000000000000000000000000000000000038
:10E8E0000000000000000000000000000000000028
:10E8F0000000000000000000000000000000000018
:10E900000000000000000000000000000000000007
:10E9100000000000000000000000000000000000F7
:10E9200000000000000000000000000000000000E7
:10E9300000000000000000000000000000000000D7
:10E9400000000000000000000000000000000000C7
:10E9500000000000000000000000000000000000B7
:10E9600000000000000000000000000000000000A7
:10E970000000000000000000000000000000000097
:10E980000000000000000000000000000000000087
:10E990000000000000000000000000000000000077
:10E9A0000000000000000000000000000000000067
:10E9B00000000000000000000001FFFFFFE3600016
:10E9C00007736000000000000001FFFFFFE360002C
:10E9D0000EE3600000000000000180000003600002
:10E9E0001DC36000000000000001BFFFFFE36000E6
:10E9F0003B836000000000000001BFFFFFE36000F8
:10EA000077036000000000000001B0000003600018
:10EA1000EE036000000000000001B0000003600190
:10EA2000DC036000000000000001B0000003600390
:10EA3000B8036000000000200001B0000003600780
:10EA400070036000000000600001BFFFFFE3600E84
:10EA5000E0036000000000600001BFFFFFE3601DF5
:10EA6000C003600000030060000180000003603B01
:10EA700080036000000300E00001BFFFFFE3607758
:10EA800000036000000300C00001BFFFFFE360EE71
:10EA900000036000000380C00001B000000361DCDF
:10EAA00000036000000780C00001B000000363B8ED
:10EAB000000360000007C0C00001B00000036770E1
:10EAC000000360000006C0C00001B00000036EE05B
:10EAD00000036000000660C10101B00000037DC0BA
:10EAE00000036000000630C30301BFFFFFE37B802B
:10EAF00000036000000C30C30701BFFFFFE3770095
:10EB000000036000000C1CC30601800000030E001F
:10EB100000036000000C0CC20E01FFFFFFE3FC00CD
:10EB200000036000000C0EC61E01FFFFFFE3F800AB
:10EB300000036000000C07C61E000000000000007B
:10EB400000000000000C03C676000000000000007A
:10EB500000000000000C01C7E600000000000000FB
:10EB600000000000000C00C7C6000000000000000C
:10EB700000000000000C0003060000000000000080
:10EB800000000000000C0000000000000000000079
:10EB900000000000000C0000000000000000000069
:10EBA0000000000000000000000000000000000065
:10EBB0000000000000000000000000000000000055
:10EBC0000000000000000000000000000000000045
:10EBD0000000000000000000000000000000000035
:10EBE0000000000000000000000000000000000025
:10EBF0000000000000000000000000000000000015
:10EC00000000000000000000000000000000000004
:10EC100000000000000000000000000000000000F4
:10EC200000000000000000000000000000000000E4
:10EC300000000000000000000000000000000000D4
:10EC400000000000000000000000000000000000C4
:10EC500000000000000000000000000000000000B4
:10EC600000000000000000000000000000000000A4
:10EC70000000000000000000000000000000000094
:10EC80000000000000000000000000000000000084
:10EC9000000000000000000040F1000010F1000042
:10ECA000B69BFF1F0000300000000000554D000023
:10ECB0008D3D0000000000000100000074F1000024
:10ECC000030000000100000054F1000009000000F2
:10ECD00001000000ACEF0000070000000000000091
:10ECE0001CF1000010F10000D89BFF1F0000300055
:10ECF00000000000654D0000F14000000000000031
:10ED0000010000005CF100000500000001000000AF
:10ED10004CF10000080000000000000098F0000026
:10ED200098F000005E9BFF1F00000C000300000035
:10ED30007D5100009D3D000000000000000000002B
:10ED400004F1000010F10000DA9BFF1F000030000A
:10ED500000000000654D0000F140000000000000D0
:10ED600000000000010000001D4100000100000043
:10ED700068F1000004000000000000007CF10000C9
:10ED800084F100003A9BFF1F010010000600000004
:10ED9000115400006D3D00001D4400002C010000D6
:10EDA0003140000006000000080000007C8DFF1FBD
:10EDB000DCF000000200030006000000088EFF1FC8
:10EDC0000000000001000000B156000054F10000F6
:10EDD000000005010A000000608BFF1F70F00000BA
:10EDE0000000010108000000608CFF1F000000000F
:10EDF00034F1000010F10000D49BFF1F0000300030
:10EE000000000000654D0000F1400000000000001F
:10EE1000ACEF000000000405080000005C8DFF1F3F
:10EE200000000000ECF00000F8F000001C9BFF1F49
:10EE30000000010001000000A94500007D3D000028
:10EE4000000000000000000008F00000D4EF000007
:10EE5000369BFF1F0000090000000000CD450000A8
:10EE6000AD3D0000000000000000000001000000B7
:10EE70007D49000010F000000000020108000000C1
:10EE8000448EFF1F4F4E00004F4646004241540043
:10EE90004C4F572000000000555342004D454E5541
:10EEA00020202020202020202058585820592E593A
:10EEB000560000005800000041540000524F54001A
:10EEC0004D454C0044594E00312F00006D73000039
:10EED00042544800424954004C5652004E524D0094
:10EEE00052455600504244004543320045435300CA
:10EEF0004C564C004C565000474C4400762E0000B7
:10EF0000312E342E330000004E7545564900000066
:10EF10006669726D7761726520762E0053455400E4
:10EF2000434C5200444F4E275400000050414E497C
:10EF3000430000004D5700004650000043460000CB
:10EF4000535000005357000042520000564C00003E
:10EF5000455800004D572B0042522B00564C2B00B9
:10EF600045582B00554E4F004252544800000000B7
:10EF700050544348000000002D3400002D330000A1
:10EF80002D3200002D3100004C494E002B31000085
:10EF90002B3200002B3300002B34000053310000D3
:10EFA000533200005A3100005A3200005649425292
:10EFB00041544F00444952454354494F4E000000CC
:10EFC000434F4E54524F4C00535155454C434820EB
:10EFD000420000004C4556454C00000053454E533E
:10EFE0004520425445000000535155454C434820AC
:10EFF0004C00000053454E5345204C565200000033
:10F0000052455455524E00004445505448000000AB
:10F010005345545550204354524C53004C4556458B
:10F020004C2043430000000050494E4B59204B45B3
:10F03000590000004445474C495443480000000033
:10F04000455843545220434332000000455854521F
:10F050004120435452000000504954434842454E19
:10F0600044000000504F52542F474C440000000011
:10F070005345545550204252454154480000000029
:10F0800056454C20424F4F535400000056454C20EB
:10F0900044454C415900000043555256450000007C
:10F0A00056454C4F434954590000000042524541D7
:10F0B00054482041540000004343322052495345F4
:10F0C0000000000042525448204343320000000038
:10F0D000425254482043433100000000524F5441F3
:10F0E000544F522053455455500000005052494F40
:10F0F00052495459000000004D4F4E4F2050524984
:10F100004F000000524F544154452034000000008D
:10F1100053454D49544F4E4553000000524F544102
:10F120005445203300000000524F544154452032D2
:10F1300000000000524F54415445203100000000AF
:10F14000504152414C4C454C0000000041424F554B
:10F150005400000045585452415300005345545543
:10F16000502043544C000000534554555020425207
:10F170000000000041444A55535400004D494449A1
:10F18000204348004D4944492043484E4C0000006C
:10F19000574C204348414E00574C20504F57455242
:10F1A000000000004641535420424F4F54000000DD
:10F1B000444143204F55540042434153204D4F4456
:10F1C00045000000335244205452494C4C0000008A
:10F1D00053504543204B45590000000047415445DA
:10F1E00020484F4C440000004C45474143592042C1
:10F1F000520000004C454741435920504200000056
:10F200004F435441564500005452414E53504F53C2
:10F210004500FFFF00211102020000000021110241
:10F220000504FFFF003E7FFF4E75455649633031B0
:10F23000000000007676764E75455649636363009C
:10F240007676764E754556496330346565767676C2
:10F250007676767676000000496E76616C69642079
:10F26000636F6E66696720666F726D61740000007F
:10F27000496E76616C696420636865636B73756D54
:10F2800000000000496E76616C696420636F6E66F1
:10F2900069672073697A6500496E76616C696420DC
:10F2A000636F6E6669672076657273696F6E0000C2
:10F2B000496E76616C6964206D6573736167652E54
:10F2C00000000000653030006330300053656E642C
:10F2D000696E6720636F6E6669672E2E2E000000D0
:10F2E000436F6E6669672073656E742E00000000C0
:10F2F0006330330053656E64696E672076657273A0
:10F30000696F6E2E00000000633032005265636545
:10F310006976696E6720636F6E6669672E2E2E00B0
:10F320004E657720636F6E666967207361766564EA
:10F330002E000000556E6B6E6F776E206D657373D7
:10F340006167652E0000000065303100436F6E6616
:10F350006967206D676D7400506F776572206F6606
:10F3600066204E7545564900746F206578697400B3
:10F3700052656164792E00FF348004404000000033
:10F380001211FFFFFF02020000001310FFFFFF0237
:10F3900002000000180000003480044080000000DB
:10F3A0001EFFFFFFFF02000000001DFFFFFFFF0226
:10F3B0000000000019000000000000000000000034
:10F3C00015720000D97100008D710000D571000028
:10F3D000917100009D710000BD71000000010307E4
:10F3E0000F1F3F7F2200FF2100FFFFFF0080C0E0D2
:10F3F000F0F8FCFE00000000000000006D9100002D
:10F40000C99500008D710000997B0000317C0000DF
:10F41000158A0000C9890000FD890000D589000017
:10F42000E9890000E5880000158A00003D8A000097
:10F430002D7E000075860000118600000D8B0000F7
:10F44000198A0000718B0000118C0000DA02818F94
:10F45000DA1281FF000060000000000000000000E0
:10F460000000000000E000000000000000000000BC
:10F4700000000001E00000000000000000000000AB
:10F48000000001F00000000000000000000000008B
:10F490000003F00000000000000000000000000079
:10F4A00007F000000000000000000000000000075E
:10F4B000F8000000000000000000000000000FF84D
:10F4C00000000003C0007E000001E0007F0FF80094
:10F4D000000003C000FE000001E000FFEFF80000A4
:10F4E0000003C000FE000001E000FFFFF800000084
:10F4F00003C000F00000000F007FFE7FC00000038B
:10F50000C000F00000000F003FFE7FF83FF1FBCF8E
:10F51000FCFEF3BC3DEFE01FFE7FFF7FFBFFDFFE45
:10F52000FEFFBC3DEFE01FC6FFFF7FFBFFDFFEFEDF
:10F53000FFBC3DEFE00FE3C7FE787BC3DE1EF0FFAC
:10F54000BC3DEF0007FF87FC787BC3DE1EF0F83C74
:10F550003DEF0001FFFFF0007BC3C01EF0F03C3D1B
:10F56000EF0001F37FE03FFBC3CFFEF0F03C3DEF47
:10F570000003E33F807FFBC3DFFEF0F03C3DEF0084
:10F5800007E73C00787BC3DE1EF0F03C3DEF000750
:10F59000FFBE00787BC3DE1EF0F03C3DEF0007FFAE
:10F5A000FE00787BC3DE1EF0F03C3DEF000FFFFE57
:10F5B000007FFBFFDFFEF0F03FFDEFE00FFFFF00FD
:10F5C0007FFBFFDFFEF0F03FFDEFE00FF9FF003EB5
:10F5D00079F9CF9EF0F01F3DE7E01FF1FF0000003A
:10F5E0000000000000000000001F80FF007FFFFF00
:10F5F000FFFFFFFFFFFFFFE01C007F007FFFFFFF1B
:10F60000FEB46D888D18E000001F007FFFFFFFFE35
:10F6100095AD7DB577E000000F007FFFFFFFFEA5F1
:10F62000AD9D8D19E0000006007FFFFFFFFEB5AD28
:10F63000EDB57EE0AED580A8D300408D2000A1C8F6
:10F64000DB40A4A62EAFFFFF0000000000018000F9
:10F650000000000000000000038000000000000027
:10F6600000000007C000000000000000000007C00C
:10F670000000000000000000000FC00000000000BB
:10F68000000000001FE00000000000000000001F5C
:10F69000E00000000000000000003FE0000000006B
:10F6A00000000000003FF00000000000000000002B
:10F6B0007FF0000000000000001FF87FF000000055
:10F6C000000000003FFE7FF0000000000000003F4F
:10F6D000FF7FF0000000000000001FFFFBE00000C3
:10F6E00000000000000FFFF9FFC000000000000054
:10F6F0000FFFF9FFF800000000000007FFF1FFFF17
:10F7000000000000000003FC73FFFF800000000009
:10F710000001FE3FFFFF80000000000000FF1E0F01
:10F72000FF000000000000007FFE1FFC0000000042
:10F730000000003FFFFFF8000000000000000FDFA6
:10F74000FFE0000000000000001F19FFC0000000E3
:10F75000000000003F3CFF00000000000000007EB1
:10F760007CF800000000000000007FFE7C0000002C
:10F770000000000000FFFFFC00000000000000008F
:10F78000FFFFFE0000000000000000FFFFFE000081
:10F79000000000000001FFEFFE000000000000007C
:10F7A00001FFCFFE0000000000000003FF07FE0085
:10F7B00000000000000003FC07FE00000000000045
:10F7C0000003F003FE00000000000000018000FEC6
:10F7D000000000000000000000007E0000000000AB
:10F7E00000000000003E00000000000000000000DB
:10F7F0000C000000000000078000FC000003C000B7
:10F800000000078001FC000003C000000007800129
:10F81000FC000003C0000000078001E00000001EA3
:10F82000000000078001E00000001E007FE3F79F5A
:10F83000F9FDE7787BDFC0FFF7FFBFFDFDFF787BB9
:10F84000DFC0FFF7FFBFFDFDFF787BDFC0F0F7876C
:10F85000BC3DE1FF787BDE00F0F787BC3DE1F0784E
:10F860007BDE0000F787803DE1E0787BDE007FF7FC
:10F87000879FFDE1E0787BDE00FFF787BFFDE1E0D9
:10F88000787BDE00F0F787BC3DE1E0787BDE00F0BE
:10F89000F787BC3DE1E0787BDE00F0F787BC3DE117
:10F8A000E0787BDE00FFF7FFBFFDE1E07FFBDFC01C
:10F8B000FFF7FFBFFDE1E07FFBDFC07CF3F39F3D7F
:10F8C000E1E03E7BCFC0000000000000000000002F
:10F8D00000FFFFFFFFFFFFFFFFFFFFC0FFFFFFFF76
:10F8E000FD68DB111A31C0FFFFFFFFFD2B5AFB6AD9
:10F8F000EFC0FFFFFFFFFD4B5B3B1A33C0FFFFFF75
:10F90000FFFD6B5BDB6AFDC0DA0281FF00000000D7
:10F91000000000006D910000C99500008D7100008D
:10F92000997B00004D9D0000158A0000C9890000E8
:10F93000FD890000D5890000E9890000E588000004
:10F94000158A00003D8A0000398A0000618A0000A3
:10F95000B98A00000D8B0000198A0000718B00002D
:10F96000118C000000000000003E5B4F5B3E3E6BD0
:10F970004F6B3E1C3E7C3E1C183C7E3C181C577D49
:10F98000571C1C5E7F5E1C00183C1800FFE7C3E795
:10F99000FF0018241800FFE7DBE7FF30483A060EA7
:10F9A0002629792926407F050507407F05253F5AEE
:10F9B0003CE73C5A7F3E1C1C08081C1C3E7F14225E
:10F9C0007F22145F5F005F5F06097F017F00668909
:10F9D000956A606060606094A2FFA29408047E044F
:10F9E0000810207E201008082A1C08081C2A080875
:10F9F0001E101010100C1E0C1E0C30383E38300635
:10FA00000E3E0E06000000000000005F0000000730
:10FA1000000700147F147F14242A7F2A122313085E
:10FA2000646236495620500008070300001C22413A
:10FA3000000041221C002A1C7F1C2A08083E0808DE
:10FA4000008070300008080808080000606000208E
:10FA5000100804023E5149453E00427F4000724971
:10FA60004949462141494D331814127F1027454515
:10FA700045393C4A4949314121110907364949492B
:10FA800036464949291E0000140000004034000099
:10FA90000008142241141414141400412214080202
:10FAA000015909063E415D594E7C1211127C7F4975
:10FAB0004949363E414141227F4141413E7F4949CA
:10FAC00049417F090909013E414151737F080808F6
:10FAD0007F00417F41002040413F017F08142241C7
:10FAE0007F404040407F021C027F7F0408107F3E21
:10FAF0004141413E7F090909063E4151215E7F098E
:10FB0000192946264949493203017F01033F4040F4
:10FB1000403F1F2040201F3F4038403F63140814DF
:10FB20006303047804036159494D43007F41414117
:10FB30000204081020004141417F040201020440F8
:10FB400040404040000307080020545478407F287C
:10FB50004444383844444428384444287F38545472
:10FB6000541800087E090218A4A49C787F08040495
:10FB70007800447D40002040403D007F1028440034
:10FB800000417F40007C047804787C0804047838C5
:10FB900044444438FC1824241818242418FC7C08F5
:10FBA000040408485454542404043F44243C404072
:10FBB000207C1C2040201C3C4030403C4428102825
:10FBC000444C9090907C4464544C4400083641006E
:10FBD0000000770000004136080002010204023CE8
:10FBE0002623263C1EA1A161123A4040207A3854B7
:10FBF0005455592155557941225454784221555430
:10FC0000784020545579400C1E5272123955555582
:10FC100059395454545939555454580000457C416D
:10FC20000002457D420001457C407D1211127DF0AD
:10FC3000282528F07C545545002054547C547C0AD7
:10FC4000097F4932494949323A4444443A324A48A0
:10FC500048303A4141217A3A42402078009DA0A0A4
:10FC60007D3D4242423D3D4040403D3C24FF2424F6
:10FC7000487E4943662B2FFC2F2BFF0929F620C015
:10FC8000887E090320545479410000447D41304866
:10FC9000484A32384040227A007A0A0A727D0D19A9
:10FCA000317D2629292F28262929292630484D400B
:10FCB00020380808080808080808382F10C8ACBA07
:10FCC0002F102834FA00007B000008142A14222286
:10FCD000142A14085500550055AA55AA55AAFF55CF
:10FCE000FF55FF000000FF00101010FF0014141457
:10FCF000FF001010FF00FF1010F010F0141414FC9F
:10FD0000001414F700FF0000FF00FF1414F404FCBB
:10FD1000141417101F10101F101F1414141F00109C
:10FD20001010F0000000001F101010101F10101015
:10FD300010F010000000FF10101010101010101024
:10FD4000FF10000000FF140000FF00FF00001F1064
:10FD5000170000FC04F414141710171414F404F41E
:10FD60000000FF00F714141414141414F700F7140F
:10FD70001414171410101F101F141414F41410105E
:10FD8000F010F000001F101F0000001F1400000002
:10FD9000FC140000F010F01010FF10FF141414FFFA
:10FDA000141010101F00000000F010FFFFFFFFFFF5
:10FDB000F0F0F0F0F0FFFFFF0000000000FFFF0F89
:10FDC0000F0F0F0F3844443844FC4A4A4A347E022D
:10FDD000020606027E027E026355494163384444AE
:10FDE0003C04407E201E2006027E020299A5E7A563
:10FDF000991C2A492A1C4C7201724C304A4D4D30D4
:10FE00003048784830BC625A463D3E494949007EF8
:10FE10000101017E2A2A2A2A2A44445F444440518F
:10FE20004A444040444A51400000FF0103E080FF43
:10FE3000000008086B6B083612362436060F090FCF
:10FE400006000018180000001010003040FF0101EB
:10FE5000001F01011E00191D1712003C3C3C3C0014
:10FE6000000000000D0AFFFF050E08090D0C060733
:10FE70000F0400130393050E08090D0C06070F0469
:10FE8000FFFFC585848687C4FFFF001303931A9282
:10FE900017FFFFFF6FF07F030370037813F0800FED
:10FEA000FBD070474008FE4340A004404408FE4396
:10FEB00044A004400018FE4300C004403000FE434C
:10FEC000309004403400FE43349004401C18FE433C
:10FED0001CC004401018FE4310C004400818FE4324
:10FEE00008C004400C18FE430CC004400C10FE4334
:10FEF0000CB004401010FE4310B004401810FE4334
:10FF000018B004401C10FE431CB004401410FE4303
:10FF100014B004400418FE4304C004400010FE4323
:10FF200000B004400008FE4300A004400408FE4363
:10FF300004A004400C08FE430CA004400808FE4343
:10FF400008A004401418FE4314C004401818FE43CF
:10FF500018C004400410FE4304B004400810FE43DF
:10FF600008B004401400FE43149004404C08FE43C3
:10FF70004CA004400420FE4304D004402410FE435F
:10FF800024B004402010FE4320B004402810FE435B
:10FF900028B004402C10FE432CB004400020FE4347
:10FFA00000D004404808FE4348A004401000FE432F
:10FFB00010900440090AFFFFFFFFFFFFFFFFFFFF54
:10FFC000FFFFFF0D00060807FFFF0E0FFF0CFFFFEE
:10FFD000FFFFFFFF0B05FFFF1519151900010000BA
:10FFE0002C91FF1F12000000000200005891FF1F1B
:10FFF0007300000000220100CC91FF1F21000000CF
:020000021000EC
:1000000000210100B491FF1F09000000000300005F
:10001000F091FF1F00000000010309044091FF1F41
:1000200000000000020309043C8FFF1F00000000D5
:1000300003030904F491FF1F00000000000000000A
:10004000000000000000000065787000FFFFFFFF67
:10005000000000000000E03F000000000000E0BFE2
:10006000763C7935EF39EA3D763C7935EF39EABDB2
:100070000000E0FE422EE63F0000E0FE422EE6BF1A
:100080001092FF1FF8B500BFF8BC08BC9E46704731
:1000900009E200003504000021330000514E000049
:0400A000096E0000E5
:0400A400F8B500BFEC
:1000A80038B5084B1C681C6054B1074D94FAA4F38A
:1000B800B3FA83F355F823309847631E1C40F5D1F3
:1000C80038BD00BFA0D004401C91FF1F38B5084BB5
:1000D8001C681C6054B1074D94FAA4F3B3FA83F377
:1000E80055F823309847631E1C40F5D138BD00BF32
:1000F800A0C00440FC90FF1F38B5084B1C681C606A
:1001080054B1074D94FAA4F3B3FA83F355F82330A6
:100118009847631E1C40F5D138BD00BFA0B004400D
:10012800CC90FF1F38B5084B1C681C6054B1074DB4
:1001380094FAA4F3B3FA83F355F823309847631E6F
:100148001C40F5D138BD00BFA0A004407C90FF1F23
:1001580038B5084B1C681C6054B1074D94FAA4F3D9
:10016800B3FA83F355F823309847631E1C40F5D142
:1001780038BD00BFA09004404490FF1F000000005D
:100188000000F04100200000000102070B010207F7
:100198000B4A14003200000001000000002000009B
:1001A8000020000000100000AB0A0000000800005A
:1001B80066060000550500009204000000040000D7
:1001C8008E03000033030000E8020000AB020000C9
:1001D800240000000020000002000200FBFFFFFFD7
:1001E8000000000000000000000000000000000007
:1001F80000000000000000000000000000000000F7
:100208000C000000140500000C000200FFFFFFFFB7
:1002180028E70000B8E70000D0E70000A0E70000EA
:1002280040E7000000000000E8EF0000D4EF000005
:10023800A089FF1F01001E00000000000000000050
:10024800000000000000000000000000F4F10000C1
:10025800F4F10000B09BFF1F000001000100000046
:100268000000000000000000000000000000000086
:1002780098F1000098F10000A09CFF1F0000030007
:100288000000000000000000000000000000000066
:1002980000000000C4F10000C4F10000529BFF1FE1
:1002A800030004000000000000000000000000003F
:1002B8000000000000000000010000000000000035
:1002C80000000000ACF00000ACF00000709BFF1FC5
:1002D8000000010001000000000000000000000014
:1002E800000000000000000080F0000080F0000026
:1002F800809AFF1F000009000100000000000000B4
:10030800000000000000000000000000B8F000003D
:10031800B8F000009E9AFF1F01000A0001000000CB
:1003280000000000000000000000000000000000C5
:1003380000F00000D4EF0000AA89FF1F00000400AD
:1003480000000000000000000000000000000000A5
:1003580000000000B8F10000B8F10000B29BFF1FD8
:100368000000010000000000000000000000000084
:10037800000000000000000058F0000058F00000E5
:10038800829BFF1F00000C0000000000000000001E
:1003980000000000000000000000000000F2000063
:1003A80000F20000189BFF1F00000600000000007C
:1003B8000000000000000000000000000100000034
:1003C800E889FF1F388DFF1F888BFF1F808CFF1F58
:1003D800308AFF1FF08AFF1F648EFF1FD08EFF1F19
:1003E8000C8AFF1FCC8CFF1F00000000DCF100000E
:1003F800DCF10000A89AFF1F0000010001000000C6
:1004080000000000000000000000000000000000E4
:1004180064F0000064F00000249BFF1F000002004D
:1004280001000000000000000000000000000000C3
:1004380000000000C4F00000C4F000007C9BFF1F17
:1004480000007F0001000000000000000000000024
:1004580000000000000000008CF000008CF000009C
:10046800749BFF1F00001E00010000000000000038
:10047800000000000000000000000000F4EF000091
:10048800D4EF00007889FF1F01000C000000000075
:100498000000000000000000000000000000000054
:1004A80034F0000034F00000F89BFF1F0000460005
:1004B8000000000000000000000000000000000034
:1004C800E48DFF1FD08BFF1FA88AFF1F608AFF1FC4
:1004D800188FFF1F18ED0000F48BFF1F848AFF1F81
:1004E80000000000D0F10000D0F10000809BFF1F49
:1004F80000000100010000000000000000000000F2
:10050800000000000000000008F2000008F20000EF
:10051800C29BFF1F00001800000000000000000040
:1005280000000000000000000400000000000000BF
:1005380090F1000090F10000C88CFF1F04005000EB
:1005480000000000000000000000000000000000A3
:1005580000000000B4EF0000B4EF0000F69BFF1F9E
:100568000000010001000000000000000000000081
:1005780000000000000000004CF000004CF00000FB
:10058800AE9BFF1F000004000100000000000000F7
:10059800000000000000000000000000E8F100007A
:1005A800E8F10000149BFF1F00000100010000009B
:1005B800000000000000000000000000F48EFF1F93
:1005C80044EE0000CC8AFF1FF08CFF1F188CFF1F21
:1005D800C489FF1F9C8DFF1FC08DFF1FA48CFF1FA8
:1005E800388BFF1F78ED0000B8EC00006CED0000C0
:1005F80000ED0000C4EC00000CED0000000000005D
:10060800DCEF0000D4EF00007A89FF1F0100110021
:1006180000000000000000000000000000000000D2
:1006280000000000C8EF0000D4EF0000A889FF1FF9
:1006380001001E0000000000000000000000000093
:100648000000000000000000D0F00000D0F0000022
:10065800849AFF1F00000A0001000000000000004B
:10066800000000000000000094EC0000ECED000029
:1006780070E80000DCEC00003CED000020EE00001B
:100688000000000028F0000028F00000F09AFF1F8A
:1006980000001D0000000000000000000000000035
:1006A80000000000AC8BFF1F148BFF1F148DFF1F71
:1006B800888EFF1FD0EC00003C8CFF1F208EFF1F90
:1006C800AC8EFF1F00000000B0F10000B0F1000088
:1006D8005A9BFF1F000001000000000000000000FE
:1006E80000000000000000000000000040F00000D2
:1006F80040F00000709AFF1F00007F00010000001A
:1007080000000000000000000000000000000000E1
:100718001CF000001CF00000A09AFF1F00007F00E2
:1007280001000000000000000000000000000000C0
:1007380000000000A4F10000A4F10000EE9BFF1FE0
:1007480000000100000000000000000000000000A0
:100758000000000000000000C0EF0000C0EF000033
:10076800829AFF1F00000200010000000000000044
:10077800000000000000000000000000A0F00000E1
:10078800A0F00000509BFF1F00007F000100000048
:1007980000000000000000000000000016034E00EA
:1007A800750045005600490020004D0049004400EE
:1007B80049000000C0F3000000000000E80300004A
:1007C800000000000060064078F300000000000010
:1007D8000000000000000000000000000000000011
:1007E8000000000000000000000000000000000001
:1007F80000000000000000000000000000000000F1
:1008080000000000000000000000000000000000E0
:1008180000000000000000000000000000000000D0
:10082800C0F3000000000000E80300000000000022
:100838000070064098F3000000000000000000006F
:1008480000000000000000000000000000000000A0
:100858000000000000000000000000000000000090
:100868000000000000000000000000000000000080
:100878000000000000000000000000000000000070
:100888000000000000000000000000009D9400002F
:100898009D9400009D9400009D9400000A040000AF
:1008A80034A1FF1FD99D0000D99D0000D99D0000EB
:1008B800D99D0000D99D0000D99D0000D99D000058
:1008C800D99D0000D99D0000D99D0000D99D000048
:1008D800D99D0000D99D0000D99D0000D99D000038
:1008E800D99D0000D99D0000D99D0000D99D000028
:1008F800D99D0000D99D0000D99D0000D99D000018
:10090800D99D0000D99D0000D99D0000D99D000007
:10091800D99D0000D99D0000D99D0000D99D0000F7
:10092800D99D0000D99D0000D99D0000D99D0000E7
:10093800D99D0000D99D0000D99D0000D99D0000D7
:10094800D99D0000D99D0000D99D0000D99D0000C7
:10095800D99D0000D99D0000D99D0000D99D0000B7
:10096800D99D0000D99D0000D99D0000D99D0000A7
:10097800D99D0000D99D0000D99D0000D99D000097
:10098800D99D000008000000FFFFFFFF12011001C1
:1009980000000040C0168504750201020301000032
:1009A80018035400650065006E0073007900640048
:1009B800750069006E006F0009027300020100C033
:1009C8003209040000020103000007240100012588
:1009D8000006240201010006240202020009240381
:1009E80001030102010009240302040101010009B5
:1009F80005040240000000000525010101090583E6
:100A0800024000000000052501010309040100025D
:100A180003000000092111010001222100070581BE
:100A280003400001070502032000020006C9FF0970
:100A380004A15C7508150026FF0095400975810220
:100A480095200976910295040976B102C00000004C
:100A5800040309040C03000000000000000000006B
:100A6800000000000000000000000100000000007D
:100A780000000000FC94FF1F6495FF1FCC95FF1F2A
:100A8800000000000000000000000000000000005E
:100A9800000000000000000000000000000000004E
:100AA800000000000000000000000000000000003E
:100AB800000000000000000000000000000000002E
:100AC800000000000000000000000000000000001E
:100AD800000000000000000000000000000000000E
:100AE80000000000000000000000000000000000FE
:100AF80000000000000000000000000000000000EE
:100B080000000000000000000000000000000000DD
:100B180000000000000000000100000000000000CC
:100B28000E33CDAB34126DE6ECDE05000B00000091
:100B380000000000000000000000000000000000AD
:100B4800000000000000000000000000000000009D
:100B5800000000000000000000000000000000008D
:100B6800000000000000000000000000000000007D
:100E980000000000000000001092FF1F000000008A
:100EA800000000003C96FF1F3C96FF1F4496FF1F62
:100EB8004496FF1F4C96FF1F4C96FF1F5496FF1F2A
:100EC8005496FF1F5C96FF1F5C96FF1F6496FF1FDA
:100ED8006496FF1F6C96FF1F6C96FF1F7496FF1F8A
:100EE8007496FF1F7C96FF1F7C96FF1F8496FF1F3A
:100EF8008496FF1F8C96FF1F8C96FF1F9496FF1FEA
:100F08009496FF1F9C96FF1F9C96FF1FA496FF1F99
:100F1800A496FF1FAC96FF1FAC96FF1FB496FF1F49
:100F2800B496FF1FBC96FF1FBC96FF1FC496FF1FF9
:100F3800C496FF1FCC96FF1FCC96FF1FD496FF1FA9
:100F4800D496FF1FDC96FF1FDC96FF1FE496FF1F59
:100F5800E496FF1FEC96FF1FEC96FF1FF496FF1F09
:100F6800F496FF1FFC96FF1FFC96FF1F0497FF1FB8
:100F78000497FF1F0C97FF1F0C97FF1F1497FF1F65
:100F88001497FF1F1C97FF1F1C97FF1F2497FF1F15
:100F98002497FF1F2C97FF1F2C97FF1F3497FF1FC5
:100FA8003497FF1F3C97FF1F3C97FF1F4497FF1F75
:100FB8004497FF1F4C97FF1F4C97FF1F5497FF1F25
:100FC8005497FF1F5C97FF1F5C97FF1F6497FF1FD5
:100FD8006497FF1F6C97FF1F6C97FF1F7497FF1F85
:100FE8007497FF1F7C97FF1F7C97FF1F8497FF1F35
:100FF8008497FF1F8C97FF1F8C97FF1F9497FF1FE5
:101008009497FF1F9C97FF1F9C97FF1FA497FF1F94
:10101800A497FF1FAC97FF1FAC97FF1FB497FF1F44
:10102800B497FF1FBC97FF1FBC97FF1FC497FF1FF4
:10103800C497FF1FCC97FF1FCC97FF1FD497FF1FA4
:10104800D497FF1FDC97FF1FDC97FF1FE497FF1F54
:10105800E497FF1FEC97FF1FEC97FF1FF497FF1F04
:10106800F497FF1FFC97FF1FFC97FF1F0498FF1FB3
:101078000498FF1F0C98FF1F0C98FF1F1498FF1F60
:101088001498FF1F1C98FF1F1C98FF1F2498FF1F10
:101098002498FF1F2C98FF1F2C98FF1F3498FF1FC0
:1010A8003498FF1F3C98FF1F3C98FF1F4498FF1F70
:1010B8004498FF1F4C98FF1F4C98FF1F5498FF1F20
:1010C8005498FF1F5C98FF1F5C98FF1F6498FF1FD0
:1010D8006498FF1F6C98FF1F6C98FF1F7498FF1F80
:1010E8007498FF1F7C98FF1F7C98FF1F8498FF1F30
:1010F8008498FF1F8C98FF1F8C98FF1F9498FF1FE0
:101108009498FF1F9C98FF1F9C98FF1FA498FF1F8F
:10111800A498FF1FAC98FF1FAC98FF1FB498FF1F3F
:10112800B498FF1FBC98FF1FBC98FF1FC498FF1FEF
:10113800C498FF1FCC98FF1FCC98FF1FD498FF1F9F
:10114800D498FF1FDC98FF1FDC98FF1FE498FF1F4F
:10115800E498FF1FEC98FF1FEC98FF1FF498FF1FFF
:10116800F498FF1FFC98FF1FFC98FF1F0499FF1FAE
:101178000499FF1F0C99FF1F0C99FF1F1499FF1F5B
:101188001499FF1F1C99FF1F1C99FF1F2499FF1F0B
:101198002499FF1F2C99FF1F2C99FF1F3499FF1FBB
:1011A8003499FF1F3C99FF1F3C99FF1F4499FF1F6B
:1011B8004499FF1F4C99FF1F4C99FF1F5499FF1F1B
:1011C8005499FF1F5C99FF1F5C99FF1F6499FF1FCB
:1011D8006499FF1F6C99FF1F6C99FF1F7499FF1F7B
:1011E8007499FF1F7C99FF1F7C99FF1F8499FF1F2B
:1011F8008499FF1F8C99FF1F8C99FF1F9499FF1FDB
:101208009499FF1F9C99FF1F9C99FF1FA499FF1F8A
:10121800A499FF1FAC99FF1FAC99FF1FB499FF1F3A
:10122800B499FF1FBC99FF1FBC99FF1FC499FF1FEA
:10123800C499FF1FCC99FF1FCC99FF1FD499FF1F9A
:10124800D499FF1FDC99FF1FDC99FF1FE499FF1F4A
:10125800E499FF1FEC99FF1FEC99FF1FF499FF1FFA
:10126800F499FF1FFC99FF1FFC99FF1F049AFF1FA9
:10127800049AFF1F0C9AFF1F0C9AFF1F149AFF1F56
:10128800149AFF1F1C9AFF1F1C9AFF1F249AFF1F06
:10129800249AFF1F2C9AFF1F2C9AFF1F349AFF1FB6
:0C12A800349AFF1F00000200FFFFFFFF50
:00000001FF
